:020000041000EA
:10000000002008205D0100101301001015010010F0
:100010001101001011010010110100101101001058
:100020001101001011010010110100101701001042
:100030001101001011010010190100101B01001026
:100040001D0100101D0100101D0100101D010010F8
:100050001D0100101D0100101D0100101D010010E8
:100060001D0100101D0100101D0100101D010010D8
:100070001D0100101D0100101D0100101D010010C8
:100080001D0100101D0100101D0100101D010010B8
:100090001D0100101D0100101D0100101D010010A8
:1000A0001D0100101D0100101D0100101D01001098
:1000B0001D0100101D0100101D0100101D01001088
:1000C0001D0100101D0100101D0100101D01001078
:1000D0001D0100101D0100101D0100101D01001068
:1000E0001D0100101D0100101D0100101D01001058
:1000F0001D0100101D0100101D0100101D01001048
:100100001D0100101D0100101D0100101D01001037
:1001100000BE00BE00BE00BE00BE00BEEFF3058004
:10012000103800BEF2EB88713428011060280110ED
:10013000A801001090A31AE7D3DEFFFF42012110AF
:10014000FF01000094370100793512AB4FF0000039
:100150002049086006C881F3088810474FF05040D6
:10016000006810B14FF00000F2E70FA40ECC002998
:1001700002D000F015F8F9E71749184A002000E00E
:1001800001C19142FCD1002080F30A8814498847BC
:10019000144988471449884700BEFDE701C901C2D8
:1001A0009A42FBD3704700BF602801101001002065
:1001B0007C110020CC38011000000820000008202D
:1001C000CC380110001008200010082000000000AA
:1001D0007047000008ED00E07C110020E0370020AF
:1001E000CD4F001059130010914F0010F8B500BF0B
:1001F000064B0749C91A891048BF0131491003D07D
:10020000044B0BB101481847704700BF7C11002018
:100210007C1100200000000008B5054B1BB105490A
:100220000548AFF30080BDE80840FFF7E1BF00BF1D
:10023000000000009432002058B20010036870B52E
:1002400004461BB101221343374E1847374A384B37
:10025000384992ED007A93ED006AD1ED007AC7EE4D
:10026000876A87EE867A344A344BC2ED006A83EDA2
:10027000007A334D2C4E01F091FF002210F57A7078
:1002800041F10001C5E900012660E2B9012070BD1D
:100290002C4E2D4D066001F081FFD5E900239042E0
:1002A0009941F3D34FF050431B68012B35D0012205
:1002B000264B1A60264A136801330B2B13601CDD92
:1002C0001F4D194ED7E701F069FF1D4DD5E90023F9
:1002D00090429941DAD34FF050431B68012B1FD055
:1002E00001221A4B1A601B4B1B68002BC3D0002243
:1002F00013461749144D134E0A60174A1360012222
:10030000164B1A6001F04AFF154B1B68266018183F
:1003100041EBE371C5E90001B8E7124A1360C9E790
:10032000104A1360DFE700BF880200107009002048
:100330006C090020DC250020E4250020E0250020B9
:10034000B813002090020010B0130020D03200201B
:1003500000260020280A0020D02500206009002067
:1003600074090020D432002038B57B4D2C68002C55
:1003700000F0A68044F001042047784B784A9B693E
:100380002A609A0600F182804FF050431B68012BCF
:1003900000F0BD800122734B1A60734BB3F900303B
:1003A0007F2B00F0AD806D4A936913F02003FBD1E1
:1003B0007F206E4910600A68013A00F19F800A6050
:1003C000632A40F38F80002302202B6038BD634BEB
:1003D000674A9B692A609B0658D44FF050431B68BC
:1003E000012B00F09E8001225E4B1A60614A5E4B39
:1003F0001178B3F900308B4200F08C80574A936932
:1004000013F02003FBD10D29116000F08D807F29AE
:1004100071D0564803685A1C02605748C154CFE750
:100420004E4B564A9B692A6098062FD44FF0504392
:100430001B68012B5CD001224A4B1A604A4BB3F96E
:1004400000300A2B00F08180444A93699B06FCD45B
:100450000A231360B7E7414B494A9B692A609C060F
:1004600014D44FF050431B68012B6BD001223D4B3D
:100470001A603D4BB3F90030202B5CD0374A9369AA
:100480009906FCD42021364B11602B60012038BD29
:10049000324B3C4A9B692A60D806F7D44FF0504350
:1004A0001B68012B21D001222E4B1A602B4A936925
:1004B000D906FCD411682E4B2E4A2B601170E5E74B
:1004C000642221462C4805F045FF284B234A1C6036
:1004D0009369D90606D49369DB06FCD41368936943
:1004E000DC06F8D5274B2B60D0E7274A1360DDE701
:1004F000254A1360A2E7224B2B60C7E70B60F1E7A8
:10050000164A93699B06FCD40D2313604BE71E4AE1
:10051000136042E7114A93699C06FCD40D231360D3
:100520006CE7194A136061E7104A13481168134ACF
:1005300043542A60AAE7094A93699806FCD40D231C
:1005400013609BE7104A136093E7044A9369990686
:10055000FCD40D23136077E74833002000000740E8
:100560007A030010D0320020D4370020CC32002093
:10057000CE030010DE370020E432002020040010FB
:100580005604001090040010D43200202DE9F84FDA
:100590003F4B1F68002F78D13E4BD3F80080B8F155
:1005A000000F1CD13C4E47463C4CDFF8F4903368BA
:1005B00011E000233A4D03EB430309EB8303284684
:1005C0009B6898472368326801339342236005F1A2
:1005D0000C05F0DB1346002B2760EADCFEE7B8F1E0
:1005E000010F01D0BDE8F88F2C4C2B4EDFF8B090F6
:1005F000DFF8BC802B4DDFF8BCA0D8F800303268A3
:100600000133002AC8F80030276000DCFEE7DFF87D
:1006100090B02F6001F0C2FD2368CAE9000103EB2E
:10062000430309EB83039B68584698472B68012BCB
:1006300008D0236832680133934223600BF10C0B1E
:10064000DBDAE6E72268184951F82230013341F835
:10065000223001F0A3FD8E46D4F800B0134BDAF837
:10066000041053F83B2003EBCB0CDAF80030D31A1C
:10067000DCF8042062EB01021B180C4842EB0E026E
:1006800040F83B30CCF80420B7E747F00107384783
:10069000D8320020E03200204C330020F825002022
:1006A00054330020D03200205834002000130020A2
:1006B00050340020A01300202DE9F84F3F4B1F6855
:1006C000002F78D13E4BD3F80080B8F1000F1CD139
:1006D0003C4E47463C4CDFF8F490336811E0002371
:1006E0003A4D03EB430309EB830328469B68984785
:1006F0002368326801339342236005F10C05F0DB77
:100700001346002B2760EADCFEE7B8F1010F01D0A9
:10071000BDE8F88F2C4C2B4EDFF8B090DFF8BC8092
:100720002B4DDFF8BCA0D8F8003032680133002A26
:10073000C8F80030276000DCFEE7DFF890B02F60DB
:1007400001F02CFD2368CAE9000103EB430309EB28
:1007500083039B68584698472B68012B08D0236871
:1007600032680133934223600BF10C0BDBDAE6E7CE
:100770002268184951F82230013341F8223001F043
:100780000DFD8E46D4F800B0134BDAF8041053F880
:100790003B2003EBCB0CDAF80030D31ADCF8042052
:1007A00062EB01021B180C4842EB0E0240F83B3092
:1007B000CCF80420B7E747F001073847DC320020C7
:1007C000E032002050330020FC250020CC330020F4
:1007D000D4320020803400205013002054340020F4
:1007E000A8130020022238B53049314B0C68012093
:1007F0001A64304900F0F4FF0121084600F0CAFFF6
:100800004FF050422C4B1268996A012A0C445C61EB
:1008100025D02A490B68092B06DD0022284B1A60D7
:10082000BDE83840FFF7B2BE0024264A03EB430080
:1008300085005451244D02EB800043608560581CB4
:100840000A280860E9D002330B6000EB40039900EE
:10085000545002EB83021D4BC2E90103DDE71C4942
:100860000B68092B06DD00221A4B1A60BDE83840E0
:10087000FFF722BF0024184A03EB430085005451C0
:10088000114D02EB800043608560581C0A28086007
:10089000E9D002330B6000EB40039900545002EBA7
:1008A00083020A4BC2E90103DDE700BF64090020AF
:1008B00000200B401D13001000000B404C330020A3
:1008C000D832002054330020890B00103D02001064
:1008D00050330020DC320020CC3300200000000028
:1008E00070B57D4C0C2004F0A3FC052201212046AC
:1008F00004F062FD794804F05FFDDC21784804F0E3
:100900005BFDEF21774804F057FD774D774804F001
:1009100053FD00220321204604F04EFD284604F03A
:100920004BFD734B7348197804F046FD19220321DF
:10093000204604F041FD704B7048196804F03CFDFE
:1009400032220321204604F037FD6D4B6D481968B3
:1009500004F032FD00220421204604F02DFD6A4BF4
:100960006A4E18680AF040FC0B460246684804F0DC
:1009700023FD19220421204604F01EFD654B186852
:100980000AF032FC0B460246634804F015FD3222A1
:100990000421204604F010FD604B186807EE900A11
:1009A000F8EEE77A17EE900A0AF01EFC48A3D3E9A6
:1009B000002301F045FF0B460246594804F0FCFCB9
:1009C00000220521204604F0F7FC564BD6ED007AB4
:1009D00093ED007AC7EE277A17EE900A0AF004FC2E
:1009E0000B460246504804F0E7FC19220521204638
:1009F00004F0E2FC4D4BD6ED007A93ED007AC7EEA1
:100A0000277A17EE900A0AF0EFFB0B460246484899
:100A100004F0D2FC32220521204604F0CDFC454BE7
:100A200018680AF0E1FB0B460246434804F0C4FC98
:100A300000220621204604F0BFFC404B18680AF053
:100A4000D3FB0B4602463E4804F0B6FC19220621B1
:100A5000204604F0B1FC3B4B3B48196804F0ACFC69
:100A600000220721204604F0A7FC384804F0A4FC2B
:100A7000374804F0A1FC374804F09EFC364804F0E7
:100A80009BFC364804F098FC354804F095FC35484A
:100A900004F092FC344804F08FFC344804F08CFCE1
:100AA000334804F089FC334804F086FC324804F0F3
:100AB00083FC324804F080FC314804F07DFC31486E
:100AC00004F07AFC2846BDE8704004F075BC00BF15
:100AD0000000000080842E4158B2001064B2001063
:100AE0006CB2001078B20010D0B2001084B20010C6
:100AF0008C090020D8B20010D4250020ECB20010E0
:100B00008409002004B300107C090020240A00207E
:100B10001CB300108009002030B3001074090020BD
:100B200044B30010700900205CB300106C09002071
:100B300070B30010DC25002084B300106809002089
:100B400098B30010200A0020B0B30010C0B300100A
:100B5000C8B30010F0B3001004B4001028B40010A3
:100B600060B4001090B40010BCB40010E4B40010E5
:100B700010B5001030B500106CB500108CB5001029
:100B8000ACB50010ECB300102DE9F0472DED028B51
:100B90000368044682B0002B5AD0A54D2560FFF7AC
:100BA000E3FB012805D8002002B0BDEC028BBDE8B4
:100BB000F087A049A04805F01FFC01469F4805F0BA
:100BC0005DFD9C49002005F017FC01469C4805F09E
:100BD00055FD9849002005F00FFC0146994805F0A5
:100BE0004DFD9449002005F007FC0146964805F0AC
:100BF00045FD9649914805F063FCF8B194498F484A
:100C000005F05EFC40BB934B1860934E3368E3B134
:100C10000023336000221721904804F0CDFB904858
:100C200004F0CAFB002217218C4804F0C5FB8D4854
:100C300004F0C2FB00228C4B1A60AFE70122854B07
:100C4000854E1A603368002BE2D1FFF749FEDFE7DB
:100C5000FFF746FE764DDDE78449784805F030FC25
:100C600000285CD08249754805F02AFC002850D045
:100C70008049724805F024FC002856D07E496F4810
:100C800005F01EFC002800F082807C496B4805F0CE
:100C900017FC002800F093807949684805F010FCA3
:100CA000002800F09A807749644805F009FC064660
:100CB000002800F0AD807449604805F001FC002870
:100CC00000F0498171495D4805F0FAFB002800F009
:100CD00048816F49594805F0F3FB002800F0548122
:100CE0006C49564805F0ECFB002840F0438101AA0E
:100CF0006949534805F080FA01980AF075FA4AA349
:100D0000D3E9002301F076FD01F01AFE634E306056
:100D10007BE7634A63494A4805F06EFA75E7624A21
:100D20006049474805F068FA6FE7604E5D49324612
:100D3000434805F061FA5E4BDFF898911B685D4F00
:100D4000C3F100083368002603FB03F307EE903A73
:100D5000B8EEE78A09F5487A07EE908AF8EEE77A66
:100D600067EEE77AC7EE887A17EE900A0AF03CFA47
:100D700002F093FA32463B4601F03CFD01F0AEFD35
:100D800049F8040BCA4508F10108E5D13DE701AA7D
:100D900041492B4805F030FA474A484B92ED007A1A
:100DA000D3ED006A464A474BDDED017A67EE877A5C
:100DB00086EEA77AC2ED007A83ED007A25E701AAD4
:100DC00035491F4805F018FA3B4A3C4B92ED007A32
:100DD000D3ED006A3C4A3D4BE6E72F4901AA18488B
:100DE00005F00AFA384A364B92ED007ADDED017AC9
:100DF00093ED006AC7EE876A87EE867A2F49334AF9
:100E0000304BC1ED007AC2ED006A83ED007AFCE65A
:100E100021490B4801AA05F0EFF9DFF8BCA00198C1
:100E20002B4FCAF800005BE00000000080842E41D8
:100E30009C0B0010BCB30010E4320020942500206D
:100E4000501500206015002070150020ECB5001032
:100E5000F4B50010280A00208015002058B20010B8
:100E6000C8B50010E0B5001048330020FCB50010F4
:100E700008B6001014B6001020B6001030B60010EE
:100E80003CB6001044B600104CB6001054B600102A
:100E90005CB6001064B600102CB600107409002077
:100EA000D425002004B600108C09002084090020FD
:100EB0008809002000409F40240A0020DC250020F3
:100EC00070090020E42500206C090020E0250020A6
:100ED00088150020442C002068090020DAF8000062
:100EE0000AF082F939A3D3E9002301F083FC07EE6D
:100EF000906AF8EEE77A804617EE900A89460AF083
:100F000073F902460B464046494601F073FC002245
:100F1000234B01F06FFC01F001FF224B002201F096
:100F200069FC01F0DBFC47F8040B04F085FF434249
:100F3000C3F30A03C0F30A0058BF5842A0F580600B
:100F400007EE900AF8EEE77A0136B6F5807FC7ED36
:100F5000FF7AC3D159E6144A1449154805F04CF9F3
:100F600053E601AA1349124805F046F9124B019ABB
:100F70001A604AE600221621104804F01DFA1048B3
:100F800004F01AFA0F4E43E601AA0A49084805F090
:100F900033F90D4B019A1A6037E600BFAFF30080BA
:100FA0000000703F00408F40200A002004B600106F
:100FB000501500202CB600107C09002058B20010FB
:100FC0006CB6001080150020800900201F85EB51B1
:100FD000B81E19402DE9F04FAD4885B00368002BCD
:100FE00040F0B4804FF0320CAA4FDFF81CB3D7EDBD
:100FF000007ADBF800E0A84BA848DFF810830393E1
:101000000CFB0EFC1B68009001930EF10100D8F858
:101010000010A34BA34ADFF8F892A34CA34E029012
:10102000D3F800A0A2489FEDA37A00EB8A00D0ED90
:10103000006A77EEA67AF4EEC77AF1EE10FA00981D
:10104000D4ED005A00EB8100CCBF9FED9B7AB0EE4F
:10105000677AD0ED006A994887ED007A90ED006AD2
:10106000C8BFF0EE477A76EEE56A94ED007AA6EE18
:10107000867A84ED007A924D924895ED007AD4ED0F
:10108000006A27EE267A00688F4FA0F59C401F3833
:10109000604587ED007A4FEA810A04DC8B480078CE
:1010A000002800F0D6801C688948DFF868C200EB91
:1010B0008400884C90ED005A97ED006AD4ED004A08
:1010C000854836EE646AD0ED006ADCED005ADFF840
:1010D00048C2E5EE066A9CED007A35EE877AC6EDE9
:1010E000006ABDEEC77AD6F800C0C4F800C03C68FC
:1010F000046017EE100A70456ADDFDEEE77A17EE20
:10110000900A99ED007A9FED756A754CC7EE066AF4
:101110002468FDEEE55A00EB0420724C04EB8004D9
:10112000D4ED007A66EEA76A6F48C0ED006A15EE4E
:10113000900A704500F387806C48D0ED007A37EE56
:10114000677AF5EE007A66EEA76A48E00021544B14
:101150000160544A186852F820008842C0F2958015
:101160005A48634C0078246800287CD14B4C0146D7
:101170002546204600261C68013152F8244040F8DC
:10118000046B8C42F7DA00954FF0010C0021DFF878
:101190007C81DFED497AE6460220C8F800C0CDF830
:1011A00008C08C463C4DDFF860B1DFF864913E4CDE
:1011B0003E4EC4ED007ACBF80010C9ED007A7146BE
:1011C000C6ED007AE646334F03952860019027E785
:1011D0009FED397A4448F0EE476A80ED007AD6ED0B
:1011E000007A77EEA67A009D18685544C5ED007A1E
:1011F000FDEEE77A52F820401B688C4252F823300B
:10120000019A0CBF01210131934218BF134617EE1A
:10121000900A08BF0123039A18BF013300F58360C9
:101220001360344E344BC0F30B0040F4405089ED52
:10123000007A3080C8F800109860029BCBF800302C
:1012400005B0BDE8F08F2D48D0ED007A37EE277A53
:1012500077E72B4897ED007AD0ED006A27EE267AE3
:1012600087ED007A1FE74FF448760C4D254806FBC2
:1012700004002C461E6850F8047B52F826600131A9
:101280008E4244F8047BF5DA7DE7044900917BE760
:10129000600900208415002048340020AC34002070
:1012A000D0250020C009002090320020D037002037
:1012B000F009002000007F430000000080090020AA
:1012C0007C09002074090020D82500208C0900200A
:1012D00090090020883200208432002000007A45E6
:1012E000200A002088150020CC370020E0250020AF
:1012F000D4250020DC37002000000840E425002031
:1013000078090020042600204C34002044340020BA
:10131000CC250020700900206C09002010B54FF08A
:101320000103022443EC40400749084A084BCC63C0
:10133000916A1B680B445361FFF74CFE4FF00003AA
:1013400043EC404010BD00BF00300B4000000B409C
:1013500064090020000000002DE9F84F02242DED63
:10136000028B974D03F05EFF964804F025F828465F
:10137000954904F049F9954B6A685C602B68944F75
:10138000944E83F00F03224003F0CF033B60012112
:101390007260062000F038F90121072000F034F9CE
:1013A0000121052000F030F9204600F04BF94FF004
:1013B000010343EC44404FF00009874DB5EE008A2D
:1013C000DFED868A4C460026DFF830B2DFF830A227
:1013D000834F05F5C86809E00134C82CC8EDC88AF8
:1013E00009F1640908F1040800F0888004F024FD84
:1013F0004342C3F30A03C0F30A0058BF5842A0F5A2
:10140000806307EE903AF8EEE77A032CE5EC017A78
:101410004EDDDAF8003015ED035A03FB03F307EE57
:10142000103AB8EEC76A15ED047ADBF8002055EDE6
:10143000025AA21A37EE057A06EE902A37EE257A7E
:10144000F8EEE66A77EE277A66EEE66A67EE887A65
:10145000C6EE866AC5EDC77A16EE900A09F0C4FE9C
:1014600001F01BFF32463B4601F0C4F901F036FAA9
:101470000A2CC8F800000FDD152CADDCC9F57A7315
:1014800007EE903AF8EEE77AC8EDC87A013409F130
:10149000640908F10408A9E707EE909AF8EEE77AE4
:1014A00008F10408013409F16409C8EDC77A9DE721
:1014B000DBF80030E31A07EE903ADAF80030F8EE85
:1014C000E77A03FB03F307EE103A67EEE77AB8EE2C
:1014D000C77AC7EE877A17EE900A09F085FE01F009
:1014E000DCFE32463B4601F085F901F0F7F907EEE4
:1014F000909AC8F80000F8EEE77AC5E700240FF2EA
:10150000B809D9E90089374DDFF8F8A0DAF800000A
:1015100009F06AFE42464B4601F06CF907EE904A2C
:10152000F8EEE77A064617EE900A0F4609F05CFEE1
:1015300002460B463046394601F05CF900222A4B40
:1015400001F058F901F0EAFB284B002201F052F9B2
:1015500001F0C4F945F8040B04F06EFC4342C3F3F8
:101560000A03C0F30A0058BF5842A0F5806007EE96
:10157000900AF8EEE77A0134B4F5807FC5EDFF7A82
:10158000C4D104F0C5F81A4804F034F94FF05043C0
:101590001B680022012B08D0164B1A60FEF7F6FFDD
:1015A000BDEC028B0020BDE8F88F134B1A60FFF7EB
:1015B00083F8F5E7AFF300801F85EB51B81E1940A3
:1015C0000000084084B60010002D310100300840B2
:1015D0000010084000200840042600200000000001
:1015E00000008940881500200000703F00408F40B7
:1015F000E5070010D8320020DC32002088090020E6
:10160000840900206809002010B44FF480740C4B4A
:1016100053F8202003EB8003C00082F0400200F169
:10162000804003F5805C02F0C00200F5203003F535
:101630004053CCF8002041601C605DF8044B7047BB
:101640000480034030B44FF0000343EC440043EC0B
:10165000400005254FF480740B4BC20053F8201056
:1016600003EB800081F0400102F1804303F5203359
:1016700001F0C00200F5805100F540500A605D6045
:10168000046030BC704700BF048003400FB400B555
:1016900083B0049C074803F00DFE3CB105A9204629
:1016A000019103F045FC044803F004FE012003F01F
:1016B00057FC00BFB4B60010C4B6001070B5864623
:1016C000EFF3108572B6124CD4E8CF6F0120002ED4
:1016D000FAD1C4E8460F002EF6D1BFF35F8F4FF06A
:1016E000010CC80801F007030CFA03F31EF800C050
:1016F0001CEA030608D14CEA030C0EF800C0C4E84B
:101700008F6F85F3108870BD1046FFF7BFFF00BFD5
:101710003B150020044A1078431CDBB2182B28BF6D
:1017200010231370704700BF2C0A00204FF0E022F6
:10173000936843F000539360704700BF0021044B4F
:1017400003F12002C3E88F1F01339342FAD170479F
:10175000301500204FF0E0234FF08032C3F8002412
:10176000C3F80424C3F80824C3F80C24C3F81024D5
:10177000C3F81424C3F81824C3F81C24C3F8202485
:10178000C3F82424C3F82824C3F82C24C3F8302435
:10179000704700BF012300F01F029340400941B190
:1017A000800000F1604000F56140C0F880310360C6
:1017B0007047024A203042F82030704700E100E0D4
:1017C0000123064A410952F8212000F01F008340FE
:1017D000134214BF01200020704700BF00E100E069
:1017E000F8B50D46EFF3108772B6124ED6E8CF2F3C
:1017F0000123002AFAD1C6E8423F002AF6D1BFF3FE
:101800005F8F0D4B00F110049B680C4A53F8243095
:10181000934203D0994201D000F0A2FE064B9B6890
:1018200043F82450BFF35F8F0023C6E88F3F87F350
:101830001088F8BD3915002000ED00E01D010010F2
:101840002DE9F04F83B0EFF3108A72B6744ED6E8EC
:10185000CF2F0123002AFAD1C6E8423F002AF6D151
:10186000BFF35F8F6F4B00F110089B686E4A53F80F
:10187000285095423FD08D420C464AD06B4FEB1B0F
:101880002F2B38D801214FEA50194FEA890909F165
:10189000604909F5614900F01F0301FA03F0D9F826
:1018A0000030C9F8800000EA030BBFF35F8FEFF34D
:1018B0000581C9B279B3884577D125F0010EDEF8EC
:1018C00008C0644505D17CE0D3F808C0644532D037
:1018D0009E469EF9062002EB4203002A07EB830393
:1018E000F2DA644500F08180BBF1000F20D0C9F826
:1018F0008001C9F800004B4B9B6843F82850BFF3A8
:101900005F8F0023C6E88F3F8AF3108803B0BDE8DD
:10191000F08F1546EFE725F0010EDEF808C06445AC
:10192000D7D19EF906407346002C08DA154666E0CA
:10193000C9F88000DFE793F90640002C56DB04EB82
:10194000440C07EB8C0CDCF8082061009A609CF8D2
:101950000720DA719CF90620002A9A715DDBBCF839
:101960000420520504D502F5FF1202F5FF521F3282
:10197000521502F1020C4FF0040E0C2212FB04E28D
:1019800002EB4C026FF0070C3A44ACEB030C6244E0
:10199000C2F34A0242F460429A80254B21441A78ED
:1019A00007EB81011C708A719EE7CDE9000100F010
:1019B000D7FDDDE9000125F0010EDEF808C0644521
:1019C00087D19EF906407346002CB8DA194A1A4CA2
:1019D000D21A083AC2F30A316FEA01516FEA115183
:1019E00044EA5202DA8099807EE773460029EDD1FD
:1019F000FF228EF806204BF60152AEF804200C4C64
:101A00004AF6AA2294F800C01946C91B49414A4324
:101A1000120D83F806C0227066E74BF60152BBE751
:101A20003915002000ED00E01D010010300A0020F3
:101A3000DF3700206A0A002000F8FFFFF0B5EFF35F
:101A40000585EDB2EFF3108C72B62649D1E8CF2FA1
:101A50000123002AFAD1C1E8423F002AF6D1BFF3A0
:101A60005F8F214E40F0010EB4684AF6AA2354F865
:101A700025701E4A0446A41A644163431B0D774532
:101A80005BB21BD092F906409C421CD092F91240E6
:101A90009C4223D092F91E409C4221D092F92A40C8
:101AA0009C4208BF03240FD0114A002415781370FC
:101AB0008571C1E88F4F8CF31088F0BDB2680D4C72
:101AC00042F82540F0E7002404EB440402EB8402D2
:101AD000FF2494714BF601549480E5E70124F3E769
:101AE0000224F1E73915002000ED00E0300A002063
:101AF000DF3700201D010010014B0B4403607047CD
:101B00003015002070B5104C104DAC420ED2FF269F
:101B1000236863B1FFF7FEFD01462046FFF7ECFFA7
:101B2000A680BFF35F8F0834AC42F1D370BDFFF7DE
:101B3000F1FD01462046FFF7DFFF2671BFF35F8FFF
:101B40000834AC42E4D370BD6C1100207C1100203D
:101B50000D4B1A68EFF3108172B6D2E8CFCF012097
:101B6000BCF1000FF9D1C2E84C0FBCF1000FF4D169
:101B7000BFF35F8F00221B68C3E88F2F81F31088AB
:101B800040BF002000217047A83400200000000062
:101B90002DE9F04F2DED028B85B0EFF30583DBB21D
:101BA000103B9A0818BF01224FF0010103F0030017
:101BB00018BFAB4DAB4B08BFAB4D00EB820201FA37
:101BC00000FB53F8226005F541539FEDA38B019074
:101BD000C3F804B0CDF800B02AE0B388180440F18F
:101BE0008C80B379002B40F0D580B6F9081000291D
:101BF000C0F21581736901EB410103EBC103D3E925
:101C00000247B7F1FF3F08BFB4F1FF3F09D0019B86
:101C100005EB8301AB6A0A69D21AE31A934238BF13
:101C20000C61284600F0B2FAA042B941C0F2F78038
:101C3000B6F90840009B002CEB63CEDBD6F814907D
:101C400004EB440A284609EBCA07D7E902B800F0BA
:101C50009DFA584571EB0801BFDBB8F1000FC0F2E7
:101C6000C180D7E90431814A934200F0EA807A8842
:101C7000B6F9080092B242EA0040984702460B4685
:101C800052EA030100F0AE80002B80F2CE80BBEB65
:101C9000020B68EB030839F93A30C7E902B8002BA8
:101CA0009BDB716903EB430201EBC202D2E90270D4
:101CB000BB4578EB000C4FEA43028EDBB4462CF8B0
:101CC000083F0BE031F93230F446002B0DDB03EB1B
:101CD000430001EBC0005A00D0E90270BB451A4432
:101CE00078EB000001EBC20EECDA29F83A30ACF8E0
:101CF0000040B38818043FF574AF3369EFF31082E6
:101D000072B6D3E8CF0F01210028FAD1C3E8401FF3
:101D10000028F6D1BFF35F8F4FF6FF74B088002321
:101D2000316900B2B480C1E88F3F82F310889842D5
:101D3000FFF657AF0746A946746906F1080807EB96
:101D4000470E04EBCE03D3E90250B6F90830C4467F
:101D5000002BA8BFB34605DA0FE034F93A309446B9
:101D6000002B09DB03EB430A04EBCA02D2E9026150
:101D7000B54270EB0101F0DA5E46ACF8007034F960
:101D80003E7024F83E30002FD9DAB3794D46002B4F
:101D90003FF42BAF0023B371B6F9083006F1080801
:101DA000591C3CD01946776903E080465A1C3FF421
:101DB0001EAF03EB430207EBC200B0F802C01C46A3
:101DC0001CF4004F9E4637F93230EED08C4280ED45
:101DD000028B05D0A8F80030318927F83210348101
:101DE0007146E3E739F83A3033813369EFF3108213
:101DF00072B6D3E8CF0F01210028FAD1C3E8401F03
:101E00000028F6D1BFF35F8F7388316929F83A3023
:101E100000237480C1E88F3F82F31088DDE640BF65
:101E200005B0BDEC028BBDE8F08F2846CDE902235A
:101E300000F0ACF9029A039B10EB020B43EB010894
:101E400029E708460B69029198470028CAD00299F1
:101E5000D1E9002314E700BFFFFFFFFFFFFFFFFFF3
:101E600000800B40AC32002000000B40911B0010A2
:101E70002DE9F84F364C25692DB1BDE8F84F0A2100
:101E80003448FFF739BEDFF8E4800321404600F014
:101E90006BF90326C4F80C80FFF73CFC4FF0504C64
:101EA0002D4B267003442361DCF800300F21637052
:101EB000636961801D834FF00405A3F878504FF0EB
:101EC0000505A3F890504FF00605A3F8A8504FF071
:101ED00007050E214FF6FF7208274FF00A0EA3F8F0
:101EE000C0504FF001094FF00C0C4FF0020B4FF0B7
:101EF000090A0D204FF00B05A3F868111749A280BD
:101F0000A3F808E1A160A3F848B0A3F8F0A0A3F8F3
:101F10002051A3F838C1A3F85001A3F83090A3F8DA
:101F20006060A3F8D8701A800D4B3046C8F8207056
:101F30000C49DC60FFF754FC49463046FFF72AFCA9
:101F4000094B0A211F640348BDE8F84FFFF7D4BDD1
:101F5000780A0020A834002030150020FFFF100070
:101F6000AC320020911B001000200B4000000B4001
:101F70000146F0B50069EFF3108772B6D0E8CF5F85
:101F80000124002DFAD1C0E8454F002DF6D1BFF352
:101F90005F8FB1F902E04C690EEB4E0CBEF1000F01
:101FA0004FEACC0504EBCC0C3DDB605B002648809F
:101FB0000869C0E88F6F87F31088BCF80200CCE98D
:101FC00002230130C0F30E00012838BF0120059B19
:101FD000ACF80200CCF81030069B40EA0E40CCF87A
:101FE00014300B69EFF3108272B6D3E8CFCF01271C
:101FF000BCF1000FF9D1C3E84C7FBCF1000FF4D164
:10200000BFF35F8F8B886353A1F804E00B69C3E8CB
:102010008F6F82F310880122CB68097803F5015392
:102020008A405A60F0BD00230A69C2E88F3F87F3F7
:1020300010884FF0FF30F0BD03464089B0EB214FD0
:1020400037DD58690A1402EB420210B500EBC200FA
:102050001C69EFF3108C72B6D4E8CFEF0122BEF109
:10206000000FF9D1C4E84E2FBEF1000FF4D1BFF339
:102070005F8F428889B292B28A4207D000221B69E0
:10208000C3E88F2F8CF31088002010BD42F400426B
:1020900042800121002218699971C0E88F2F8CF3CA
:1020A00010881C78DA68084602F50153A14059608F
:1020B00010BD0020704700BFF0B506460D4683B046
:1020C000EFF30584E4B2002C35D1244F3A78F96857
:1020D00004328B6A51F82220D21AC31A934207D3D2
:1020E00020BF1F4B586AA8421FD2002003B0F0BD8A
:1020F00000F054F8864265EB0101002911DB194B11
:102100003846CDE9003432462B46FFF731FF011E39
:1021100007DD134B5A6AAA4219D220BF0F48FFF7B6
:102120008BFF0F4B586AA842DFD39B6A9E4209D8A7
:10213000012003B0F0BD0A4B586A8842D5D39B6A90
:10214000B342F5D2401B18BF012003B0F0BD9B6A1B
:102150009E42E3D9AA42E1D1DFE700BF780A00201E
:1021600000000B40511B001010B4054B054C064AF3
:10217000A04214BF1846581C5DF8044BFFF79EBAE6
:102180009025002000800B40C8B600100346416A2D
:102190000A46986A596A8A42FAD17047034B596ACB
:1021A0000A46986A596A9142FAD1704700000B407A
:1021B00010B4174A536A9C46946A536A6345FAD12D
:1021C000001959414FF0000228BF01220346CAB14D
:1021D0000F4B596A4B1C08BF0B4608D04FF0FF311C
:1021E0000B460B48426A8A42FCD38A4207D1084A0E
:1021F00002E0506A884202D1906A9842F9D35DF8B1
:10220000044B7047024A526A9142EAD8EDE700BF98
:1022100000000B40F8B5054606200E4600F0E4F835
:10222000002842D0354A3648954214BF4FF08062AC
:102230004FF00062334B344902601A608C6832EA16
:102240000404FBD12D4B4FF48071EB1AB3FA83F3E6
:102250002E4A5B09062022F8131000F0C5F8C300CF
:10226000B3FBF6F30133DA0920D14026012169627C
:10227000AA622F6BFB0722D42B46002253F82C1F97
:10228000062003F5805422602F6300F0ADF840F281
:10229000013103228000B0FBF6F0EB6A83F070039B
:1022A00003F07E0323602963AA64F8BD4FF6FE7134
:1022B0008A421BD922464FF6FF71154ED7E740F2EE
:1022C000013205F540531A636B6AAC6A062004EBD1
:1022D000831400F089F80F4BA402A3FB0023DB0A50
:1022E0000021B4FBF3F0FFF763FFC5E7C3F3450339
:1022F000114603EB82161A46B9E700BF008007407B
:10230000002002400030024000000240D43700208C
:10231000C0FF3F00757B2B8F00EB400C4FEA8C0C0D
:102320000CF1804C0CF5803CF0B51646DCF804202E
:10233000051FB2F5803F38BF4FF48032EDB238BF91
:10234000CCF80420012D2AD94FF40067254C0CF558
:102350004052176054F82020B2B9DCF80020012D5B
:1023600082EA461202F0E0020CF5805632602AD969
:102370004FF4006144F820304FF480330CF50052E4
:102380001160CCF80430F0BD6769B7FBF2FE0EF1C6
:10239000010E0EEB4E0EBEF1030EFCD2DDE701295D
:1023A000D2D103240CF540521460DCF80820D20787
:1023B000FBD5DCF800200B4C82EA461202F0E0026A
:1023C0000CF5805632600122DCF800504D4005F0DB
:1023D0000305356002FA01F1DCF808200A42FBD05F
:1023E000C6E700BFA4250020014B53F8200070472A
:1023F000A425002070B4039D04682D0345EA03451D
:102400001B4B002CB3FBF1F3B2FBF3F61FDB194AB5
:10241000194B904214BF4FF480424FF40042174CC6
:102420001A6003F580531A60A36832EA0303FBD1F4
:10243000212200F540530433016086601A6002686F
:10244000002AFCDA0822C5601A6070BC7047036875
:1024500003F03F038B42DAD18368C3F30B03B3422B
:10246000D5D1C36803F4EE23AB42D0D1EDE700BF72
:10247000001BB70000800540002002400000024021
:10248000012300EB4000800000F1804000F5841043
:1024900041600360704700BF002370B5DB8A0446CB
:1024A0000D46002242E800F2520254BF10210421DE
:1024B00044F25220984786462B462246F446BDE811
:1024C00070400A214FF48170604700BF0023DB8A0F
:1024D000002242E800F2520201D4102118470421E0
:1024E000184700BF08B503460846191E02DB1AB19B
:1024F00040F03000FFF7D0FF40F02000FAE700BFC7
:10250000034AD2F82838002BFBD0BFF35F8F704707
:1025100000000E400021044B044ABFF35F8F43F8D4
:10252000041B9342F9D170470C080E402C080E4052
:1025300010B42F204FF42A64054A064B0649146054
:10254000D06019605368002BFCDA5DF8044B7047CB
:102550000080044000A0044000B0FA00704700BFB3
:1025600008B50148FFF792F8ECB6001038B5054CF5
:10257000054DAC4204D254F8043B9847AC42FAD320
:1025800038BD00BF10B2001050B2001038B5054C75
:10259000054DAC4204D254F8043B9847AC42FAD300
:1025A00038BD00BF3CB2001050B2001010B4074854
:1025B000074C084B084A094904601A608B6832EAE4
:1025C0000303FBD15DF8044B704700BF00200240BD
:1025D0007F3BEFEF00300240F6FFF30300000240C4
:1025E000044BDB6CB3F5004F03D14FF48022024B58
:1025F000DA64704700001150002011504FF0E022C3
:10260000044BD2F8881D0B43C2F8883D10EE30040D
:10261000704700BF030330006FF06041044B054A70
:1026200019609368DB4333F06043FAD1704700BF11
:10263000003002400000024010B545F25320FFF781
:1026400045FFBDE8104003460420184710B545F289
:102650005320FFF73BFFBDE8104003460120184719
:10266000FFF76CB810B5054B054C4FF4887218464F
:10267000A16804F061F8A06010BD00BF0000002058
:1026800000ED00E0002370B52B4C82B0C4F884301C
:10269000FFF74EFF0122294BDA63636C012BFCD15B
:1026A0000321264A244B11639C6B012CFCD102268A
:1026B000052521460523224A22480096FFF79AFE67
:1026C00021462B46204A21480095FFF793FE002221
:1026D000042031461E4BFFF71FFE214628460022EC
:1026E0001C4BFFF719FE0022082011461A4BFFF77A
:1026F00013FE002209201146174BFFF70DFE0022A2
:1027000006201146134BFFF707FE0022114B07204E
:102710001146FFF701FE0420FFF766FE00240F4B71
:10272000A3FB0035AD0CE0B229460134FFF7A8FE4B
:10273000062CF8D102B070BD00000140003001400D
:10274000002F685900000540008C86470080054036
:10275000001BB70080D1F008006CDC0283DE1B4355
:1027600086B003B451FC0804CDE9020151FC090410
:10277000CDE9040151EC0A04CDE9060103BCF047A0
:10278000BDE800504EEC00C4BDE800504EEC01C462
:10279000BDE800504EEC02C400BD000000B5FFF7DC
:1027A000DFFF02E010FE30F4F8D441EC100443ECFB
:1027B000112400EE010410EE010480EE200451EC1F
:1027C0001004704700B5FFF7CBFF02E010FE30F4B5
:1027D000F8D441EC100443EC112400EE010410EE97
:1027E000210480EE200451EC3004704700B5FFF75F
:1027F000B7FF02E010FE30F4F8D410B541EC10043D
:1028000043EC112451EC040453EC0524A0FB024CCE
:102810005FF0000EE0FB03CEE1FB02CE4CEC204467
:102820000024E1FB03E444EC30E480EE200451ECAE
:102830005004BDE81040704700B5FFF791FF02E07B
:1028400010FE30F4F8D441EC100443EC112451ECA8
:102850002104A0FB01126FEA820252FB100052FB1E
:1028600012F252FB1000A0EBD07C53EC04245CFB72
:1028700013F153EC1524A1FB022001FB030053ECE0
:102880004424A2EB000050FB1CF24FEA111312EBA0
:10289000017043EBE27140EA515020EA915020F080
:1028A000070053EC7524A0FB023C53EC752400FB9D
:1028B00003CC01FB02CC53EC0424ACEB824C40EA89
:1028C0005C70A0F1010041EC400480EE200451EC6A
:1028D0007004704700B5FFF743FF02E010FE30F4CC
:1028E000F8D441EC100480EE220410EEB2047047DC
:1028F00000B5FFF735FF02E010FE30F4F8D440ECED
:10290000700400EE010410EE210480EE200451EC6E
:102910003004704700B5FFF723FF02E010FE30F4EB
:10292000F8D440EC600400EE010410EE210480EEC7
:10293000200451EC3004704700B5FFF711FF02E0AE
:1029400010FE30F4F8D441EC800400EE010410EEE7
:10295000010480EE400410EE1304704700B5FFF749
:10296000FFFE02E010FE30F4F8D441EC800400EEEB
:10297000010410EE010480EE400410EE33047047B1
:1029800000B5FFF7EDFE02E010FE30F4F8D441ECA4
:10299000100443EC112400EE010410EE3004C0F3E7
:1029A0000070704700B5FFF7DBFE02E010FE30F468
:1029B000F8D441EC100443EC112400EE010410EEB5
:1029C0003004C0F38070704700B5FFF7C9FE02E025
:1029D00010FE30F4F8D443EC102441EC110400EE66
:1029E000010410EE30F48CBF01200020704700BFBE
:1029F00000B5FFF7B5FE02E010FE30F4F8D443EC6A
:102A0000102441EC110400EE010410EE30F42CBF50
:102A100001200020704700BF00B5FFF7A1FE02E0D3
:102A200010FE30F4F8D441EC100443EC112400EE15
:102A3000010410EE30F42CBF01200020704700BFCD
:102A400000B5FFF78DFE02E010FE30F4F8D441EC43
:102A5000100443EC112400EE010410EE30F48CBF9E
:102A600001200020704700BF0000000000000000AF
:102A700000000000DB60BE284A059193F4D5097F71
:102A800070374D7D66A5D83610E4104FEA58947F14
:102A900058F1AEF78E1BC96DB8749390BA4B920182
:102AA00087647482C77A873FCF694A2C7D8D20BAAC
:102AB00021D1AE4B091C673A90DF17AD8E75644E7D
:102AC0007DCED460E21721270E4A7EEFFF25FEC798
:102AD000036681F762C4CBFB479B82D6B39F4DDB75
:102AE0006DC2F2C9D98FD1D38BFA97A7B1EE495DE8
:102AF0005E7CF9FA7DCE41CFBAA494E2ECD7FE9A7F
:102B00004257E34711CC8015174B02F01F054FF0D9
:102B10000107AF405FEA6218A7FB00450026E7FB0C
:102B2000015603EB8803D3F81090A9FB06A7D3F84E
:102B30000C90A9FB05A8E9FB6678D3F8089009FB7F
:102B40000688E9FB0578A9FB04A6D3F8049009FBE5
:102B50000588E9FB0478D3F8009009FB0488BF19C5
:102B600048F10008704700006C2A001050EA01325A
:102B700008BF41F0004141F400210B000200704702
:102B80000BB900200021002240F20003C3F6F073CD
:102B90001CF0020F1CBF104619467047002200238C
:102BA00000245FF0004504E14DF804CD5FF0000C17
:102BB0000CF1040C02F10402FFF7A6FF98EAE87991
:102BC000B9F1807F02D2BCF1400FF1D197EAE877EA
:102BD00041F2A616C0F64636A9FB06A04DF21156E4
:102BE000C4F67E06A7FB06A1E9FB66010626E7FB05
:102BF000060109FB0611DCF1200A57D421FA0CF377
:102C000020FA0CF201FA0AF942EA0902A2FB039443
:102C1000A2FB0395E3FB6345A4FB0596A4FB059784
:102C2000E5FB6567F60856EA47764FF0AA39A6FB3A
:102C30000967D4EB070675EB45075FEA2739360BC2
:102C400056EB075659F17F6717F14057C0B4A0FB08
:102C50000592A1FB0493E1FB6523A2FB0596A3FB70
:102C60000497E3FB65674FF0AA39A2FB09A400258E
:102C7000E3FB0945641955F100054FF08839A6FBBF
:102C80000923B4EB131465F10005B0EB940061EB7C
:102C9000A501B0EB857061F10001CCF58064A4F171
:102CA0000E0400F082F9BDE8C0100CE0CCF58064A1
:102CB000A4F10E0400F079F95DF804CB002640F28F
:102CC0000007C3F6F0775FEAD87868F3000C5FEA94
:102CD0006C090FD45FEA690906D31CF0040C57EAAB
:102CE0004C713000BDE8F0879CEA9C0C51EACC7135
:102CF000BDE8F0871CF0040497EA4477C0B4A6E06E
:102D00003CB500F004F830BC03C40CC530BD11F074
:102D1000004C5FEA5C0C5CF0004C06E05FEA517C22
:102D20001CF0040C01E05FF0020CC1F30A53A3F2A3
:102D3000FF32B2F5806F3FF419AF12F1200FFFF6AA
:102D40001FAF012363F31F512DE9F04702F10C027D
:102D5000FFF7DAFE5FEA987444F10004A8EB847888
:102D60000CEB440C4CEAD87C97EAE87798EAE878D0
:102D7000B8F5800FFFF418AF41F2A619C0F6463936
:102D8000A8FB09A04DF21159C4F67E09A7FB09A1C1
:102D9000E8FB69015FF00609E7FB090108FB09117F
:102DA000B1F1007FFFF4FAAECA0E7C4B03EB0213C5
:102DB0003CCB801A994110D45FEA6C0636D4761069
:102DC0001CD200F06CF800F0AFF800F0ECF89CEAD0
:102DD0009C0C51EACC71BDE8F0875FEA6C0649D4DF
:102DE000761017D200F058F800F0ACF800F0D8F8E0
:102DF0009CEA9C0C51EACC71BDE8F08700F04FF8DA
:102E000000F0AFF800F0CCF81CF0040C51EA4C7163
:102E1000BDE8F08700F040F800F0B2F800F0C3F829
:102E20001CF0040C51EA4C71BDE8F08700F037F853
:102E3000FCB400F096F800F0B3F81CF0040491EA3A
:102E40004471FCBC03B400F06FF800F0ACF89CEAED
:102E50005C0494EA9C0491EAC4711CF0020F1DBF4B
:102E600002460B4603BC0CBC1CF0804491EA4401B2
:102E7000BDE8F08700F010F8FCB400F081F800F035
:102E800092F81CF0040491EA4471FCBC03B400F015
:102E900059F800F085F8DAE7404261EB4101A1FB07
:102EA0000167A0FB01237F084FEA3606F21847F1BD
:102EB0000003A3FB0076E2FB01760027E3FB01673A
:102EC0004FF05538A6FB08964FF00009E7FB08695C
:102ED00016EB090659F10007861B71EB07074FEA4D
:102EE000033040EA1250A0FB0009E9FB0809A9FBE6
:102EF00001084FF03330A8FB000858FB11FA4AF6DE
:102F0000AA20C2F6AA2060FB1A99B2EB491273EB11
:102F1000D9635AFB11FA4FF0C3606AFB108816EBB5
:102F2000481657EBD8677047A2FB04804FF00001AA
:102F3000E3FB0401A6FB0583E7FB0534181A64EBE9
:102F400001017047A2FB04804FF00001E3FB040184
:102F5000A6FB05836442E7FB0534181844EB010126
:102F60007047A2FB05804FF00001E3FB0501A6FBC3
:102F700004836D42E7FB0435181845EB01017047E7
:102F8000A2FB05804FF00001E3FB0501A6FB0483D3
:102F9000E7FB0435181A65EB01017047B8330010E0
:102FA000404261EB410140F2F334B1FA81F20C2A64
:102FB0000CD2153211FA02F3C2F12002D04021FAEC
:102FC00002F12244584141EB0251704769B1C2F10C
:102FD0002B0230FA02F3C2F12002914090401943D3
:102FE000A4EB020201EB0251704701004FF0000018
:102FF000A4F12004D9D17047012767F31F5117FAB4
:1030000003F817D0A0FB080701FB0871A1FB0678A5
:103010005FEAD8469219A6FB047806FB05880903E7
:1030200051EA1051D7EB003061EB0801A94238BFDB
:1030300070470BE00C33012717FA03F80FD0A0FB01
:10304000080701FB0871A94238BF704708BFA042BA
:1030500038BF7047001B61EB05010132704703F177
:10306000200311FA03F6D3F12003D840D9403043AE
:103070007047000000000000000000000453B10889
:103080006018850FC8E5F22A6E07271E0D12B221BF
:103090000412572F12557CBCDA30723F17A717A5C0
:1030A0005531994E9D0DBF0AEEE0AB5FE3EF6D9C8D
:1030B0007636AD6F697BCCE33D62BD7EF0810682E2
:1030C000F3FA428F37D5B78A5313C89E7FABB3202C
:1030D000491570AF0000000000000000025E881576
:1030E0005580FF00907806B1A602FE01DC4E21F06B
:1030F000EB88FB027A7C801F1615F8033C5DA9D192
:1031000010A9F304AA466CF5C146EE05FF65E4EB91
:1031100009F0E70613C00C9EC3A6E007E1BFEC91DF
:10312000C46CD808D5AF5EFFDC43CF09466A72E4B1
:10313000D72DC50A237E6E197B2CBA0BBFF571649F
:103140008741AE0C61DFB88CB86EA10D09A9856D01
:10315000C5B5930E3153B1086018850F3071E498EE
:10316000359875105915550580FF0F0009C3EB8F71
:1031700080FB2F00B1910E9A82F34F001FE7FD22D2
:1031800087E76F00C3A09A298FD78F004F4366ACA3
:103190009BC3AF00412A83A9ADABCF004FB7B41E8C
:1031A000C68FEF00B6815F09E66F0F0167858966FC
:1031B0000E4C2F011A52DA3240244F01483A9B6AD2
:1031C0007CF86E01FF81B709C4C88E019C8DBC0BD1
:1031D0001895AE017010DA6B795DCE013A3BE224AE
:1031E000E921EE0138739533427FECA03114FAF5F2
:1031F000BD8689916B02FAE6E0F29183E6821207BE
:1032000013A85177212621686AB2736A9D0DBF0AFF
:10321000EEE0AB5F19B4E0B71CB66A549596E53D95
:10322000EF07A548D1CBE555DC0E4E3CCE68ADE8A6
:1032300039B5A432CB3CFA96D9569A28C9B21CA10A
:10324000F9FCAE21864B6BE58AD2F0160453B10827
:103250006018850F02C00C9EC3A6E00700000000A6
:1032600000000000AC79CFD1F71772B1293BAAB8A2
:103270004FEAC12040F00040490043F1200340F2F2
:103280000001C3F6F071C3F10B0320FA03F038BF5D
:103290007047404261F1000170475FEAD17CC1F3A1
:1032A0000A53A3F2FF330C2B62DA13F1200FDFDD98
:1032B0002DE9F0413C4C70CC4FF00002FFF79CFE32
:1032C0001CF0010F04D06FEA0202201A65EB010125
:1032D00002F2FE3C40F2FE739C455CD20A0F334B77
:1032E00003EBC2030CCB02F03F0545F04005801A0A
:1032F00099410A0E2E4B03EBC20318CB02F58072E4
:103300005543C01AA1414A0D2A4B03EBC20318CB07
:10331000124402F5805205FB0255C01AA1418A02EF
:1033200052EA905242F1000282FB02345B0D53EAF2
:10333000C423C01841EB545184FB02344FF0553381
:1033400083FB043454FB11F304EB930410EB4402AD
:1033500041EBE473E900A1FB0240C1FB0301400A19
:1033600050EBC1504FEA512151EB0C51BDE8F081B7
:10337000B3F5806F07D150EA01320CBF21EAE17149
:1033800041F400217047002000211CF0010F08BF0C
:10339000C7F6F07170474FF000004FF00001A8BF72
:1033A000C7F6F071BDE8F08164320010743000108F
:1033B000D4300010643100100B5C7325A974F50340
:1033C00029B5FA010015FC7FEB2FAA0054D9440C53
:1033D000C8D221061F60DA7F3663E842CFD3D91303
:1033E0003C5EEA09F0889D7F2FC46D04D9860A1CD3
:1033F0001F17FE0DD09E3B7FA79B50EC3EF5EB23A5
:10340000BCE7E611C7EFBD7ED21C9C03B212F12BC4
:1034100046F5DC1549771E7ECA057A3DF493F233F2
:1034200014C0CB199CAC5F7DA0A0EF7A1D32193C73
:103430001D22C61D2F2F7D7CB50FFB1270EF50444F
:10344000530CC1213522787B5C8D6B4745A0F14B35
:1034500018DC6A2516AD687AC14069576DD9EA5300
:10346000391636293C2D2F79DFEA4ED38942B35BDA
:10347000D639E02C2526E0776950EA31D907116466
:10348000C0D3C43070625876CB5667F3B3A2FD6BDD
:103490001C7E6834227AC7740EED7A2F3175E07382
:1034A000CCE7FA3727111C73C08EC4FC0E79147C4C
:1034B0000EA7A33B8ECD417113B7043B8F7B548382
:1034C000D489D23EEBD8856F9A365B13D96F0B8CBB
:1034D000D4EA9442A3EF516D5F52CA4A26D339947D
:1034E000706E0A464005236B8340C441340B0E9C2A
:1034F0003DB0484907EFF168BF086DA3FD6179A4AD
:1035000085F2B14C9D847A663616F8C8D247E5AB91
:103510001E22A24F2F623664ADC9C8D0E1ADFEB302
:103520002470C35286AFA461730E73646A35FEBB08
:1035300028F0C555A3A3025FC6A58CB055B912C427
:103540000892BA58A394415C90005354372DB0CBE5
:1035500019F46E5BD88E9359367C8DA16E3CAAD33C
:1035600025022E5EFC32AF56D0C7A248F619FFDB0B
:103570003253F3607EED9253949AAD7AE1AD22E43A
:10358000CADF8E63C72B7350FF15EF19BD85FBEBA8
:10359000BB18FA65C7615C4DBD960F7E494B4CF474
:1035A000F7816F68E617024AEB09EF1DFDBD4DFC80
:1035B000C4D2B26A13E4B4460022002950DA404271
:1035C00061EB4101C9B1B1FA81F30B3B17D4D3F1DF
:1035D000200C30FA0CFC9840994051EA0C011A4436
:1035E000524202F2324201EB025141F0004140F2FC
:1035F000FE739A4238BF704721E011467EE003F126
:10360000210310FA03FCA3F1010301FA03FCC3F147
:10361000200320FA03F021FA03F140EA0C00A3EBA7
:10362000020202F2324214D050F1000041EB02518A
:1036300041F0004140F2FE739A4238BF70474FF0AC
:103640000001A8BFC7F6F0714FF0000070470021DD
:103650007047EBD350F1000020F00100E6E70022B4
:10366000B9B1B1FA81F30B3B16D4D3F1200C30FA87
:103670000CFC9840994051EA0C011A44524202F263
:10368000324201EB025140F2FE739A4238BF70475A
:1036900020E0114600F066B803F1210310FA03FCA4
:1036A000A3F1010301FA03FCC3F1200320FA03F0A4
:1036B00021FA03F140EA0C00A3EB020202F23242CB
:1036C00012D050F1000041EB025140F2FE739A42D9
:1036D00038BF70474FF00001A8BFC7F6F0714FF038
:1036E0000000704700217047EDD350F1000020F03A
:1036F0000100E8E7002880F235804042B0FA80F30C
:103700000B3B11D4984001EB0302524202F21242E9
:1037100000EB025141F000414FF0000040F2FE7317
:103720009A4238BF704713E0C3F1000330FA03FC3C
:10373000C3F120029040A3EB010202F212420CEB13
:10374000025141F0004140F2FE739A4238BF704787
:103750004FF00041A8BFCFF6F0714FF00000704766
:103760000021704760B3B0FA80F30B3B0FD4984050
:1037700001EB0302524202F2124200EB02514FF0FF
:10378000000040F2FE739A4238BF704710E05B427F
:1037900030FA03FCC3F120029040A3EB010202F2D5
:1037A00012420CEB025140F2FE739A4238BF70474E
:1037B0004FF00001A8BFC7F6F0714FF0000070474E
:1037C000002170470022A2F232425FEA215CACF194
:1037D0000103A1EB03515B0513F5800F32D212EB0D
:1037E000535210D40B2A36DA9140D2F1200330FA2A
:1037F00003F319439040BCF1000FA8BF704740424B
:1038000061EB4101704720320EDD01FA02F3D2F183
:103810002002D140D0401843BCF1000FA8BF704730
:10382000404261EB41017047524282F3050231FA96
:1038300002F00021BCF1000FA8BF7047404261EBCD
:103840004101704702D000200021704750EA013149
:1038500018BF4FF0000C6FF0004101EBDC716FEA14
:10386000EC70704738B50446094807F0C9FC20469B
:1038700002F01CF80546064807F0BEFC2DB1054BCA
:103880002C449C4201D8284638BD0348FDF7FEFE73
:103890006C11002000000820F8B6001038B505466D
:1038A0000C460A4807F0ACFC2846214602F0E4FA30
:1038B0000546064807F0A0FC2DB1054B2C449C4260
:1038C00001D8284638BD0348FDF7E0FE6C11002002
:1038D00000000820F8B6001038B50446054D28460B
:1038E00007F08EFC204601F0E9FF2846BDE838408D
:1038F00007F082BC6C1100209A4238BF8854704790
:10390000704700BF2DE9F04F83B09946DDE90DAB5C
:103910000F9B884611469A07074616D1DA453AD2D8
:103920000C460D46ABEB0A060E4422464B4641467A
:1039300020200134B847B442F7D12946BAF1000F2C
:1039400008D1204603B0BDE8F08F0C46BAF1000F55
:1039500010D00E4655460C9B2E449A440191721B82
:103960004B46013D41461AF8010D3446B847002D3B
:10397000F5D101990F9B9B07E3D5651AAB45E0D9BB
:1039800022464B46414620200135B8475D4504F1AB
:103990000104F5D3D5E7BAF1000FDAD10C46D0E730
:1039A0002DE9F04F0F9FDDF824E017F0020F0A9C7D
:1039B0009DF82C900E9DDDE90C8629D1002D6FD14C
:1039C000B44225D2202C07F0010B00F0128104F143
:1039D000FF3C4FF0300AF44401E0202C7AD001344F
:1039E000A6420CF801AFF8D8BBF1000F10D0AC42E2
:1039F0000ED2202C74D004F1FF3C4FF0300AF44476
:103A000001E0202C29D00134AC420CF801AFF8D1F0
:103A100017F0100F3AD017F4806F28D11CBBB8F103
:103A2000100F00F0CA80B8F1020F00F0D4803024EB
:103A30008EF800400124B9F1000F67D17E0740F1F4
:103A4000AA802B260EF804600134CDE90B57CDE98E
:103A500009E4BDE8F04FFFF755BFFC0640F189804F
:103A60007C0535D42024A6426AD0AC4268D0B8F197
:103A7000100F00F08780B8F1020F5AD0202CE4D04C
:103A8000264601344FF0300C0EF806C0202CD2D15F
:103A9000CDE90B57CDE909E4BDE8F04FFFF732BFA0
:103AA00017F0010B3ED0B9F1000F47D117F00C0F02
:103AB00044D1B4429BD2202C89D1202D10D8FC06B1
:103AC00057D57C0555D4202E00F0B980202D10D07C
:103AD0002024CCE7BBF1000F00F0A580202DBCD93D
:103AE000FC0646D57C0544D4202E00F0A880202D6D
:103AF0003FD12C461F26B8F1100F7FD0B8F1020F2E
:103B0000C0D14FF0620C0EF806C0B7E72D260EF8B4
:103B100004600134CDE90B57CDE909E4BDE8F04F6D
:103B2000FFF7F0BEB442BFF473AF202C7FF44FAF69
:103B3000D6E7202C89D026460134E2E7013DB8E7DC
:103B4000661ED8D1B8F1100F64D0B8F1020F7FF41F
:103B50006EAF62268EF80060302644468EF8016013
:103B6000B9F1000F3FF46AAFD0E7B8F1100F7FF45E
:103B70006CAF2024CDE90B57CDE909E4BDE8F04F47
:103B8000FFF7C0BEBE060ED4202CF2D078260EF869
:103B90000460013472E73E077FF557AF20260EF828
:103BA0000460013451E7202CE3D04FF0580C0EEBA9
:103BB000040686F800C0013460E7BE0617D5582415
:103BC0008EF8004030248EF801400224B9F1000F35
:103BD0003FF434AF9AE762248EF8004030248EF828
:103BE00001400224B9F1000F3FF428AF8EE778249A
:103BF000F2E7BBF1000F7FF462AF71E717F0200F1F
:103C00000CBF4FF0780C4FF0580CA61E0EF806C0F3
:103C1000013C35E7BC06EAD558248EF80040302434
:103C20008EF80140DDE717F0100F3FF40EAF17F4E8
:103C3000806F9AD1202E7FF418AF1F265BE73446A1
:103C40001F2658E700B9704701F0F2BA10B1D1E968
:103C500000311847704700BF2DE9F04F9FB09DED30
:103C6000287BDDE92AA558EC177B83461E460D917B
:103C7000109243463A46384641468DED087B2C9CCF
:103C8000FEF782FE002840F0D880384641464FF0CB
:103C9000FF32754BFEF7D8FE002840F0CE80384644
:103CA00041464FF0FF326FF48013FEF791FE00287B
:103CB00040F0C380DDE90878002238464146002301
:103CC000FEF786FE002840F0C081CDE90A78DDE9E4
:103CD0000A2390461F4614F4806308BF4FF0060A7B
:103CE000139304F4006258EA0703119240F0C08075
:103CF000002A00F0A2819FED5A7B00278DED0E7BFC
:103D00004FF00009BA45CCBFAAEB070A4FF0000AF2
:103D10004F46C8BF0AF1FF3A44F480644D4594BF52
:103D20004FF00008A5EB090814F00203119304D02A
:103D3000B9F1000F18BF4FF000083FB1DDE90A01EB
:103D4000DDE90E23FEF77CFDCDE90A01DDE908017E
:103D500000220023FEF73CFE30B1DDE90A010246F5
:103D600001F10043CDE90A239DED0A7BCDE902A8CC
:103D7000DDF834A024F4006304938DED007B33461A
:103D800051465846109A00F097F98046B9F1000F55
:103D90004FD014F0200F024600F1010433460CBF4F
:103DA000652045205146D84709F1FF3087EAE77C76
:103DB0000DF1580900224B46DFF8B080ACEBE77CF0
:103DC0004FEAD77E01E0202A10D0E246A8FB0C7112
:103DD000C90801EB8107ACEB47073037BAF1090F8F
:103DE0008C4602F1010203F8017BECD80523059013
:103DF000069300200A230D9FCDE90330CDE9012E63
:103E00003346224639465846CDF80090FFF7C8FDA4
:103E1000119B80466BB1109BC41AA54209D942463A
:103E20003346394620200134D847A54208F101081D
:103E3000F5D840461FB0BDE8F08F9DED087B3346B6
:103E40005846109A0D998DED287BCDE92B54CDF86D
:103E5000A8A01FB0BDE8F04F00F02EB9AFF300806E
:103E60000000000000000000FFFFEF7FCDCCCCCCB5
:103E7000C7F30A50A0F2FF30FEF73EFD8AA3D3E954
:103E80000023FEF7B7FC8AA3D3E90023FEF78AFCE0
:103E9000C7F31307CDE90E0147F07F5140460022DA
:103EA0007B4B41F44011FEF791FC6BA3D3E9002357
:103EB000FEF7A0FC02460B46DDE90E01FEF772FCA0
:103EC000FEF73EFD0746FEF717FD65A3D3E9002385
:103ED00080468946FEF78EFC00226E4BFEF762FCA0
:103EE000FEF72EFD03464946404612935EA3D3E9F2
:103EF0000023FEF77FFC804612988946FEF7FCFC03
:103F00005BA3D3E90023FEF775FC02460B4640464F
:103F10004946FEF75BFC02460B4680468946FEF7A3
:103F200069FC42464B46CDE90E0140464946FEF744
:103F300039FC0022CDE91401DDE90E01564BFEF7F4
:103F40007FFC0022554BFEF72DFC02460B46DDE9B7
:103F50000E01FEF775FC0022514BFEF723FC0246D2
:103F60000B46DDE90E01FEF76BFC42464B468046F0
:103F7000894600204FF08041FEF728FC02460B46A0
:103F800040464946FEF70EFC02460B46DDE91401A9
:103F9000FEF756FC0022434BFEF704FC129B002266
:103FA00003F2FF3C4FEA0C53FEF724FC804689469F
:103FB000DDE90A0142464B46CDE90E89FEF708FDD0
:103FC00068BB4346494607F16302C62A119A8CBF73
:103FD0004FF005094FF00409002A3FF49FAE0B4350
:103FE0003FF48EAEDDE90A0123A3D3E90023FEF7F7
:103FF00017FD48B1DDE90A0121A3D3E90023FEF74B
:10400000E7FC00287FF47CAEBAF1000F3FF486AEE7
:10401000139B002B3FF482AE0AF1FF3A7EE60022AA
:104020001E4B40464946FEF70BFC0A460146034636
:10403000CDE90E12013F1146C5E79FED137B1746F0
:104040004FF004098DED0E7B68E608F100430A97F6
:104050000B933CE6AFF3008061436F63A787D23FC9
:1040600071A379094F930A401655B5BBB16B024055
:10407000EF39FAFE422EE63F2D431CEBE2361A3FA3
:104080000000000080842E410000000000000000BD
:104090000000F83F0000E03F00002C4000002440FA
:1040A000000018400000F03FFB799F501344D33FBD
:1040B000B3C8608B288AC63F2DE9F04F97B0DDE981
:1040C0002089CDE90401DDE9224BCDE906234046F4
:1040D00042464B464946DDF890A0FEF755FC0028C5
:1040E00040F0C581404649464FF0FF326FF48013DF
:1040F000FEF76EFC002840F01D81404649464FF017
:10410000FF32C14BFEF7A0FC002840F0E380B8A3CB
:10411000D3E9002340464946FEF796FC002840F0CC
:10412000CB80B5A3D3E9002340464946FEF750FCB7
:10413000002840F0C1804046494600220023FEF797
:1041400047FC002840F0E0801AF480650D9000F0F4
:10415000E980092C40F296810EAB1A460C9330216F
:104160000023A4F109050133202B02F8011BA4EB65
:10417000030600F03A81AB42F5D19FED9D7B8DEDBA
:10418000087B49464046FEF7DBFB0446FEF7B4FBDE
:1041900002460B4640464946FEF718FBDDE9082378
:1041A000FEF728FB02460B46CDE90A23FEF7DAFBB1
:1041B0000746FEF7B3FB02460B46DDE90A01FEF7B0
:1041C00005FB02460B46CDE90A2300228F4BFEF782
:1041D0003BFC002800F0DB8001373846FEF79EFBF1
:1041E000DDE90823FEF71CFC08B100270134002E8E
:1041F00040F0B1802046FEF77FFB02460B4640466A
:104200004946FEF7E3FA0022804B06460F46FEF7CA
:10421000DFFB40B93046394600227C4BFEF714FCE8
:10422000002800F015810C9B691E7948194410E0A4
:1042300080FB0462C3EBA20303EB8302A4EB420402
:1042400004F1300201351C4601F8012F002B00F06B
:10425000AB80202D4FEAE473EAD10AF00303012B6F
:104260001CD1BBF1000F19D00D9B002B40F0F98041
:104270001AF00C0F40F0F580AB4540F2D380202DB2
:104280000BD030220C996B1E0B4401355D4503F8B1
:10429000012F00F08D80202DF7D12025DDE90623A8
:1042A000DDE904010C9CCDE902BA01950094FFF709
:1042B00029FB17B0BDE8F08FCDE92089DDE90623A1
:1042C000DDE90401CDE923BA229417B0BDE8F04F2F
:1042D000FFF7C2BC4F4DCDF88CA00AF0040ABAF12A
:1042E000000F4D4C18BF2C46DDE90623DDE9040123
:1042F00020940CBF03240424CDF888B0219417B077
:10430000BDE8F04FFFF7FEBA4B46424600200021C1
:10431000FEF75CFA01231AF48065804689460D9306
:104320007FF417AF9FED367B0EAB06268DED087B35
:104330000C9326E70424DDE90623DDE90401374D6B
:10434000CDF88CA0CDF888B02095219417B0BDE8A9
:10435000F04FFFF7D7BA0C9B681EDFF8C4C01844B3
:104360000DE0ACFB0721C90801EB8102A7EB42027B
:104370003032092F00F8012F27D90F461D46202D76
:1043800005F1010306F1FF36EBD120254BE70022B2
:10439000DDE90A011D4BFEF71BFB00287FF427AF68
:1043A000002F5AD1013722E70AF00303012B75D001
:1043B000202D3FF473AF0D9BBBB32D2205F15803A5
:1043C0006B4403F8202C013568E7202BDDD0AEB319
:1043D0000C9A1E441544302201E0B3422ED0013322
:1043E000202B05F8012FF8D1CFE71D46C5E600BF09
:1043F0000000000065CDCD410000000065CDCDC1BD
:104400000000000080842E41FFFFEF7F0000E03FAE
:10441000676666664CB7001054B700105CB70010B2
:10442000CDCCCCCC202D3FF439AF1AF0040F0DD1F8
:104430001AF0080F3FF432AF2022BFE72E2103F11C
:1044400058026A4402F8201C5D1CECE62B22B5E7FA
:10445000E3077FF5E8AE0134E5E6FA077FF5C7AE7E
:10446000A0E70BF1FF3BAB453FF609AFA0E7032404
:10447000DDE90623DDE904010A4DCDF88CA0CDF875
:1044800088B061E7084B264603EBC40393ED007B3D
:104490000EAB8DED087B00250C9372E6BBF1000F8F
:1044A00086D0E1E658B7001088B900102DE9F04F2A
:1044B0009A469BB0249C964D0B94964C0B1E18BFAD
:1044C000834625609AF80000934C0A9308BFA346E0
:1044D0000992002800F0BC824FF000090AE04A4629
:1044E000099B0A9909F10109D8479AF800000028A8
:1044F00000F0CE8025280AF1010AF0D100235246AF
:1045000012F8010BA0F1200110290AD8DFE801F010
:104510004009093C09090909090909380934090947
:104520003000A0F13001092940F28C802A2800F0E7
:10453000F58000210C912E2800F099800027A0F131
:10454000680112292DD8DFE811F057012C00510124
:104550002C0045012C002C002C002C002C002C00E1
:104560002C0027002C002C002C002C002C002700F5
:10457000924643F00103C2E7924643F00203BEE7CE
:10458000924643F00403BAE7924643F01003B6E7BD
:10459000924643F00803B2E79AF8010043F48073AF
:1045A00001326728924600F28280242840F2C680B9
:1045B000A0F12502422A00F2C180DFE812F05F017B
:1045C000BF00BF00BF00BF00BF00BF00BF00BF00F3
:1045D000BF00BF00BF00BF00BF00BF00BF00BF00E3
:1045E000BF00BF00BF00BF00BF00BF00BF00BF00D3
:1045F000BF00BF00BF00BF00BF00BF00BF0026015B
:1046000045012601BF00BF00BF00BF00BF00BF00C3
:10461000BF00BF00BF00BF00BF00BF00BF00BF00A2
:10462000BF00BF00D301BF00BF00BF00BF00BF007D
:10463000BF00BF00BF00BF00D3016701D301260147
:1046400045012601002100E0013201EB810100EB70
:10465000410110789246A0F13004092CA1F13001FB
:10466000F2D92E280C9102F101027FF467AF9AF87B
:1046700001001146A0F13006092E43F4806340F298
:1046800031812A2800F03E8192460027013256E708
:104690004C46099B994501D303F1FF394A46002056
:1046A000099B0A99D84720461BB0BDE8F08FA0F1BE
:1046B0006902D2B20F2A41D8012649F2410196403F
:1046C0000E4040F001810A2A3FD0072A36D10B9CC8
:1046D00054F8042B002A00F0288143F021010DF149
:1046E000480E704603E0202E00F029811A4602F0A1
:1046F0000F052B46092D94BF303337330F2A00F8AE
:10470000013B06F101064FEA1213ECD817E100BF96
:10471000AD4400108C320020013900100B9C9AF837
:10472000010054F8045B9246002DBDBF694243F07E
:1047300002030C910C950B940132FCE64A46099B4E
:104740000A9909F10109D847CFE60B9951F8048B72
:1047500098F800201046002F40F0E18072B16FF011
:10476000010C0CF1010C4646C44401E0664503D03F
:1047700016F8014F002CF9D1A6EB080613F4806C53
:1047800002D0BE4228BF3E4613F0020400F08781EB
:10479000002A00F02B81BCF1000F00F041810B9446
:1047A0000D964A46DDE909540E464F4408E02B4673
:1047B0002146D84718F8010F09F1010910B14A46FE
:1047C0004F45F4D131460B9C0D9E002C40F00E81DC
:1047D0000B918AE69AF801006C287FF4DFAE9AF814
:1047E000020043F440730AF10302DAE69AF801008A
:1047F00043F400730132D4E69AF80100682800F00F
:10480000208143F080030132CBE6672800F0E78087
:10481000472800F00081452800F0FF800B9C04939E
:104820000C9B0734CDE9027324F007031C46DDE935
:104830000931F4E802674A465846CDE900670B940F
:10484000FFF70AFA814650E646280B9C08BF43F062
:10485000200304930C9B0734CDE9027324F0070373
:104860001C46DDE90931F4E802674A465846CDE9BD
:1048700000670B94FFF720FC814636E64A46252068
:10488000099B0A9909F10109D8472EE60B9A9C0762
:1048900002F1040709F1010640F1E6801078099B56
:1048A0004A460A99D8470C9B012B40F22C81DDE93E
:1048B0000954994432462B46214620200136D847D8
:1048C0004E45F7D10B9710E66F2800F08B8040F231
:1048D0006581782800F008814FF00A0823F0100362
:1048E000C44647E0002707EB870700EB4700A0F12D
:1048F000300711F8010FA0F13002092AF3D98A46D6
:104900004A1C1CE60B9C9AF8020054F8047B0AF13E
:10491000020A0AF101020B9427EAE7770FE6002A60
:104920003FF42CAF07F1FF3C1BE723F0100113F419
:10493000806241F021013FF4D2AE0DF1480E082310
:104940001020059300234A46CDE9023006915846CF
:10495000DDE90931CDE900E60497FFF721F80B9472
:104960008146C2E5582879D0622840F051824FF044
:104970000208C44613F480606DD123F00C0313F4D5
:10498000007240F0C2800B9904310D9113F48071D4
:1049900040F02E825E060B9A40F1AA801278002A1F
:1049A00040F0DA8023F01003002800F0D580114693
:1049B0000DF1480E06930C9BCDF80CC0CDE90473A5
:1049C000019100234A4602935846DDE90931CDF8AA
:1049D00000E0FEF7E5FF0D9B81460B9385E543F470
:1049E00000631BE74FF00808C446C3E70C9B4C4626
:1049F000B3427FF6EDAE0F464B44A3EB0609DDE96B
:104A0000096522463346294620200134D8474C45C3
:104A1000F7D13946DCE643F4006343F02003FDE6BA
:104A20000F460B94DDE909544A462B462146D847E8
:104A300018F8010F09F101090028F5D139460B9C3E
:104A4000C3E69AF8020043F0C0030AF10302A8E5A6
:104A5000044681461DE623F00D0390E74FF0100851
:104A600043F02003C44685E70C9B012B45D9DDE9C3
:104A700009544E4609F1FF38984432462B462146E8
:104A800020200136D8474645F7D10C9B3246994441
:104A90000B9B1878DDE90931D8470B9725E50C9B6E
:104AA000B34240F2EE81CDE90D48DDE90954884674
:104AB0004B449E1BCDF82CC04A462B462146202055
:104AC00009F10109D847B145F6D14146DDF83880F2
:104AD0000C9BDDF82CC00D9C98F800205E1C104645
:104AE000002A7FF458AE73E64FF01008C44641E741
:104AF0001D064CBF1288126851E713464A461878C3
:104B0000DDE90931D847B146DCE60B9C073424F0D7
:104B100007042246656852F8084B0B9254EA0502D6
:104B200040F02C8123F01003002800F0278100269C
:104B30000DF1480E06930C9B4A46CDE90473002301
:104B4000CDE900E6CDF80CC002935846DDE9093105
:104B5000FEF726FF8146C8E413F0200F14BF412062
:104B600061200DF1480E7646A0F10A0803E02029E5
:104B70003FF420AF2246B2FBFCF40CFB1425E8B254
:104B8000092D00F130058ABF4044E8B2C0B2624549
:104B900006F8010B01F10101E9D20BE723F0100245
:104BA00069280D9240F06F8113F4806204D04FF4B5
:104BB000806223F011030D930D9B13F4007640D116
:104BC0000B9B03F104080D9B13F4807040F0988058
:104BD000590640F1C6800B9B19780C46CB0F002973
:104BE00000F0B98022460DF1480E74461646DFF8F3
:104BF000A0C201E020280FD03546ACFB0621C90831
:104C000001EB8102A6EB42023032092D0E4600F183
:104C1000010004F8012BEDD80D9ACDE901030692AD
:104C20000C9ACDE904720A234A4603935846DDE9FB
:104C30000931CDF800E0FEF7B3FECDF82C808146B7
:104C400053E40B9C073424F00704214608466368AC
:104C500050F8081BDC0F0B9051EA030000F0C380F2
:104C60000A46191E48DB13460DF1480EF44600268D
:104C7000CDE90E94DFF8188201E0202E2DD05A18CD
:104C800042F10002A8FB025929F0030505EB990542
:104C9000521B1C469B1A61F1000508464FF0CC31AF
:104CA00001FB03F108FB0511A3FB0853194405237D
:104CB00005F00109A9FB03399B180A2C03F1300305
:104CC0004FEA550570F100000CF8013B06F10106B2
:104CD00045EAC1734FEA5101CFD2DDE90E940D9B35
:104CE0004A4606930C9BCDE90164CDE904730A237F
:104CF000CDF800E0039328E7524261EB4101B2E7AF
:104D00000B9B1968CB0F002900F0AB8081EAE172A0
:104D1000A2EBE1720DF1480E7046DFF874C101E0BC
:104D2000202E10D01546ACFB0241C90801EB8104CE
:104D3000A2EB440404F13002092D00F8012B06F126
:104D400001060A46ECD80D9ACDE9016306920C9A49
:104D5000CDE9047267E7002A3FF445AF0DF1480E34
:104D60005AE713F0800F0B9B00F08180B3F900101D
:104D700081EAE174A4EBE174A4B22FE713F0200FF1
:104D800014BF412261220DF1480E0A3ACDE90D9778
:104D9000CDF844B000267746F3469146CDE90F3C66
:104DA00003E0202E17D004460D4629464246002334
:104DB000204606F01DFAD2B2092A02F1300388BF5C
:104DC00002EB09034445DBB275F1000507F8013B2E
:104DD00006F10106E5D2DE46DDE90D97DDE90F3C7F
:104DE000DDF844B0A6E6002A47D1134611463BE75A
:104DF0000B990968A1B923F0100388B10DF1480E91
:104E000006930C9BCDF80CC0CDE904730192D8E554
:104E100013F480627FF4CBAE23F010030D93CBE646
:104E200013F0200F14BF412061200DF1480E76468B
:104E3000A0F10A0802E0202AE2D02146B1FBFCF4EE
:104E40000CFB1415E8B2092D00F130058ABF40446F
:104E5000E8B2C0B2614506F8010B02F10102EAD2E4
:104E6000CEE7002A3FF456AF0DF1480E6BE7196804
:104E700081EAE174A4EBE174B0E600260DF1480E7E
:104E80002DE701362BE64FF00A081346C44671E5BC
:104E9000CDCCCCCC0EB410B585B007AC54F8043BE7
:104EA00001464FF0FF32009404480394FFF7FEFAE6
:104EB00005B0BDE8104003B0704700BFF9380010DE
:104EC00070B594461E4605460C4684B04FF0FF323E
:104ED000634602A900960348CDE90254FFF7E6FABB
:104EE00004B070BD4D3C00100FB410B50E4B84B033
:104EF00006A91C6851F8043B03915CB100914FF086
:104F0000FF3202A90948A047012004B0BDE81040C3
:104F100004B07047184600F0CDF9204604B0BDE853
:104F2000104004B0704700BF8C320020453C001098
:104F300010B5094B84B01C684CB1034600914FF08A
:104F4000FF3203A90548A047012004B010BD00F0BE
:104F5000B1F9204604B010BD8C320020453C001051
:104F600000BEFDE7074A0346106838B1064903440E
:104F70008B428CBF4FF0FF301360704703490846E7
:104F80001160F3E7F425002000000820E03700203E
:104F900008B5FFF7E5FF00BF9C46144600B50B4679
:104FA0000246614683B044B1054D06480194009520
:104FB000FFF79AFF0120FFF7D3FF034D2C46F4E7DC
:104FC00064B7001074B700100CB5001038B5064C6B
:104FD000064DFDF7CBFAAC4204D254F8043B984797
:104FE000AC42FAD338BD00BF50B2001058B2001026
:104FF0000368084611461847437D2DE9F04781466E
:105000000F461646002B43D0002A3BDD037D0020CF
:105010004D1E014615F8012FDFF884800A2A01F1A0
:1050200001040ED0A6421CD02B782146A3F10D031B
:10503000B3FA83F315F8012F5B090A2A01F1010481
:10504000F0D1002BEED18142A1EB000138441BDCF2
:1050500002214046D9F800309847A64208D02046A1
:10506000E2E7864204DD311AD9F800303844984727
:10507000374417F8013CA3F10D03B3FA83F35B093E
:1050800089F81430BDE8F087D9F800309847DFE799
:105090003846D9F800301146BDE8F047184700BF40
:1050A000D8B900100B682DE9F041802B0D4606465B
:1050B00005D05A1C2B442A601E71BDE8F0810F4BAD
:1050C0001C68A4B10E4F01F1040801E0246974B119
:1050D0002368002BFAD03B680BB1A342F6D12046DF
:1050E00041462A68FFF788FF2469002CF0D100238D
:1050F00001222B442A601E71BDE8F081E8250020C2
:10510000F02500202DE9F04782B00D4692469946E1
:105110000746FDF743F84FF0FF366FF000442F4A83
:10512000821841F10003964274EB03013CBF324602
:1051300023462B4806F068F86B1C804603D138469E
:1051400001F070FB0546274B274E1C68274BB9F131
:10515000000F18BF1E46B4B1BAF1000F1AD1DFF824
:10516000909001E0246974B12368002BFAD0D9F83B
:1051700000300BB19C42F5D120462A463946B04753
:105180002469002CF0D1B8F1000F1FD1284602B0DD
:10519000BDE8F0874FF00A0ADFF8549002E0246976
:1051A000002CF0D02368002BF9D0D9F800300BB1D7
:1051B000A342F4D12A4639462046B0470122204670
:1051C0000DF107018DF807A0B047E8E7044806F0A5
:1051D00013F8284602B0BDE8F08700BF40420F0038
:1051E00074110020E8250020F14F0010F94F001045
:1051F000F02500200A4A13684BB1834202D109E02E
:10520000984207D003F110021B69002BF8D101B1BD
:10521000106070470029FCD1036913600161704779
:10522000E825002008B500F0A5F9012008BD00BF61
:10523000F0B583B006468DF80700FCF7AFFF4FF0DE
:10524000FF356FF00044174A821841F10003954280
:1052500074EB03013CBF23462A46134805F0D4FFF4
:10526000124B07461C689CB1114D01E024697CB1CA
:105270002368002BFAD02B680BB19C42F6D1204654
:1052800001220DF10701FFF7B7FE2469002CEFD1D1
:1052900017B9304603B0F0BD034805F0ADFF304606
:1052A00003B0F0BD40420F0074110020E82500203B
:1052B000F025002038B5044601F0B4FA0123054674
:1052C0001A4620462946FFF71DFF084B1C682CB1E3
:1052D00063682BB198472469002CF9D1284638BD62
:1052E0002469002CF4D1284638BD00BFE8250020F1
:1052F0002DE9F041A2B004460D46FCF74FFF4FF0F8
:10530000FF376FF00046274A821841F100039742A9
:1053100076EB03013CBF3A463346234805F074FF61
:1053200000262B4607462246204801A90196FFF792
:10533000C7FD019B06467BB91D4B1C682CB16368F9
:1053400043B198472469002CF9D10FBB304622B0F5
:10535000BDE8F0812469F1E7DFF85480D8F8005007
:10536000EDB1144C01E02D6975B12B68002BFAD01A
:1053700023680BB1AB42F6D12846019A02A9FFF788
:105380003BFE2D69002DF0D1D8F800400195D5E7FE
:10539000054805F031FF304622B0BDE8F0810195A7
:1053A000D3E700BF40420F0074110020A550001049
:1053B000E8250020F02500200FB400B583B004A933
:1053C00051F8040B0191FFF793FF03B05DF804EB74
:1053D00004B07047B1F1000C1DDD0F4A0F4B12688D
:1053E00030B5D31AB3FA83F30D240D4D5B09411E7A
:1053F00035F913E08C4411F8010F864506D0936906
:105400009B06FCD461451060F5D130BD93699D06C3
:10541000FCD41460F3E77047D837002000800740C1
:10542000D4370020224BB1F1000C10B41C682EDDE3
:10543000034600201F4A591E12689369DB0617D4E1
:1054400001309369DB06FCD41368844501F8013F01
:10545000F3D14CB150211346916353F8342F02F02D
:10546000380203F580531A6060465DF8044B7047BC
:105470004CB150211346916353F8342F02F0380297
:1054800003F580531A6078B15DF8044B70475CB146
:10549000084B50211A681346916353F8342F02F0D9
:1054A000380203F580531A606FF00200ECE700BF8A
:1054B00088250020D8370020054B1B6833B1002118
:1054C000044A05481268006891631847704700BF96
:1054D00088250020D83700208C250020024B1A6830
:1054E00093691B07FCD47047D8370020F8B51C4FD0
:1054F0001C4D3A681C4EAA4214BF212522250446A1
:10550000D6F800C018B1BCF1000F10D0F8BDBCF146
:10551000000FFBD0014690632846FCF73BF9284674
:105520001249FCF78DF9124B34601C60F8BD0B4634
:105530000F4A0E49306028461360FCF751F90121EB
:105540002846FCF727F93A6850211346916353F82F
:10555000342F02F0380203F580531A60F8BD00BF03
:10556000D83700200080074088250020B95400105B
:105570008C25002010B50E490E4C0F480F4A104BD9
:10558000007821600020022112781B78FCF73CF89B
:1055900002210120FCF738F84FF4E1312068FCF7D4
:1055A00039FEBDE8104001210648FFF723BE00BFC9
:1055B00000000740D83700205C280110582801104F
:1055C00054280110900A00200B4B10B5DB6ADB0752
:1055D00009D40124094B0021DC620948FCF7E8FDED
:1055E000084BDC6210BD01210022064B4FF0FF305A
:1055F000D9621146FCF776FF0000104000201040F1
:10560000400D0300003010402DE9F84F374B07469E
:10561000984214BF4FF400234FF480230E46344DBC
:10562000344C354A2B602360946833EA0404FBD180
:105630000620FCF7D9FE3946022351F8042F4FEA21
:10564000462E4FEAD65B704502EA030801F5405941
:1056500074EB0B02C9F8003011D34FEA965CB2022A
:1056600001E05246AC460233B3F5807F07D01EEB13
:10567000020A4BEB0C05904274EB0C0CF1D24FF488
:105680008072C3EB03249446013A2DD0B0FBF4F5AD
:10569000AE42A4EB0304F6D20CFB03FC120202247C
:1056A0003B613B4603253E6801F500517240B0FB6B
:1056B000FCF002F47F4207F5805CCCF80020C1F8D2
:1056C00000807E68C9F8004053F8242B264082F001
:1056D000070202F0CF0203F50053CCF800200E6061
:1056E0001D600C60BDE8F88F9C46D8E700000840BC
:1056F00000200240003002400000024003BD00BF15
:1057000010B50446FCF742FF2346BDE81040184799
:105710004FF08071124B134A10B559605368D8018D
:10572000FCD51920FCF74CF8002104461920FCF7A1
:1057300031F84FF080714FF050420B4B5960136DB0
:10574000D90703D420BF136DDB07FBD54FF05043BF
:105750002146BDE8104019209B6DFCF71BB800BF27
:1057600000A001400080014000B00140F0B50546B6
:1057700087B0192017460E46FCF722F80021044690
:105780001920FCF707F80021CDE9046503970026EE
:10579000002701224FF050438C46CDE9006702926A
:1057A000B9B11A6D9507FCD5596540BF1A6DD00780
:1057B00003D420BF1A6DD207FBD59A6D8A420DD053
:1057C0004FF0000C06AA02EB8C0252F8181CE7E717
:1057D0009A6D1A6DD607FBD440BFE2E70CF1010CBD
:1057E000BCF1060FEED12146192007B0BDE8F0400C
:1057F000FBF7D0BF0C4B0D4A93420ED39C4603F2ED
:10580000F4710B4A9268CCF8F4070A48CCF8F837E0
:10581000CCF8FC070848FFF7A9BF4FF0FF3340F270
:10582000F3719C46EDE700BF000808200000082047
:1058300000ED00E001570010FD56001038B5A1FB47
:10584000021434BB00F042F8054630B350F8042C83
:1058500022F00302043A242A0CD8132A0FD91B2A57
:10586000C0E9004412D9242AC0E9024418D000F14A
:10587000100205E0214600F06DFD284638BD0246C5
:1058800000232846C2E90033936038BD00F10802C6
:10589000F6E700F0FDFD0C2303600025284638BD27
:1058A00000F11802C0E90444EAE700BF024B0146D8
:1058B000186800F00BB800BFB80E0020024B01467C
:1058C000186801F039B800BFB80E002001F10B03D1
:1058D000162B2DE9F04F074683B023D8102900F28C
:1058E000AF8000F09DFA102518230220BC4E3344EF
:1058F0005C68A3F10802944200F080816368384636
:1059000023F00303D4E902122344CA6091605A6869
:10591000083442F001025A6000F088FA204603B0D1
:10592000BDE8F08F002B23F00705C0F28980A94263
:1059300000F2868000F074FAB5F5FC7FC0F0B48107
:105940006B0A00F08180042B00F27E81AB0903F129
:10595000390003F1380EC300A14E3344A3F1080C03
:105960005C68A44507D10DE0002AE16880F232812D
:105970008C450C4606D0636823F003035A1B0F2A9C
:10598000F2DD7046DFF870823469444500F0E7804C
:10599000636823F0030CACEB05030F2B00F3948139
:1059A000002BC6E9048880F28381BCF5007FD6F81D
:1059B00004E080F029814FEADC0301224FEA5C1CFD
:1059C000013302FA0CF256F833104EEA020E06EBDF
:1059D000C302083AC6F804E0C4E9021246F83340AC
:1059E000CC6083104FF0010C0CFA03FCF44531D865
:1059F0001CEA0E0F07D120F003004FEA4C0C0430D4
:105A00001CEA0E0FF9D006EBC00A8146D646DEF836
:105A10000C300BE05A681C46DB6822F00302511B75
:105A20000F2900F31D81002980F231819E45F1D1BB
:105A300009F101090EF1080E19F0030FE7D167E132
:105A40000C233B60002469E74FF4007340204FF0C3
:105A50003F0E81E7B468636823F00309A9EB0503EF
:105A60000F2B02DDA94580F0A4805E4B08201B6847
:105A700003F1100804EB0903009300F013FD5A4AE8
:105A8000A84483461368013305D008F1FF38434228
:105A9000804403EA08084146384600F0E7FCB0F1CC
:105AA000FF3F8246504A79D0009B83425AD9B44284
:105AB00074D14E4B0BF1FF3C186800EB080EC3F895
:105AC00000E01168013100F07381009AAAEB020234
:105AD00072441A601AF00702CDE9002300F04281F7
:105AE000C2F10802384692445A44D04408EA0C01F4
:105AF000521A02EA0C0B594600F0B8FC421C019BFA
:105B000000F06E81A0EB0A0000EB0B08196848F06A
:105B10000102B442C6F808A05944CAF8042019602A
:105B200032D0B9F10F0F40F20C816068A9F10C027C
:105B30004FF0050C22F0070200F0010010430F2A7D
:105B4000606004EB0200C0E901CC1DD904F108013A
:105B50003846009300F0F0FE009B196814E0D6F878
:105B600004E03EE7214B0BF1FF3C196841448E46AF
:105B70001960A6D1009810EA0C0FA2D109EB080316
:105B8000B26843F001035360194B1A688A4238BF68
:105B90001960184B1A688A4238BF1960B468626885
:105BA00022F00302531B0F2B40F3CE80954200F2EC
:105BB000CB80621945F0010543F00103083444F835
:105BC000045C3846B260536000F030F9204603B000
:105BD000BDE8F08FA26823443846D1608A6096E61B
:105BE000B00A0020F4130020A80A0020C4130020EB
:105BF000EC130020F0130020B80A0020DC68A34258
:105C00007FF47CAE0230BDE6BCF5206F4FEA5C222B
:105C10006CD3142A00F2B98002F15C035B32DB0022
:105C2000F118F3580839994203D191E09B689942E1
:105C300004D05A6822F003026245F7D8D968C4E953
:105C400002318C60DC60CCE6142B56D9542B00F268
:105C5000A5802B0B03F16F0003F16E0EC3007BE6F2
:105C6000D4F808C03846671945F001056560CCF8DE
:105C70000C30C3F808C041F00103C6E90477C7E956
:105C800002887B60A150083400F0D0F846E6224438
:105C90003846516841F00101516054F8082FD36033
:105CA0009A6000F0C3F839E6E80805F108031DE63C
:105CB000A44438460834DCF8043043F00103CCF83F
:105CC000043000F0B3F829E6621943F0010145F011
:105CD000010538466560C6E90422C2E902885160C0
:105CE00044F80C30083400F0A1F817E64FEA9C1293
:105CF00002F139033832DB0092E703F15C0003F173
:105D00005B0EC30028E65AF80839534540F08580F9
:105D100010F0030F00F1FF30F5D1736823EA0C0394
:105D200073604FEA4C0C0CF1FF329A4204D391E6B7
:105D30004FEA4C0C09F104091CEA030FF8D048465D
:105D400061E60123CAF80430384600F06FF879E6BE
:105D500092104FF0010C0CFA02F24EEA020EC6F855
:105D600004E06CE70AEB0802384602EA0C02ABEBEF
:105D7000020B0BEA0C0B594600F078FB431C019B0D
:105D80007FF4C0AEDDF800B0C0E6542A13D84FEA65
:105D90001C3202F16F036E32DB0041E7B3F5AA7FDC
:105DA00013D8EB0B03F1780003F1770EC300D3E5B2
:105DB000C2F800A08EE6B2F5AA7F19D84FEADC320D
:105DC00002F178037732DB002AE740F25452934223
:105DD00019D8AB0C03F17D0003F17C0EC300BBE5C9
:105DE000009A4FF0000B083A9044A8EB0A088DE6A1
:105DF00040F254539A420CD84FEA9C4202F17D0380
:105E00007C32DB000CE74FF47E737F204FF07E0E78
:105E1000A2E54FF47E737E2202E7736881E700BF3C
:105E2000014800F03BBB00BFC0130020014800F058
:105E300037BB00BFC01300200C4B0D4819680D4A3A
:105E4000D1F8983010B403FB00F0D1F89C4002FB6D
:105E500004005DF8044BA3FB0232013340EB020067
:105E6000C1E9263020F00040704700BFB80E002086
:105E70002DF451582D7F954C024B0A460146186867
:105E800000F002B8B80E00202DE9F04F164683B09E
:105E9000002900F09E800C4606F10B058046FFF7B6
:105EA000BFFF54F8040C162DA4F1080920F00307D5
:105EB00062D8102200231546B542C0F0A280002B04
:105EC00040F09F80974261DADFF828B309EB0701C1
:105ED000DBF80830D1F804C08B4200F097802CF03A
:105EE00001030B445B68DB0768D42CF0030C07EB61
:105EF0000C03934245DAC30712D454F8083CA9EBCB
:105F0000030ADAF8043023F0030084440CEB070B97
:105F10005A4540F3FE8007EB000B5A4540F3D4800E
:105F200031464046FFF7D2FC0646002800F02981A2
:105F300054F8043CA0F1080223F001034B449342BF
:105F400000F0B1803A1F242A00F2DF80132A00F209
:105F5000B080034622461168196051685960926802
:105F60009A602146404600F0E7FC4046FFF75EFF9E
:105F7000304603B0BDE8F08F25F007052A46EB0F49
:105F80009AE71F46D1E90223D3609A60781BD9F8BB
:105F9000043009EB07020F2803F001031FD83B432D
:105FA000C9F80430536843F0010353602646404665
:105FB000FFF73CFF304603B0BDE8F08FC307AFD416
:105FC00054F8083CA9EB030ADAF8043023F0030084
:105FD000A1E7114603B0BDE8F04FFFF777BC2B43B4
:105FE00009EB050140F00100C9F80430083141F81F
:105FF000040C4046536843F00103536000F09CFCDE
:10600000D4E70C23C8F800300026D3E72CF0030CAB
:1060100005F110010CEB07038B4280F29280C00760
:106020003FF57EAF54F8083CA9EB030ADAF80430D8
:1060300023F0030084440CEB070399423FF76BAF56
:106040003A1F5646DAF80C1056F8080F242AC16099
:10605000886000F2B080132A40F2AB8021681B2ACE
:10606000CAF808106168CAF80C1000F2AB80083456
:106070000AF110022168116061685160A1689160A5
:106080005B1B0AEB0502404643F00103CBF80820F6
:106090005360DAF8043003F001032B43CAF80430EC
:1060A000FFF7C4FE86E750F8043C23F003031F44C7
:1060B0006CE723681B2A03606368436036D804F1E9
:1060C000080200F1080346E73A1F5646DAF80C309A
:1060D000242A56F8081FCB60996022D8132A1ED9AB
:1060E00023681B2ACAF808306368CAF80C303CD809
:1060F00008340AF1100322681A6062685A60A268C4
:106100009A6034465F46D14640E7214600F0A2F847
:1061100027E7D1E902133A1FCB609960D5E73346F0
:10612000E9E72146304600F095F8EAE7A368242A1B
:106130008360E368C36028D004F1100200F110030B
:1061400009E75B1B09EB05024046264643F00103C5
:10615000CBF80820536054F8043C03F001032B43B0
:1061600044F8043CFFF762FE24E7A368242ACAF837
:106170001030E368CAF8143010D010340AF1180354
:10618000B9E74046FFF752FE3EE7236904F11802E3
:1061900003616369436100F11803DCE62369183485
:1061A000CAF8183054F8043CCAF81C300AF120032D
:1061B000A1E732465EE721463046019300F04AF8F7
:1061C000019B5DE7A168242ACAF81010E168CAF8AB
:1061D000141003D010340AF118024BE72269183466
:1061E000CAF8182054F8042CCAF81C200AF120021E
:1061F00040E700BFB00A00200EB470B59DB0002586
:106200004FF4017221AC1B95ADF8142054F8046BC7
:106210000290069000F006FB0B4903464FF6FF7014
:1062200032460A910949ADF81600039307932346B5
:10623000086802A90E951395019400F0BBFD1DB0EE
:10624000BDE8704003B0704751620010B80E0020E6
:106250000020704788420ED98B1883420BD900EB7F
:10626000020C002A6ED0624613F801CD994202F862
:1062700001CDF9D170470F2A0FD8034602F1FF3C38
:10628000002A5FD00CF1010C013B8C4411F8012B6A
:10629000614503F8012FF9D1704740EA01039B07DC
:1062A00051D1A2F1100301F1200C70B523F00F05BC
:1062B00001F1100E00F110041B09AC445EF8105CF3
:1062C0000EF1100E103444F8205C5EF81C5C44F8AB
:1062D0001C5C5EF8185C44F8185C5EF8145CE645DB
:1062E00044F8145CEAD1013312F00C0F02F00F0CE9
:1062F00001EB031100EB031329D0ACF1040C1C1FBC
:106300008E462CF003064FEA9C0C1E445EF8045B9C
:1063100044F8045FB442F9D10CF1010402F0030225
:1063200003EB840301EB840102F1FF3C4AB10CF161
:10633000010C013B8C4411F8012B614503F8012F3E
:10634000F9D170BD704702F1FF3C03469AE76246FF
:10635000EAE700BF70B5860747D0541E002A3ED03A
:10636000CAB2034601E0013C39D303F8012B9D0773
:10637000F9D1032C2CD9CDB20F2C05EB052505EB5B
:10638000054535D9A4F1100C03F1100E1A462CF076
:106390000F064FEA1C1CB644C2E90055C2E902557B
:1063A00010327245F8D10CF1010214F00C0F04F018
:1063B0000F0C03EB021213D0ACF1040323F0030320
:1063C0000433134442F8045B9342FBD10CF0030402
:1063D0002CB1C9B21C4403F8011BA342FBD170BD10
:1063E00064461346002CF4D1F9E703461446C0E78F
:1063F0001A46A446E0E700BF024A01231268503261
:1064000000F002B8B80E002018B3F0B407468C466E
:1064100017F8015B01E0A54214D01CF8014B002CD9
:10642000F9D1DDB13E460C4616F8015B00E063B1E0
:1064300014F8013B9D42FAD14DB100233B70166028
:10644000F0BC704773B13846E0E73746EAE72E46BE
:10645000F5E710680028D8D10020704700201560AB
:10646000F0BC704717600370EAE700BF38B5002240
:10647000064D044608462A60FEF774FD431C00D012
:1064800038BD2B68002BFBD0236038BDEC250020E5
:10649000014B1868704700BFB80E0020704700BF5E
:1064A000704700BF082802D14FF48050704708B5EC
:1064B000FFF7EEFF162203464FF0FF301A6008BDCB
:1064C00080EA010C1CF0030F37D110F0030C20F010
:1064D000030021F0030150F8042B08BF51F8043BDE
:1064E0000ED08CF0030C6FF07F434FEACC0C23FAF4
:1064F0000CFC51F8043B42EA0C0243EA0C0300BFD7
:10650000A2F1013C9A4201BF2CEA020C1CF0803F30
:1065100050F8042B51F8043BF2D04FEA02604FEAE6
:106520001222012828BFB0EB036F08BF1B0AF4D06A
:1065300003F0FF03000EC01A704710F0030F0AD0DB
:1065400010F8012B11F8013B012A28BF9A42F4D020
:10655000A2EB030070474DF8045D50F8042B01F0E6
:10656000030521F0030151F8043B022D26D04DD83C
:1065700022F07F45B5EB132FA2F1013C2CEA020C6F
:106580000DD11CF0803C08BF51F8043B0AD185EACC
:106590000205B5EB036F0CD150F8042BE8E74FEA86
:1065A00013235BE03CF07F4C54D10B784FEA12652B
:1065B00054E04FEA126503F0FF034FE04FEA024553
:1065C000A2F1013C4FEA15452CEA020CB5EB134F42
:1065D00018D11CF0803C08BF51F8043B07D185EA74
:1065E0000205B5EB034F09D150F8042BE6E75FEA4B
:1065F0000C4C2FD10B884FEA12452FE04FEA034392
:106600004FEA12454FEA134328E000BF02F0FF05AE
:10661000B5EB136FA2F1013C2CEA020C0DD11CF07A
:10662000803C08BF51F8043B0AD185EA0205B5EB6E
:10663000032F0AD150F8042BE8E74FEA13630DE06B
:1066400012F0FF0F06D051F8043B4FEA122523F059
:106650007F4303E04FF0000020BC704705F0FF02CD
:1066600003F0FF00012828BF904204BF2D0A1B0A37
:10667000F4D0A2EB000020BC704700BF80EA01020A
:10668000844612F0030F4FD111F0030F32D14DF8B1
:10669000044D11F0040F51F8043B0BD0A3F101326B
:1066A0009A4312F0803F04BF4CF8043B51F8043B7E
:1066B00016D100BF51F8044BA3F101329A4312F0F6
:1066C000803FA4F101320BD14CF8043BA24312F0FD
:1066D000803F04BF51F8043B4CF8044BEAD02346FA
:1066E0000CF8013B13F0FF0F4FEA3323F8D15DF8AC
:1066F000044B704711F0010F06D011F8012B0CF874
:10670000012B002A08BF704711F0020FBFD031F8EB
:10671000022B12F0FF0F16BF2CF8022B8CF8002072
:1067200012F47F4FB3D1704711F8012B0CF8012BF5
:10673000002AF9D1704700BF844641EA000313F0F4
:10674000030349D1403A23D30B6803604B6843608D
:106750008B688360CB68C3600B6903614B694361DD
:106760008B698361CB69C3610B6A03624B6A4362C5
:106770008B6A8362CB6AC3620B6B03634B6B4363AD
:106780008B6B8363CB6BC36340304031403ADBD2C9
:1067900030320BD30B6803604B6843608B688360B7
:1067A000CB68C36010301031103AF3D20C3205D3ED
:1067B00051F8043B40F8043B043AF9D2043208D0C3
:1067C000D2071CBF11F8013B00F8013B01D30B8835
:1067D00003806046704700BF082A13D38B07B1D0EF
:1067E00010F00303AED0C3F10403D21ADB071CBFC1
:1067F00011F8013B00F8013BA4D331F8023B20F82B
:10680000023B9FE7043AD9D3013A11F8013B00F863
:10681000013BF9D20B7803704B7843708B7883700F
:106820006046704720F0030110F00300C0F1000043
:1068300051F8043B00F1040C4FEACC0C6FF000025D
:106840001CBF22FA0CF213434FF0010C4CEA0C2C43
:106850004CEA0C4CA3EB0C0222EA030212EACC1223
:1068600004BF51F8043B0430F4D0C2F1000102EA45
:106870000102B2FA82F2C2F11F0200EBD2007047AD
:106880002DE9F8430646DFF8AC8008208946FFF77B
:1068900009FE05463046FFF7C3FAD8F808305F68AE
:1068A00027F00307A7F11104A4EB09042C44B4FB5F
:1068B000F5F4013C05FB04F4A54208DC0021304658
:1068C000FFF7D4FDD8F808303B44984205D0304655
:1068D000FFF7ACFA0020BDE8F88361423046FFF7CD
:1068E000C5FD01300FD03F1B104AD8F808303046A4
:1068F00047F001075F6013681B1B1360FFF796FAF0
:106900000120BDE8F88300213046FFF7AFFDD8F83D
:106910000820831A0F2BDADD43F00103034953608B
:10692000034B1B68C01A0860D1E700BFC4130020E6
:10693000A80A0020B00A002000297CD02DE9F041EF
:106940000C468046FFF76CFA764F54F8043CA4F1ED
:106950000805BE6823F0010168184268864222F0EB
:10696000030200F08380DE0700EB020C426033D4A8
:1069700054F8084CDCF8043007F1080C2D1B2144B6
:1069800003F00103AC68644564D0D5F80CE0C4F8AA
:106990000CE0CEF80840002B00F0818041F00103AC
:1069A0006B600160B1F5007F22D2CB08012249095A
:1069B00001338A4079680A4357F833107A6007EB4D
:1069C000C302083AC5E9021247F83350CD60404689
:1069D000BDE8F041FFF72ABADCF80430DB072BD51D
:1069E00041F00103B1F5007F44F8043C0160DCD3C1
:1069F000B1F5206F4FEA512353D28B0903F13900CF
:106A000003F13802C300F818FB580838984203D144
:106A100061E09B68984204D05A6822F003028A42DF
:106A2000F7D8D868C5E9023085604046DD60BDE82A
:106A3000F041FFF7FBB97047114407F1080C836878
:106A400063453FD0C268DA60936041F001036B6038
:106A50006950A7E7002B5FD10A44D0E90213CB604D
:106A6000996042F001036B60AA50B0E7DB070A446B
:106A700007D454F8083CED1A1A44D5E90213CB6048
:106A8000996042F001036B60274BBD601B68934225
:106A90009DD8264B40461968FFF7F2FE97E7114450
:106AA000CDE7142B08D9542B1DD80B0B03F16F0025
:106AB00003F16E02C300A6E703F15C0003F15B0281
:106AC000C300A0E741F00103C7E90455C5E902CCC2
:106AD0006B6069507BE70121921001FA02F279683C
:106AE0000A437A609EE7B3F5AA7F06D8CB0B03F181
:106AF000780003F17702C30085E740F254529342D5
:106B000006D88B0C03F17D0003F17C02C3007AE709
:106B10004FF47E737E2276E741F001036B600160E3
:106B200055E700BFB00A0020AC0A0020F413002093
:106B30002DE9F04780460C464548264614F801EBFF
:106B400010F80EC01CF0080CF7D1BEF12D0F5BD071
:106B5000BEF12B0F3AD0654633F010003ED04FF017
:106B6000FF379A46B7FBF3F703FB07F96FEA09090A
:106B7000002630460EE0AEF1370C63451DDD002ED9
:106B800004DBB84202D833D1CC4531DD4FF0FF36BB
:106B900014F801EBAEF1300CBCF1090FEDD9AEF1F8
:106BA000410CBCF1190FE6D9AEF1610CBCF1190F23
:106BB00003D8AEF1570C6345E1DC731C1CD005B162
:106BC00040420AB1F6B91160BDE8F08733F0100019
:106BD00094F800E0654606F10204C0D1BEF1300F22
:106BE00017D06BBB0A234FF005091A4F9A46BFE72F
:106BF00000FB0AC00126CBE722233046C8F800304C
:106C0000002AE1D0611EDEE794F800E00125B41C03
:106C1000A2E7207800F0DF00582807D083B90823C6
:106C20004FF007096FF060479A46A1E7102394F8E8
:106C300001E04FF00F0902346FF070479A4697E772
:106C400010234FF00F096FF070479A4690E700BF8E
:106C500005BA001099999919FFF76ABF38B54B1C0E
:106C60001AD0938914465268CDB223F02003A38131
:106C7000236BA3B1636B934209DD23685A1E226024
:106C800003F8015C636801336360284638BD214620
:106C900001F03AFD0028F0D04FF0FF35F5E7236909
:106CA00021682BB18B4203D211F8013CAB420ED0CC
:106CB000234604F14000C4E90E120321012220639F
:106CC0002846616303F8425FC4E9003238BD0139E8
:106CD0000132C4E90012D8E710B50C46096B69B15E
:106CE00004F14003994201D0FFF726FE0020E36B38
:106CF0002063636013B1A36B236010BDA2890021E0
:106D000023694FF0FF3042F020026160A281F3E777
:106D10002DE9F04F834685B002FB03F00E9C0193F2
:106D2000A0B388460646D4E90015A84223D94FF0FF
:106D3000000904F1400ACDE9020240462A46FFF765
:106D4000FBFC2168236B58464F19A8441946C4F828
:106D5000049027603746761BDBB1534501D0FFF71F
:106D6000EBFDE06BC4F83090606090B1A16BB04275
:106D700005462160E1D332464046FFF7DDFC01982D
:106D8000D4E90032921B3344C4E9003205B0BDE8B7
:106D9000F08FDDE90202A389284443F02003C01BE1
:106DA000A3810023B0FBF2F02269C4E9002305B0FF
:106DB000BDE8F08F2DE9F04FADF5377D8A4602AF83
:106DC000C7E91202B1F90C20FB6296044B6E05D4A0
:106DD00042F4005223F400538A814B669D04C3F3AE
:106DE000403401F18C80A1460822214607F1580069
:106DF000FFF7B0FABC63FC617C633C64BC62954BFA
:106E0000D3F8E44001F03AFD07F15802034607F1D8
:106E100054010092FA6CB86CA04700285CDBFB6C54
:106E200002460344FB647B6D002B00F0D4800128F4
:106E300061D0252B68D00028E1D0FB6C01389E1A68
:106E4000DAF804301A463418751E002A16DDDAF80E
:106E50000030691C6A7818780133904240F0BB809A
:106E6000DAF804208C42CAF8003002F1FF32CAF886
:106E7000042000F0BB80002A0D46E8DC5146B86CC7
:106E8000FFF72AFF0028E2D03B6C002B40F09E80E9
:106E9000BB6B002B01F03380BB6BDE8818687EB1C2
:106EA0000024051F8146A04655F8043F01341868A8
:106EB000FCF712FD2B68A642C3F80080F4D14846C7
:106EC0004FF0FF333B6408B1FCF706FD386C07F563
:106ED0003577BD46BDE8F08F4FF6FD7308220021DF
:106EE00007F158007B65FFF735FAFB6C0133FB6453
:106EF0007B6D002B6FD0584AD25C140700F1F184EF
:106F00000120252B024698D10024FE6C25463178BD
:106F1000A1F1250306F1010B552B5CD8DFE813F036
:106F20004F075B005B005B005B0031075B005B00B1
:106F30005B005B005B001E061E061E061E061E068C
:106F40001E061E061E061E061E065B005B005B007C
:106F50005B005B005B005B002B065B005704770067
:106F60002B062B062B065B005B005B005B007000B2
:106F70005B005B0066045B005B005B00AC045B00D5
:106F80005B005B005B003C065B005B0039075B005D
:106F90005B005B005B005B002B065B005904790023
:106FA0002B062B062B060107530770005B004307D7
:106FB0000D071B0768042E075B005B00AE046B0027
:106FC000FA065B005B003C065B006B00BAF80C3015
:106FD0005A063FF55DAFBB6B002B3FF477AFBB6B41
:106FE00018683B6C01337FF46EAF55E702354D44B2
:106FF000A5EB060903E72307EDD171785E4687E725
:107000002107E8D1717844F002045E4680E744F03D
:107010000104124B0326BB620A237B63DAF80430B7
:10702000002B00F3EF835146B86CFFF755FE0028A4
:107030007FF42AAFC7F84CB0600641F10682731E98
:10704000032B01F26981DFE813F02D02DE01340128
:107050000B0000BF0010002005BA00107999001045
:10706000B86C44F4F06801F00FFC03683B626B1EDF
:10707000B3F5AE7F40F232876FF4AE7405EB040CCB
:1070800040F25D1507F5B87B0023C7F80CC05C46DD
:107090007B64FB633B63BB61C7F824B0C7E904337F
:1070A000DAF800100A78A2F12B034E2B50D8DFE853
:1070B00013F039034F0039034F004F007D039D004B
:1070C0009D009D009D009D009D009D009D009D00D8
:1070D0004F004F004F004F004F004F004F002E0356
:1070E0009A009A009A00600355034F004F00400336
:1070F0004F004F004F004F000E034F00EE024F00B5
:107100004F004F00E7024F004F004F00D20227030D
:107110004F004F004F004F004F004F004F002E0315
:107120009A009A009A00600355034F004F004003F5
:107130004F004F004F004F000E034F00EE024F0074
:107140004F004F00E7024F004F004F00D2022703CD
:1071500018F4007F67D0386A0378934263D183467E
:107160000026C7E901545546C24606E029609BF84F
:10717000000091F800E086451BD11BF8010F344652
:10718000C8460131013609F10109002800F0918655
:107190006868013800286860E8DC2946B86CFFF7A9
:1071A0009BFD30B929689BF8000091F800E0864506
:1071B000E3D04346D046AA462246BC689146D7E96A
:1071C000085B7C622E443B623446BE6C14F8011DA1
:1071D00052463046FFF742FDA542F7D13B6A7C6A32
:1071E000A3EB090921E018F4006F1CD0FB6B796C4C
:1071F0005B1818D128F4C0787B64FB6304F8012B7A
:10720000013DDAF8043009F10109013B002BCAF80D
:10721000043040F35B83DAF800300133CAF8003001
:10722000002D7FF43DAFD7F824B03B6B0BB128F4B1
:107230008078FB6B013B012B41F2DE807B6C013BD4
:10724000062B40F27C8618F4807F00F06A8418F4E4
:10725000806F40F0948714F8011C01F0DF03452B88
:1072600040F09786651E09F1FF395246B86CFFF76A
:10727000F5FC18F010037FF4C2AD2B707B69002B76
:1072800040F0A08700225946B86C02F0E9FAFB6A88
:1072900018F0010F024605460E4603F1040400F003
:1072A0006D861B68C3E900563B6CFC6201333B648E
:1072B000A5E56B1E44F45864B3F5AE7F40F2A98394
:1072C0006FF4AE72A91840F25D1507F5B87B4FF068
:1072D00000087A6B5E46CB46D146C246B046F9639B
:1072E000D9F8000090F800C0ACF12B034D2B62D808
:1072F000DFE813F056026100560261006100C70228
:10730000AB01AB01AB01AB01AB01AB01AB01430284
:107310004302610061006100610061006100610081
:107320004E004E004E004E004E004E0061006100C7
:107330006100610061006100610061006100610045
:1073400061006100610061006100610061004A024A
:107350006100610061006100610061006100610025
:107360004E004E004E004E004E004E006100610087
:107370006100610061006100610061006100610005
:1073800061006100610061006100610061004A020A
:107390000A2A10DD24F4386406F801CBD9F8043049
:1073A000013B002BC9F8043040F386820130C9F854
:1073B0000000013D94D14346E105D0467A63CA46B8
:1073C000D9469B4605D59E4200F29B845E453FF41C
:1073D00002AE14F0100211D17B6B5946BD6A3270B7
:1073E000B86CA847FB6AA20603F1040540F1E183EB
:1073F0001B6818603B6CFD6201333B64A6EB0B0617
:107400004644B144FBE4002D04F0100208BF4FF0E5
:10741000FF35E00740F1FF82002A40F01D85FE6A3B
:10742000210656F804BB40F1D7867A64BBF1000F01
:107430003FF4D1AD8020FCF715FA7A6C03460028A2
:1074400000F0D587B96BCBF80000CC88B1F8048088
:10745000444580F0D9850868B96B9E4640F824B051
:107460004FF0200C0134FE62CC80DAF80010DFF817
:10747000BC83097818F8016016F0080600F0B8839C
:10748000002A7FF4BCAC1A60A3EB0E039910013103
:107490008C4503D9BBF1000F40F028863B6C0133CB
:1074A0003B64ACE4002D04F0100308BF4FF0FF353F
:1074B000E0073B6340F13582D7F82CB0002B40F059
:1074C000C2845BF8043B21063B6240F18C86002BB2
:1074D0003FF481AD8020FCF7C5F98046002800F01C
:1074E00086873B6A1860BB6BDC889A88944280F080
:1074F000A58518683B6AC7F82C8040F82430013411
:10750000BB6BDC8020237B62C7F818B00024FE69C7
:10751000CB467D6401F0B2F9A0423FF4B5AC032E36
:1075200007F16009DAE9003202F1FF3213F8011BBA
:10753000CAF8042007F5B872CAF80030115504F1F2
:10754000010403D1D9F80030042B04D00822002113
:107550004846FEF7FFFECDF8009007F5B8722346C7
:107560004146B86C02F0A2FB421C06463FF48CACCC
:10757000002840F079840346C8F800000822002162
:1075800007F16800FB63FEF7E5FEFB6BB86C07F1E3
:1075900050011A46A24BD3F8E0301D4607F16803AC
:1075A000A84701280CBF97F85030002307F170025C
:1075B000D35C002B00F02386032EA34400F05D84EF
:1075C0007B6C013B7B643B6BBBB908F10408F86A38
:1075D0007D6AA8EB0004B5EBA40F0ED83B6A63B13B
:1075E000E900FCF75BF9F862002800F00087690009
:1075F0003B6A00EB040879621860DAF80430002472
:10760000002B40F346847B6C002B83D1D946D7F8FE
:1076100018B0FE613B6BA3B9C8F80030FB6A7A6A08
:10762000A8EB03018B1001339A4207D93C6A2CB1B5
:1076300004312068FCF732F900B120603B6C013363
:107640003B64C7F82CB0FFF7DABB764B24F4386400
:1076500033F91220A0E608F41863B3F5807F7FF4B5
:10766000E2AD3B6B012B7FF4DEAD302328F4807854
:10767000013D04F8013B002348F400683B63BDE58D
:107680007B6C062B7FF4CFAD07237B64B6E518F443
:10769000006F3FF4C8AD08F4A063B3F5806F07D066
:1076A00018F4806F3FF4BFAD3B6B002B00F0B38646
:1076B00018F4007F04D13B6BB9695B1AC7E9044336
:1076C00028F47868002348F4C0783B6396E5FB6BA8
:1076D000002B40F075823B6B002B40F0718208F468
:1076E000E063B3F5E06F00F0A1857B6C012B02D065
:1076F000042B7FF498AD7B6C0133DBB27B647DE5BA
:107700007B6C072B7FF48FAD08237B6476E518F440
:10771000006F40F03A82FB6B012B7FF484AD0223B3
:10772000FB636BE518F0800F3FF47DAD28F0800817
:1077300064E57B6C002B40F04B823B6B002B40F0F0
:10774000478208F4E063B3F5E06F00F0778500232B
:10775000D7F824B07B6400233B636AE518F4006F1C
:1077600040F00C827B6C022B7FF45DAD03237B64C5
:1077700044E518F4006F8ED038E52A4B33F9122017
:10778000082A3FF707AE16E604F4C063B3F5007F9E
:107790007FF411AE24F40074102244F4A064FBE5DD
:1077A00023067FF508AE24F08004F5E518F4807F09
:1077B0003FF41CAD3B6B28F0800801333B63FB6852
:1077C000002B3FF41DADFB68013BFB6019E544F065
:1077D000010444F040040026C7F84CB0DAF8043045
:1077E000002B3FF729ACD7F84CB01CE444F001045F
:1077F0000D4B0326BB6208237B63DAF80430002BB1
:107800007FF711ACDAF80020DFF82080137818F841
:107810000330190740F124854346D0469A460EE0CE
:107820000010002008BB0010596C001005BA0010B1
:10783000C8F8002013781AF803301B0717D5D8F8BA
:10784000043009F101090132013B002BC8F8043072
:10785000EEDC4146B86CFFF73FFA002840F0488361
:10786000D8F8002013781AF803301B07E7D4C24673
:10787000C7F84CB0FFF7E3BB44F001040226FFF762
:10788000CDBB23057FF588AD12B944F400740822FE
:10789000610500F18A81FB6B24F4607413B1013B34
:1078A0000135FB63D9F804300AF1010A013B002BD2
:1078B000C9F804303FF77AAD4946B86C7A64FFF7EF
:1078C0000BFA7A6C00283FF474AD74E55146B86C3D
:1078D000FFF702FA00287FF4A6AC002D7FF4E0AB9E
:1078E000A1E4DAF80420BC6C11E0DAF80030BD49FC
:1078F0001A7801338A5C10077FF581AADAF8042030
:1079000009F10109CAF80030013ACAF80420002A36
:10791000EBDC51462046FFF7DFF90028E5D0FFF702
:107920006EBA3B6B002B40F05682FB6A53F8042B77
:107930003B6314F080031646FA6300F05C84002A6F
:107940003FF449AB2020FBF78DFF044600283FF4AD
:107950009FAABB6B3060B3F80480DE88464580F098
:107960003A831868FB6B40F826300136BB6BDE802B
:107970002023DAF8000007F170020178515C002939
:107980003FF429ABF96B2646C7F82C909046B1F12D
:10799000000B994618BF4FF0010B07E0DAF8000022
:1079A000027818F80220002A00F0B282DAF80420E7
:1079B000411C013ACAE90012027804F8012BA21B0B
:1079C0004A457A6410D33046BBF1000F0CD04FEA21
:1079D00049094946FBF762FF064600283FF458AACA
:1079E0007A6CFB6B84181860013D00F09182DAF824
:1079F0000420002AD2DC5146B86CFFF76DF900284C
:107A0000CCD0B4424B46D7F82C903FF43DAAA61BED
:107A100084E2002159E4002A40F07483FA6A14F0E9
:107A2000800452F8043B7B64FA6300F0C0831C4678
:107A3000002B3FF4D0AA2020FBF714FF06460028B5
:107A40003FF426AABB6B2060B3F80480DC88444571
:107A500080F0AA8218687B6C4FF0010B40F824304C
:107A60000134BB6BDC802023DAF80000DFF874817E
:107A7000017818F80110090700F1AB82424634463C
:107A8000314698462E464B469146DAF804200D467C
:107A9000013ACAF80420421CCAF80020027805F80E
:107AA000012B2A1B42453A6312D32046BBF1000F3B
:107AB0000ED04FEA4808FB624146FBF7EFFE044652
:107AC00000283FF4E5A97B6C3A6B18608518FB6AC7
:107AD000013E0CD0DAF80420002A40F3B783DAF82C
:107AE00000002946027819F802201207CDD59946E0
:107AF000291B43462E468944013100208B423070B9
:107B000008D9BBF1000F05D07C6C2068FBF7C6FEDE
:107B100000B120603B6C01333B64FB6BFB62FFF701
:107B20006EB918F010037FF46AA9237008F4C063DB
:107B3000B3F5806F7FF4A2ABBB693A6B93423FF41D
:107B4000A1AB9A1A07F2C32327499C4228BF07F228
:107B5000C2242046FDF79EF9FFF794BB14F08F0F67
:107B60007FF439AA05EB850501EB450571785E4682
:107B7000303DFFF7CDB90426FFF750BAFB6B796CA7
:107B80005B187FF4EFADFFF735BBFB6B796C5B18CF
:107B90007FF4C1ADFFF72EBB44F40074134B0326F2
:107BA000BB6210237B63FFF739BA24F4B064FFF79C
:107BB000F3BB210740F16282FB6A1B68187019E46D
:107BC000FB6B022B7FF491AD0323FB63FFF716BB26
:107BD0007B6C032B3FF48FAD052B3FF48CADFFF78F
:107BE00022BB00BF05BA0010E8B70010596C0010A6
:107BF000C7F824B0C7F82080A846D7F81CB01D46A7
:107C0000C7F830E0C7F83CC07A6400F037FEB042F5
:107C10003FF43AA9BBF1030F07F16804DAE9003237
:107C200002F1FF3213F8011BCAF8042007F5B872FD
:107C3000CAF80030915506F1010602D12368042BE1
:107C400004D0082200212046FEF784FB009433462E
:107C500007F5B8722946B86C02F028F8B0F1FF3F7A
:107C600083463FF411A9002800F02F8210F1020F83
:107C70002CD0286802F044F8002840F01E83BBF1A5
:107C8000030FB14402D12368042B01D008F1FF385F
:107C90007E6C002E40F089820435386BFB6B2C1A09
:107CA000B3EBA40F00F281827A6A002A00F07D8291
:107CB000D900FBF7F3FD01463863002800F09783F5
:107CC000FB6B051958007B6AF8631960DAF8043019
:107CD000002B40F3C982DAF800303A6A1B78D35C93
:107CE0001B0702D4B8F1000F8FD1C7F81CB02B4688
:107CF000D7F824B0D7F830E0D7F83CC07A6CFFF75B
:107D0000BFBB16F8011C5246B86C013EFEF7A6FF39
:107D1000FFF75CBBBA4B0326BB620A237B63FFF70A
:107D20007DB923077FF457A97178682900F0A081F5
:107D300044F004045E46FFF7EBB814F08F037FF4C1
:107D40004AA9B96B002900F03782717844F08004A9
:107D50005E46FFF7DDB8E10600F1C680FA6A52F828
:107D6000043BFA62220700F1BD80660740F192826F
:107D7000A3F80090C7F84CB0FFF741B844F408747A
:107D80000CE725437FF427A9717810245E46FFF79E
:107D9000BFB8594607F1700000F066FC44F040049B
:107DA0000126F8641AE521077FF415A971786C297A
:107DB00000F0588144F001045E46FFF7A9B8C7F807
:107DC0004CB0FFF738B88F4B0326C7F84CB0BB62F6
:107DD00000237B6302E5DAF8003007F170021978BE
:107DE000515C00293FF4F7A80133012DCAF8003097
:107DF000DAF8043003F1FF33CAF804303FF401AB82
:107E0000BC6C904614E0DAF800301A78013318F8A8
:107E10000220002A3FF4F5AA0136CAF80030DAF849
:107E20000430B54203F1FF33CAF804303FF4E9AA45
:107E3000002BE8DC51462046FEF74EFF0028E2D03A
:107E4000B144FEF7DCBF002307F154027B62904689
:107E5000FB623B62FFF758BB4FF0000C07F1540385
:107E6000E646E346FFF701BB831C0DD0D8F800308F
:107E70005D1C7FF483ABFFF799BBD9F80030042B6E
:107E80007FF49EABFFF79FBBDAF80430002B3FF77F
:107E900041AB5146B86CFEF71FFF00283FF4B3AB6F
:107EA000D946FE61D7F818B0002C3FF4B3ABFEF70B
:107EB000EBBFBC683246396A2046C7F81880D04606
:107EC000AA467D6800F09AFCBB6928F42078013D41
:107ED000044699463B6BBB61FFF793B94FF0000C2A
:107EE000FFF7D0B883F80090C7F84CB0FEF787BF13
:107EF0003B6CC246002B3EF4CBAFFFF767B84FF0A8
:107F0000FF333B64386C07F53577BD46BDE8F08F2D
:107F1000A61B4B46D7F82C903FF45DA8711C00229D
:107F20008B42227003D9BBF1000F40F0D680B144E0
:107F30003B6C01333B643B6BFB62FEF760BF7B6CC9
:107F4000022B40F26C82032B3FF47DA97B6C1E1F39
:107F5000F6B2F5437E6426462544BC6C16F8011D36
:107F600052462046FEF77AFEAE42F7D1344609F17A
:107F7000FF397E6CA9EB0609FFF765B9FB6A18F0BB
:107F8000020FD3F800B000F09380CBE90056FFF762
:107F90008BB95246B86CFEF761FEA9F10209A51E25
:107FA00014F8021CFFF761B94FF6F67188453EF6EA
:107FB00073AF08F10808BB6B4FEA88011868FBF73C
:107FC0006DFC00283EF468AFBB6BA3F8048018601A
:107FD00041E5012191E54FF6F67398453EF65CAF19
:107FE00008F10808BB6B4FEA88011868FBF756FCDC
:107FF00000283EF451AFBB6BA3F804801860B1E4D5
:10800000596C0010799900104FF6F671FA63786494
:10801000884500F2EC8108F10808BB6B4FEA880143
:108020001868FBF73BFC002800F0E181BB6BFA6BA2
:10803000A3F8048018607B6CFFF70EBA4FF6F67356
:108040009A4200F2D48102F10806BB6BB1001868B5
:10805000FBF724FC002800F0CA81BB6B9E801860EF
:10806000FFF748BAB17844F002040236FEF750BF79
:10807000B17844F008040236FEF74ABF620779D4AB
:1080800014F0010240F01081A30740F10D819F4BD5
:10809000B96AB86C99427B6B594600F0CE8101F009
:1080A0003BFD0B46FA6A1168C1E90003FFF7A2B96C
:1080B0000B46FAF769FC002870D128463146FAF7DA
:1080C0000DFCCBF80000FFF7EFB8286001F018FEB8
:1080D000002840F0F280B144D8E5FC6B2068FBF743
:1080E000DDFB00283FF423AF206020E7191DDBF8FB
:1080F0000000FBF7D3FB00283FF4D0A9CBF8000029
:10810000FFF7CCB9DAF80030DFF808821A7818F8EF
:10811000022014073EF573AE0133012DCAF800307A
:10812000DAF8043003F1FF33CAF8043000F0898133
:108130000124BE6C13E0DAF800301A78013318F825
:108140000220100713D40134CAF80030DAF80430E2
:10815000A54203F1FF33CAF8043000F0AB80002BD6
:10816000E9DC51463046FEF7B7FD0028E3D0A144D4
:10817000FEF745BEFB6A1B681880FFF73BB95C45FC
:108180005E467EF628AFBD6C14F8011D52462846A7
:10819000FEF764FDB442F7D1FEF71DBF5C4800F066
:1081A00077FBCBF80000FFF77FB800268EE57E6CEA
:1081B000A34623467C6457E482B0CDE9023302AB88
:1081C000BB63C2E53C690A230022B86C611C01F064
:1081D000D3FB7B69C21AB5E45B4694469646934648
:1081E000FE62FFF742B93B6BD7F820807B62FB62EF
:1081F0003B62FFF789B9FC6BFB63FFF7BABBD9465B
:10820000FE61D7F818B02646002C3FF403AA07F504
:10821000B873BD6C1C19013E524614F8011D284666
:10822000FEF71CFD002EF6D1FFF7F4B9012328F468
:10823000F068FB6300233B63FEF7E0BF012328F4F3
:10824000F0687B6400233B63FEF7D8BF5146B86CEF
:108250003B63FEF741FD3B6B00283FF440AC46E436
:10826000C7F84CB0FEF7EBBE5146B86CFEF734FDD4
:1082700000283FF430ADC7F81CB02B46D7F824B027
:10828000D7F830E0D7F83CC07A6C002E7EF4FCAD15
:10829000FFF7F6B8E5070AD4A40708D54FEAE97254
:1082A000C3F800905A601FE6FB6AFFF7A1B8C3F855
:1082B000009019E6A944FEF7A2BDC7F81CB02B46F2
:1082C000D7F824B0D7F830E0D7F83CC07A6C002E4D
:1082D0003FF4D6A807F5B871C7F84490FD63F0469F
:1082E0008C19E146BD6C3A63013E524614F8011DFB
:1082F0002846FEF7B3FC002EF6D1CC46FB6BC646F3
:10830000D7F844903A6BFFF7BBB800BF596C001028
:108310000CB5001005BA0010012D04F0100238BF92
:10832000012514F001037A6400F09380FB6A002AAF
:1083300040F0DE8053F804BB24063B6300F1028169
:10834000D846D7F844B05B46DC46C7F83CB00026B8
:1083500064469B4600F092FAB0423EF495ADDAE9ED
:108360000032013A13F8011BCAF8042007F5B8726D
:10837000CAF80030731C915507F16806FA69032AA0
:1083800002D13268042A06D0082200213046FB625E
:10839000FDF7E0FFFB6A009607F5B8724146B86C3E
:1083A000FB6201F083FC0246F861501C3EF46CADA8
:1083B000FB6A002A40F00A8199447B6C013D002B46
:1083C00040F01281C8F80030A8EB0406BBEBA60F02
:1083D00000F23D81FB6B002B00F0398120464FEA13
:1083E000CB01FBF75BFA0446002840F02A814FF0EE
:1083F000FF333B64FEF7EFBD5C455E467EF6EBADBA
:10840000BD6C14F8011D52462846FEF727FCB44205
:10841000F7D1FEF7E0BDD7F824B0FFF79CB95C4573
:108420007EF6D9AD5D4614F8011D5246B86CFEF7D4
:1084300015FCAC42F7D1FEF7CEBD01F035FC0B4682
:1084400030E609F10109FEF7DABCD7F84CB0FFF7C6
:10845000D9B97A6C002A51D1D7F82C80240658F863
:10846000046B62D5002E3EF4B6AD2846FBF7FAF950
:10847000024600283EF40CADBB6B3060B3F806B08A
:108480009C88A345C0F093804FF6F67378649C42B5
:108490003EF602AD0834BB6BA1001868FBF7FEF98D
:1084A00000283EF4F9ACBB6B7A6C9C801860B96B09
:1084B0000BF1010340F82B60CB801146CDF800A0F2
:1084C0002B460122B86CFEF723FC0446002870D02E
:1084D000854205D901463068FBF7E0F900B130600C
:1084E0003B6CA144C7F82C8001333B64FEF787BC8A
:1084F0003B6300239C469B46984626E71C46DAE9E8
:1085000000239D4202EB030147DDCAF800105146EB
:10851000B86C1C44ED1AFEF7DFFB0028EFD0002CEE
:108520003EF4B2ACA144FEF76ABCCDF800A02B46E5
:1085300031460122B86CFEF7EBFB04460028CFD190
:10854000FEF7A2BCBBF1000F3EF445AD8020FBF767
:1085500089F9804600283FF44AAFBB6BCBF8000096
:10856000DE889C88A6422FD34FF6F6739C423FF6D6
:108570003EAF0834BB6BA1001868FBF78FF90028E9
:108580003FF435AFBB6B9C801860BB6BC44640F8B2
:1085900026B00136DE802023D7E65B1B2A442C441C
:1085A000CAF80430A144CAF80020FEF728BC1868B5
:1085B0007DE73B6C002B3EF46FACBAF80C305B06E9
:1085C0007EF50DADFEF768BC1868DEE7FA69911C10
:1085D00023D0032A994402D13368042B00D0013DF3
:1085E0007B6C002B3FF4F0AEDAF804300026002B51
:1085F00019DD002D7FF4AEAE5B46A446D7F83CB043
:10860000A8EB0C01B3EBA10F02D9BBF1000F21D1F4
:108610007B6C002B7FF48FAC8AE4DAF804201E46D2
:10862000002A3FF797AE5146B86CFEF755FB00287D
:10863000DFD05B46A446D7F83CB0002EE0D0FEF772
:1086400023BCFB6B00EB06084FEA4B0B186008F1EC
:108650000408C9E7DBF80000FBF720F90028D7D0B1
:10866000CBF80000D4E700BF70B50C7884465E2CD0
:1086700024D00023481C9E4600220CF5807163F331
:10868000070263F30F2263F3174263F31F6263462B
:1086900043F8042B8B42FBD174B18EF00101451CD1
:1086A0000CF8041015F8013C2D2B0ED05D2B0AD0D0
:1086B0001BB11C462846F2E7013870BD0123881C17
:1086C0004C789E46D8E7284670BD90F801E0BEF190
:1086D0005D0F15D0744513DC661C02300CEB0602EE
:1086E00002F8011BA2EB0C03013B9E45F8DCAEEB4C
:1086F00004030235013B7445A8BF00239C19D1E750
:108700002D242846CBE700BF2DE9F0410C46096B2C
:1087100004F14003994214D0666B77003A46FDF7A6
:10872000B3FB054630B300EB06080146324640462F
:10873000FEF702F8C4F80080C4E90C570020BDE839
:10874000F0814FF48061FDF7C1F898B194F84220B0
:108750004FF48061206300F2FD33616380F8FF23F2
:1087600094F8412080F8FE2394F8402080F8FD23FF
:108770002360E3E74FF0FF30E1E700BFCAB3844670
:108780000B4630B504460843800719D09CF800001A
:108790000C78A04212D150B3012A28D0E64603E05B
:1087A0001CEB030F23D010B31EF8010F11F8014F7B
:1087B000A2EB0E03A04203F1FF33F1D0001B30BD4A
:1087C000032A07D8E2E7043A11D01EF0803F0ED109
:1087D000032A10D92068194653F8045BA446A0F177
:1087E000013E0434A8422EEA000EECD0CEE7002071
:1087F00030BD10467047A4461946C7E740EA01035A
:108800009B0710B4044601D1032A1CD801F1FF3C98
:1088100007E01CF8011F501E03F8011B41B102467E
:108820001C462346002AF4D120465DF8044B7047CD
:10883000F8B1A01803F8011B8342FBD1002CF3D13F
:108840005DF8044B70478C4604E0043A44F8040B8E
:10885000032A0CD9DCF8000061460CF1040CA0F1ED
:10886000013323EA000313F0803FEED0CEE76146E8
:10887000CCE71846002CD7D1E2E700BF014B93F8B4
:10888000280170470010002000487047F0100020B9
:10889000004870470000C07F82B049B15AB16BB147
:1088A00013780B601278101E18BF012002B07047B9
:1088B00001A9002AF3D1104602B070476FF0010001
:1088C000F4E700BF000000002DE9F04F88469FB09C
:1088D00000218346079200221A910021CDE904125B
:1088E00042461746199212F8019BB9F12D0F5FD835
:1088F00001A151F829F000BF458A0010B18900108C
:10890000B1890010B1890010B1890010B18900103F
:10891000B1890010B1890010B1890010E3880010FE
:10892000E3880010E3880010E3880010E38800105B
:10893000B1890010B1890010B1890010B18900100F
:10894000B1890010B1890010B1890010B1890010FF
:10895000B1890010B1890010B1890010B1890010EF
:10896000B1890010B1890010B1890010B1890010DF
:10897000B1890010B1890010E3880010B18900109E
:10898000B1890010B1890010B1890010B1890010BF
:10899000B1890010B1890010B1890010B1890010AF
:1089A000B1890010B38F0010B1890010CB8F001077
:1089B00000220892B9F1300F7ED000230A93A9F16A
:1089C0003003092B00F23484002538462E462C460D
:1089D0000130082C05EB850204F1010406EB860149
:1089E000199090F80090CCBF03EB420503EB4106D1
:1089F000A9F13003092BEBD90122A349FFF7BEFEF1
:108A000058BB199BA24609905A1C19925B78A3F196
:108A10003002092A09D8013091461999002A40F0FC
:108A2000D4844B1C19934B78F1E74FF0010923F0E4
:108A30002002452A40F0B78244EA00030A9A134311
:108A400040F05082079B002600270BB1C3F800803E
:108A5000304639461FB0BDE8F08F29F020020020D3
:108A60004B46A246452A8146099000F03B820E9073
:108A7000002C35D10A9A024340F08382B9F1000FED
:108A8000E0D1692B00F0CC8400F31F83492B00F068
:108A9000C7844E2BD6D17D4919A801F047FD002887
:108AA000D0D0199B1B78282B00F08385784801F0E3
:108AB00017FA06460F4666E27A7802F0DF02582A75
:108AC00000F03F840137199797F80090B9F1300F03
:108AD000F8D0B9F1000F00F0548201230A936EE739
:108AE000099ABAF1000F08BFA2460E9B102C30461F
:108AF000A046A3EB0203A8BF4FF010080D93F9F7AF
:108B00000DFF092C02460B46CDE9042317DD614B0E
:108B100003EBC80353E91223F9F76CFE02460B4638
:108B20002846CDE90423F9F7F9FE02460B46DDE9B4
:108B30000401F9F737FE0F2CCDE9040124DC0D9B6D
:108B4000002B00F0B5830D9B40F3AD82162B40F354
:108B50008484C4F125030D9A934215DBC4F10F04FC
:108B60004C4D05EBC401DDE90423D1E90001F9F71F
:108B700041FE0D9B1C1B05EBC405D5E90023F9F74D
:108B800039FE06460F46FEE1A4EB08030D9A9D1838
:108B9000002D40F32B8215F00F000AD03D4901EB68
:108BA000C001DDE90423D1E90001F9F723FECDE995
:108BB000040135F00F034BD0B3F59A7F00F35A84CC
:108BC000102B4FEA231540F3B385DFF8DCE04FF0BC
:108BD000000C0A96F046E1467646DDE9042315F0DE
:108BE000010F1046194607D0D8E90023F9F702FE15
:108BF0004FF0010C02460B466D1009F1010908F116
:108C00000808012DEBD1B6460A9EBCF1000F01D039
:108C1000CDE90423059B0EEBC901A3F15473059321
:108C2000DDE90423D1E90001F9F7E4FD1A4B0A4616
:108C30000B40CDE9040119498B4200F21B8418490D
:108C40008B4240F2C9844FF0FF32164BCDE904232A
:108C500000230C932346524639465846009601F0AD
:108C6000E1FD1590002800F005840E9A099B9B1ADF
:108C70000D9A002A22EAE272A8BF002314920E93F2
:108C800000239A460993EBE0F0B7001044B80010B7
:108C90000CB5001088F100100000F07F0000A07CEF
:108CA0000000907CFFFFEF7F60F10010D21A1F2AB6
:108CB000A4EB020400F37C820123002593401E46AE
:108CC000A0444C440C9BA14598444B46A8BF234666
:108CD0004345A8BF4346002B04DDE41AA8EB030874
:108CE000A9EB03090E9B002B00F30382002C00F379
:108CF00019820D9B002B00F34C82B8F1000F00F39A
:108D00003C82B9F1000F08DD51464A46584601F051
:108D10006FFF8246002800F039823A461A99584679
:108D200001F0FCFF0990002800F03082099A00232E
:108D3000D168D3600F91514601F0CEFF0028C0F2F8
:108D40007984DDF8149000F0E7835146099802F029
:108D50008DF900224FF0804304460D46F9F74CFE92
:108D6000002800F0B6810F9B002B40F02882049B66
:108D7000002B40F01283C9F31303002B40F09B82B9
:108D80000022954B20462946F9F722FE002840F0A4
:108D9000BA830022914B20462946F9F72BFD0A465B
:108DA0000146109002F10043CDE912121193DFF851
:108DB00034828B4B09EA08089845DDE9104500F03C
:108DC0000A820C9B1BB3B8F1D46F20D880A3D3E9DF
:108DD0000023DDE91201F9F70FFEA0B1DDE9120170
:108DE000F9F7C0FD012838BF0120F9F797FD0F9B67
:108DF000CDE91201002B40F0E38201F1004316900F
:108E00001793DDE9164505F1D663A3EB0805DDE907
:108E10000A0102F043F802460B4620462946F9F7BC
:108E2000E9FCDDE90A23F9F7BDFC0C46CDE90401B4
:108E30006C4B2340434503D10C9B002B00F05C821C
:108E40001A99584601F092FC3946584601F08EFCBA
:108E50005146584601F08AFC0999584601F086FCB3
:108E6000159C5846616801F05BFC0746002800F03D
:108E70008D81226904F10C010C3002329200FDF761
:108E80005BFC1CAB584601931BAB9DED047B009330
:108E900053EC172B8DED0A7B02F088F81A9000280E
:108EA00000F049810121584601F068FD8246002802
:108EB00000F06C811B9B002BC0F259810E9ADDF8EB
:108EC000508003EB02090C9A1C9C9B1A464A2344CF
:108ED000C4F13604013B9342FFF6E8AE01230025BE
:108EE0001E46EDE6DDF8648008F10103199398F859
:108EF00001302B2B00F099812D2B57D14FF0010E13
:108F000008F10203199398F80230A3F1300CBCF178
:108F1000090F00F24881199A302B0C920BD10132C3
:108F200019921378302BFAD0A3F131010C92082951
:108F300039D8A3F1300C0C9B591C19915B78A3F123
:108F40003002092A00F2818201310CEB8C0C19915C
:108F500003EB4C0C0B78ACF1300CA3F13002092A76
:108F6000F2D90C9A891A082940F36F8244F61F62DD
:108F70000E92BEF1000F3FF47BAD0E9A52420E925C
:108F800076E500260027079A0AB1199B1360089B13
:108F9000002B3FF45DAD07F1004330461F463946D4
:108FA0001FB0BDE8F08F00220E9261E54FF0000E79
:108FB000ABE7002208927A1C199297F80190B9F158
:108FC000000F3FF43FAD1746F4E401220892F2E7A8
:108FD0000000C0FFFFFFDF410000F03F0000E03F66
:108FE0000000E07F0000F07F02FCFFFF3FF430AEA6
:108FF0006D4215F00F020AD0B74B03EBC203DDE957
:109000000401D3E90023F9F71BFCCDE904012D117C
:109010003FF41EAE1F2D40DC15F01003DFF8D482A4
:109020004FF0000C18BF6A230C93DDE9042315F000
:10903000010F1046194607D0D8E90023F9F7DAFBEB
:109040004FF0010C02460B466D1008F10808EED1F6
:10905000BCF1000F01D0CDE904230C9BA3B1DDE9E5
:109060000401C1F30A52C2F16B03002B0ADD1F2B6E
:1090700040F382830020342B049040F3B8834FF0F8
:109080005C7305936A230C9300220023DDE904013D
:10909000F9F78CFC00283FF4DDAD222300260027E1
:1090A000CBF800306FE71633FFF66EAD099B0E9AD2
:1090B0009A1A894B03EBC203DDE90401D3E90023CB
:1090C000F9F7BEFB06460F465DE76E2B3FF4E3ACB7
:1090D000B8E4824B204629460022F9F78BFB0F9B10
:1090E000CDE91201002B71D101F1004310901193D1
:1090F0005DE651461A46584601F020FD824600289A
:1091000044D001461A9A584601F066FC00283DD02A
:109110000F9058461A9901F029FB0F9B002C1A93C7
:109120007FF7E7AD22461A99584601F061FD1A9083
:1091300000287FF4DEADB946054622230026684F9D
:10914000CBF800302946584601F010FB49465846F6
:1091500001F00CFB5146584601F008FB15995846A2
:1091600001F004FB0999584601F000FB0BE7149A43
:10917000DDF83890A2EB0308A5E63946424658468A
:1091800001F036FD074600287FF4BBADB9461A9DB5
:10919000D3E73946149A584601F0D0FC0746002818
:1091A0007FF4ABADF2E70022CDF864800E925FE46D
:1091B0004C4AD31A012202FA03F5164680E59FEDC8
:1091C000427B8DED107B8DED127BF0E59DED127BEA
:1091D0008DED107BEBE5A9F15473DFF80491059355
:1091E000DDE904452046294601F058FEDDE910235B
:1091F000F9F700FB2B462246F9F7D4FA3A4B01EA7D
:1092000009099945CDE9040140F2D68003F1547370
:10921000DDE90A01994202D106460136B6D04FF087
:10922000FF33324CCDE904340AE64FF0000E67E616
:1092300001222F493846FFF7A1FA824658B14FF074
:10924000000A4B465546564650465446D146CDF840
:1092500024A0FFF7ECBB19994B1C19934B78302BCA
:1092600040F04F818A1C1046199201320378302B4E
:10927000F9D0401A0138A3F13102082A0FD8199FFA
:109280000026A3F130090124431C394635460993D1
:1092900006EB8606002009EB4606FFF7C2BB00225C
:1092A0004FF001091646144615460992FFF7BFBB59
:1092B000DDE9046767E69FED067B8DED107B9FED92
:1092C000027B8DED127B72E5000000000000F03F94
:1092D000000000000000F0BF88F100100000E03F37
:1092E0000000F07FE2FBFFFFFFFF9F7CFFFFEF7FAF
:1092F000F0B7001058BB0010DDE912562846314681
:10930000FAF760FAFAF758F90B4602463146284652
:10931000F9F75CFA049D0F9EC4F3130C04462E4328
:109320000D4656EA0C0326D1C0A3D3E90023F9F772
:109330004FFB00283FF484ADB946DDE904671A9D70
:1093400000E7029319A9089B5846AF4A01931AAB4C
:1093500000931BAB00F01CFE10F00F0504463FF419
:1093600010AE062D40F08A807B1C002200260027CC
:109370000892199307E69CA3D3E90023F9F728FB89
:109380000028D9D12046294699A3D3E90023F9F72B
:109390005BFB00283FF454ADCEE7049B012B8AD140
:1093A000B9F1000F87D1B9461A9C22232546002621
:1093B0000027CBF80030C5E601F15474059437E579
:1093C0009DED127B8DED167B1BE5012840F33B8262
:1093D00004EB000E0C900EF1FF3C02E046006445E9
:1093E0000BD0082C06EB860004F10104F6DD05EB3A
:1093F0008503102CD8BF5D00F1E70C987446099BDB
:10940000BCF1080F034409937FF742AF102C4FF0D3
:109410000000DCBF05EB850502EB4505FFF701BB4E
:109420007A4919A801F082F800283FF40BAB199B88
:1094300019A87749013B199301F078F810B9199BE5
:10944000013319930026734F9DE544F61F6294453E
:10945000A8BF9446CDF838C08BE50D986E4901EB56
:10946000C001DDE90423D1E90001F9F7C3F906469B
:109470000F4688E52223CBF80030E3E71A9A3AB189
:1094800035211CA801F020FE58461A9901F06EF90A
:10949000013D1B9B042D00F2D981DFE805F0032C70
:1094A000291E030003F233421C9B04931D9B23F4EB
:1094B000801343EA02530593E20502D543F00043CB
:1094C0000593544A1A40DDE90467002A7FF45BAD36
:1094D000FCF7DEFF2223036055E54FF0FF326FF00B
:1094E0000043CDE90423E3057FF5E2AE059BE5E704
:1094F000484B0593F7E7DDE91C121D9BCDE90412EB
:10950000DAE75046B7E69FED3C7B8DED107B9FED93
:109510003C7B8DED127B4AE44B460F98B646B9462C
:10952000AC463E49C3F31302DDE90A67002800F0A8
:10953000B5808A4200F00A81A5BB049A1EEA020F98
:1095400033D030463946049301F0A8FC0C9B002B25
:1095500000F02581049BC3F30A53C3F16B0CBCF1EB
:10956000000F40F365812E4C002204EB0C53F9F7F9
:1095700041F902460B4630463946F9F713F90646DB
:109580000F4630463946274B0022F9F733F9214B75
:1095900006460F460B40002B7FF4D1AE2223CBF8BA
:1095A0000030CCE61CEA030FCBD10C9B002BE8D19A
:1095B000C5E619A81CAA1C4900F0D2FF05287FF4B3
:1095C00075AA1D9B43F0FF4343F4E00305931C9BE6
:1095D0000493DDE90467D6E402F154730593FFF7C1
:1095E00037BB00BFAFF300809535A094FFFFDF3F8E
:1095F00035E5AF350000E03F000000000000E0BFAF
:10960000000000000000E03F40BB001038B8001030
:109610003CB800100000F07F88F10010FFFF0F0041
:109620000000F03F000050392CBB00109535A0948D
:10963000FFFFCF3F0F9BB946DDE90401DDE90A6773
:109640000343B2D1C1F31303002BAED121F0004488
:10965000240D2405B4F1D66F2546A6D9099A53697D
:1096600013B91369012BA0DD09990122584601F0B5
:10967000BFFA5146099001F02FFB002895DD0C9BA5
:10968000D3B1A5F580136FEA13536FEA0353059323
:109690004FF0FF330493DDE9046772E7D2B9DDE9E7
:1096A00004452246002C49D10C9A002A40F08E80B5
:1096B00025F00044240D2405A4F580141A9D6FEABA
:1096C00014536FEA035305934FF0FF330493DDE91E
:1096D000046737E5ADBB049A1EEA020F3FF465AF9D
:1096E00030463946049301F0D9FB0C9B002B00F067
:1096F0008680049BC3F30A53C3F16B0CBCF1000FCB
:1097000040F39E80524C002204EB0C53F9F772F8A0
:1097100002460B4630463946F9F758F80022002336
:1097200006460F46F9F742F900283FF42AAF3BE618
:109730004FF00009DFF824E1FFF76CBABCF1000F2D
:10974000CAD01CEA030F3FF430AFC9E70C9A049C5F
:10975000D2B1404A1A40B2F1D46F15D8100D4FF073
:10976000FF31C0F16B0081408C4227D0002D62D0C8
:109770001D423FF406AFE4E64FF0FF3202FA03F376
:10978000049A1A4004927DE4621C12D0BCF1000FCE
:109790007FF408AF14EA0E0F3FF407AFD1E602469C
:1097A0000B4630463946F8F7FDFF1A9D06460F4630
:1097B000C8E4294A934234D001321A4002F580139A
:1097C000059300230493DDE90467EEE6214D1D4077
:1097D000B5F1D66F3FF655AFB5F15C7F3FF6D1AE30
:1097E00022231A9D00260027CBF80030AAE4C2F1FC
:1097F0004B024FF0FF3393400B40059342E4024687
:109800000B4630463946F8F7E1FF1A9C0022002348
:1098100006460F462546F9F7C9F800283FF492ACF2
:10982000C3E522231A9D00260A4FCBF8003089E4B5
:1098300002460B469FE614EA0E0F3FF4A2AE80E606
:1098400002460B4666E7A4460134D8E5002333E61A
:109850000000F03F0000F07FFFFFEF7F60F100109D
:10986000014BFFF731B800BF001000202DE9F04F89
:1098700082468E463F4875461EF801BB10F80B40E5
:1098800014F00804F7D1BBF12D0F5BD0BBF12B0F07
:109890006FF0004904BF9EF800B005F1020E33F0EE
:1098A000100010D1BBF1300F04D0002B5ED10A2381
:1098B0001F4609E09EF8000000F0DF0058284ED057
:1098C000002B53D108231F460025B9FBF7F6284685
:1098D00007FB16980EE0ABF1370C63451DDD002D3C
:1098E00004DB864202D321D1E0451FDA4FF0FF3579
:1098F0001EF801BBABF1300CBCF1090FEDD9ABF197
:10990000410CBCF1190FE6D9ABF1610CBCF1190F98
:1099100003D8ABF1570C6345E1DC6B1C0AD004B1F2
:1099200040420AB1CDB91160BDE8F08F07FB00C01D
:109930000125DDE72223CAF800305AB10EF1FF31CC
:109940004846F0E79EF800B04FF0004905F1020EDE
:109950000124A4E74846BDE8F08F8146EEE71023D6
:109960009EF801B00EF1020E1F46ADE710231F4610
:10997000AAE700BF05BA0010242B03D8012B01D0A1
:10998000FFF774BF10B5FCF783FD162303600020BA
:1099900010BD00BF034649B1FF2A02D801200A705A
:1099A00070478A224FF0FF301A60704708467047B0
:1099B0002DE9F04F924685B089461E460D46554A20
:1099C0000390294615F8014B135D13F00803F8D1F5
:1099D0002D2C7CD02B2C4ED04FF0FF3102936FF00A
:1099E0000043CDE9001336F0100851D037464FEA56
:1099F000E6783A464346DDE9000101F0F9FB002331
:109A000083468E4618461946A44613E0ACF1370447
:109A1000A6421FDD002B09DB83457EEB010305D346
:109A20008E4508BF83453BD1A24239DA4FF0FF3360
:109A300015F801CBACF13004092CE9D9ACF14104A3
:109A4000192CE3D9ACF16104192C03D8ACF15704FB
:109A5000A642DFDC5A1C2FD0029A12B1404261EBC1
:109A60004101BAF1000F03D0002B48D1CAF8009091
:109A700005B0BDE8F08F4FF0FF30029336F01008CC
:109A80006FF000432C7801F10205CDE90003ADD160
:109A9000302C25D0002E3AD10A27B0463E46A8E702
:109AA00000FB08F307FB0133A0FB07010B44201860
:109AB00043EBE4710123BBE72223039A1360BAF15D
:109AC000000F17D005F1FF39DDE90001CEE74FF0B7
:109AD0000047009301232C788D1CCDE9017382E7A8
:109AE0002B7803F0DF03582B0CD086B90827B0463B
:109AF0003E467EE7DDE9000105B0BDE8F08FCDE927
:109B00000001DFE710276C7802353E4671E7102729
:109B10003E466EE705BA0010FFF74ABF2DE9F04F49
:109B200085B08B461E460D4601925D4A039029463C
:109B300015F8014B135D13F00803F8D12D2C00F03C
:109B400082802B2C51D0029336F0100A54D04FEA69
:109B5000E67A32464FF0FF304FF0FF315346B146C0
:109B600001F046FB32460746884653464FF0FF3029
:109B70004FF0FF3101F03CFB9446002210461146A5
:109B800013E0A4F137039E421FDD002A09DB874260
:109B900078EB010205D3414508BFB8423BD163458C
:109BA00039DD4FF0FF3215F8014BA4F13003092BDA
:109BB000E9D9A4F14103192BE3D9A4F16103192BCD
:109BC00003D8A4F157039E42DFDC531C30D0029B24
:109BD00013B1404261EB4101019B1BB182BB019B70
:109BE000C3F800B005B0BDE8F08F36F0100A2C784D
:109BF000029301F10205AAD1302C29D0002E44D1C4
:109C00004FF00A09B2464FF0050C4FF09937DFF8D4
:109C100094804E46B1E709FB01F100FB0A11A9FB54
:109C20000002114418184FF0010241EBE371BAE74A
:109C30002223039910460B601146019B002BD1D0C3
:109C400005F1FF3BCBE701232C788D1C02937BE7CA
:109C50002B7803F0DF03582B0BD0B6B94FF008096F
:109C6000B2464FF0070C4FF0FF376FF060484E469A
:109C700083E74FF010096C784FF00F0C02354FF06E
:109C8000FF376FF070484E4677E74FF010094FF0FE
:109C90000F0C4FF0FF376FF070484E466DE700BF76
:109CA00005BA001099999919FFF738BF70B582B0BD
:109CB0000446069D55B11048D0F8E4606AB12046CC
:109CC0000095B047431C10D002B070BD00F1F40500
:109CD0000948D0F8E460002AF1D10123114620465A
:109CE000064A0095B047431CEED100228A232A6021
:109CF000236002B070BD00BF001000200CB5001042
:109D0000002100F001B800BF10B500F0B7F804461C
:109D100001F036FAA0F11A03DBB2022B01D80120C0
:109D200010BDA4F1090004288CBF0020012010BD43
:109D30000229C0F307235FFA80FC25D0032903D052
:109D400083F080038CF0800C03F15002D2B21F2A02
:109D50000BD903F13002D2B2242A3BD84FF2A642EB
:109D600090422CD94FF0FF3070474CF6D37290429E
:109D7000F8D8B03BACF1A10C384AC3EBC3130CEBE1
:109D8000430332F813007047BCF19E0F11D90CF158
:109D9000230C80225FFA8CFC9F2B94BF703B5033C6
:109DA00002EB4302D3B203F15002D2B21F2AD0D841
:109DB000DBE7ACF17E0C7F225FFA8CFCECE7D03B5A
:109DC000ACF1A10C264AC3EBC3130CEB430332F8EE
:109DD00013007047A13B072BC4D8DFE803F0382EEF
:109DE000241D17120D04BCF1C00FBBD81D4AACF1E5
:109DF000A10332F813007047BCF1F10FB2D81A4A30
:109E00001CE0BCF1D80FADD8184A17E0BCF1F60F32
:109E1000A8D80CF540507047BCF1F30FA2D842F619
:109E2000A07060447047124B634413F8A13C002BB0
:109E300098D04FF66060604470470E4AACF1A103C1
:109E400032F81300002808BF4FF0FF3070470A4A6D
:109E5000ACF1A10332F81300704700BFFCD500102D
:109E600080BB001028ED001068ED00100CEE001013
:109E70007CEE0010D8EE001094EF001038B50546C7
:109E8000B9B101F5957412492046FCF719FB28B9C0
:109E900028460121BDE83840FFF74ABF0D4920465A
:109EA000FCF70EFB38B928460221BDE83840FFF721
:109EB0003FBF094CE7E709492046FCF701FB28B9F9
:109EC00028460321BDE83840FFF732BF284638BD99
:109ED00048B800104CB800102A11002054B80010E7
:109EE00000200149704700BF0000F87F2DE9F041D4
:109EF0000469B4EB611F05DC0023036100234361A7
:109F0000BDE8F08100F114054E1111F01F0C05EBB6
:109F1000840E05EB860321D0043355F82610CCF1CE
:109F200020089E4521FA0CF12DD92F461A6802FA15
:109F300008F20A4347F8042B53F8041B9E4521FA04
:109F40000CF1F3D8A31B9B00053B9B08013305EBE9
:109F5000830445F8231071B104340CE09E45CBD93D
:109F600000F1100253F8041B9E4542F8041FF9D873
:109F7000A41B05EB8404631BAC424FEAA3030361FB
:109F8000BCD0BDE8F08141610029B5D02C46E3E7A3
:109F90002DE9F04F8A4685B0096803938B78302B02
:109FA000CDE9002040F0EE81CA1C1378144601323E
:109FB000302BFAD0A4EB0109A9F10209DFF81083D4
:109FC00018F80330002B00F0D3802378002718F80E
:109FD00003303D46002B00F06D81264616F8013F08
:109FE00018F80330002BF9D10122B8493046FEF7AA
:109FF000C5FB8346002843D03278002D00F0A381B2
:10A00000AB1B4FEA830B02F0DF023546502A43D0E8
:10A01000CAF80060002F54D12A1B3946013A072A9A
:10A0200003DD52100131072AFBDC019800F078FBB8
:10A030008246002800F06A8200F11406A5420296CA
:10A0400040F2CC810027B9460CE03A4604372B7821
:10A05000AC4218F8033003F00F0303FA02F349EAA5
:10A06000030940D015F8013D2E2B01D1AC4231D966
:10A07000202FEAD1002246F8049B04279146E6E708
:10A08000002D00F070813278AB1B354602F0DF0204
:10A090004FEA830B502ABBD16A782B2A00F05181FA
:10A0A0002D2A40F0C5800120AA78AE1C18F80210B5
:10A0B0004A1E182A40F2C4802E46CAF80060002FBB
:10A0C000AAD0B9F1000F0CBF06250025284605B01F
:10A0D000BDE8F08F01227D492846FEF74FFB00289E
:10A0E000C6D1AC42BED1029B484646F8049BF61A44
:10A0F000B610CAF81060760100F0ECFB009B361A2F
:10A100001C68A64277DCC0F220810027009B9A6879
:10A110005A45C0F25881009B5A685A454BDDA2EB64
:10A120000B0B5C4500F3A780DB68022B00F0F98085
:10A13000032B00F06A81012B40F0F7805C4540F072
:10A14000F480012C08D0611E504600F0EBFF00287F
:10A1500000F0EB80009B5A680399012362250A6096
:10A16000029ACAF8103013600E9BC3F800A0ADE746
:10A17000012256492046FEF701FB0746002840F021
:10A180009B806378651C18F80320002A00F09680F5
:10A19000302B2C4640F0448114F8013F302BFBD08B
:10A1A00018F803304FF00109B3FA83F77F09002B49
:10A1B0007FF413AF7EE001259FB1009BDA68022A8D
:10A1C00000F08880032A00F08980012A07D1B907AE
:10A1D00005D5029B1A681743FA0700F1838045F002
:10A1E00010050E9B2846C3F800A0039BC3F800B0DF
:10A1F00005B0BDE8F08F361B5046314600F092FFA7
:10A20000074678B1711E029B01274A1153F82200BC
:10A2100001F01F0207FA02F2024203D0B94200F332
:10A22000E780022731465046B344FFF75FFE6DE7F3
:10A2300018F802106E1C00204A1E182A3FF63CAF88
:10A2400072781039013618F8022002F1FF3CBCF197
:10A25000180F0CD801EB810116F8013F02EB410207
:10A26000A2F1100118F80320531E182BF2D900B1E7
:10A2700049428B44CCE60BF1FF36002F40F0AC8016
:10A28000002E40F0AF807311029A06F01F06594667
:10A2900052F8232001235046A4EB0B04B3400225BF
:10A2A000134218BF47F00207FFF720FE009BD3F8C8
:10A2B00004B081E7264697E62378254603F0DF03BE
:10A2C000502B00F09E80CAF80050FAE6F0B700105C
:10A2D00050F000100F9BC3F101030F930F9B002B55
:10A2E0003FF47DAF029B0026DAF8107098461A46BC
:10A2F0004FEA870903EB870003E0904242F8046CC1
:10A3000044D9944652F8041B4B1CF6D00131022D5F
:10A31000CCF800107DD014F01F0440F0AB80212554
:10A320005FE70F9B002B3FF417AF50250198514674
:10A3300000F01CFA00230E9A2846136005B0BDE811
:10A34000F08F0020B0E6AB465DE6A61B51460198B3
:10A3500000273246ABEB060B00F04AFC00F1140379
:10A3600082460293D2E67278751C18F802102E46C7
:10A3700000293FF448AE16F8012F18F80230002BE0
:10A38000F9D13DE68C1C4FF0000917E6DAF80820F9
:10A39000974248DA7A1C01210AEB8707022DCAF896
:10A3A0001020DDF80880796133D0002A6FDC0022AC
:10A3B000CAF810200022CAF81420009B0BF1010BF0
:10A3C0009A685A45ABDA5146019800F0CFF900235C
:10A3D0000E9AA325136079E6012754E7029E4FF0F9
:10A3E000000980E63146504600F09CFE07464AE7E9
:10A3F000B11E504600F096FE00283FF412AF03272E
:10A4000010E74FF0000B012746E60F9B002B8CD086
:10A41000A2E6009B1A68013AA24263D02225E0E638
:10A420004FF00109D9E5DAF804100198013100F084
:10A4300077F9064600286FD0DAF810200AF10C01EF
:10A440000C3006F1140802329200FCF775F95146FF
:10A450000198B24600F08AF931690120022D01EB22
:10A46000000206EB810132614861D2D09742BFF60B
:10A4700052AF9AE7C144C4F1200459F8040C00F02B
:10A4800029FAA042BFF64BAFDAF810208DE708EBAF
:10A4900082000AF11804DAF81420A0424FEA5202AE
:10A4A0002CD94546236842EAC37245F8042B54F878
:10A4B000042BA0424FEA5202F4D8A0EB0A0119394A
:10A4C0008908013148F8212008EB810102B10431EB
:10A4D000A1EB080241454FEAA202CAF810207FF41E
:10A4E0006CAF67E7621104F01F0458F822100122D4
:10A4F000A2400A4214BF2125222572E6C8F8002096
:10A500000AB14146E3E7CAF8102053E70246054B7B
:10A51000E4210548FAF740FD0246024B8421024837
:10A52000FAF73AFD5CB8001070B8001010B5046876
:10A530008646013409E014F8013BA3F1410CBCF15B
:10A54000190F98BF2033934207D111F8012B002A2D
:10A55000F1D10120CEF8004010BD002010BD00BF99
:10A5600009682DE9F04F4B1185B011F01F01044629
:10A5700002EB8303029140F09A80181F1946256868
:10A58000002641F8046C01352B78002B00F0A780E1
:10A59000B446019106468646DFF88081E14667466B
:10A5A000E346AA460146039418F8030000285CD14C
:10A5B000202B00F28E804F4520DD76451AD9BCF164
:10A5C000070F17DCCCF10804DEF800307046CDF838
:10A5D00000E0A400C4F1200CA646446804FA0CF57F
:10A5E0001D4324FA0EF3056040F8043F8642F4D878
:10A5F000DDF800E0724551D34FF0080C1AF8013F26
:10A60000002BD1D108460199002F68D0B64502D25F
:10A61000BCF1070F67DD72454CD2141F734653F827
:10A62000045B834244F8045FF9D9A0EB0E03441C99
:10A630000EF1010E23F003030433A64588BF042363
:10A640000024134443F8044B8342FBD951F8044CD3
:10A650001CB106E050F8043D1BB98242FAD1012337
:10A660000360052005B0BDE8F08F0CF1010C013747
:10A67000BCF1080F08DCDEF800301B0100F00F0011
:10A680001843CEF80000B9E77245B7D24EF804BCC3
:10A690000023AEF1040E4FF0010CEFE7AEF104061B
:10A6A0004EF804BCB9464FF0000CB646A6E7191D9B
:10A6B000184664E7029B51F8044C002BC8D0C3F144
:10A6C00020034FF0FF3525FA03F31C4041F8044CFA
:10A6D000BEE7292B084655460199039C1BD0042050
:10A6E00005B0BDE8F08FCCF10803DEF800407746F6
:10A6F0009B002546C3F120089C467B6803FA08F4BA
:10A700002C4323FA0CF53C6047F8045FBE42F4D8B2
:10A71000724582D3CEE70135256075E750F0001011
:10A7200038B5436C05460C464BB153F8240080B154
:10A73000026843F824200023C0E9033338BD2122F6
:10A740000421FBF77BF8034668640028EDD1002064
:10A7500038BD0121284601FA04F56A1D9200FBF775
:10A760006DF80028F3D0C0E90145E4E731B1436C4E
:10A770004A6853F82200086043F82210704700BF6F
:10A780002DE9F04107460E461C460D6901F1140EF5
:10A790000020DEF8001001308BB285424FEA1141F3
:10A7A00002FB03434FEA134C9BB202FB01CC03EBC9
:10A7B0000C434FEA1C444EF8043BEADC3CB1B3685E
:10A7C000AB4207DD06EB850301355C613561304640
:10A7D000BDE8F081716838460131FFF7A1FF80467E
:10A7E000A8B1326906F10C010C3002329200FBF77D
:10A7F000A3FF7B6C726853F82210316043F822602B
:10A80000464606EB850301355C613561DFE70246AC
:10A81000024BBA210248FAF7BFFB00BF5CB8001038
:10A82000D4B800102DE9F8431E4617460833264ACF
:10A830000C46092E82FB03124FEAE3730546C3EB75
:10A84000620338DD4FF0010C00214FEA4C0C01315E
:10A850006345FADC2846FFF763FF014668B3089BAF
:10A86000092F43614FF00103036112DC0A34092709
:10A87000BE420BDDF61B264414F8013B0A22284693
:10A88000303BFFF77DFFB4420146F5D10846BDE8F5
:10A89000F88304F109093C44C84618F8013B0A2230
:10A8A0002846303BFFF76CFFA0450146F5D1A7F1E4
:10A8B00008044C44DCE70021CCE70246034BD321DB
:10A8C0000348FAF769FB00BF398EE3385CB8001023
:10A8D000D4B80010B0F5803F034618D2030410200E
:10A8E000B3F1807F01D208301B02B3F1805F01D247
:10A8F00004301B01B3F1804F03D3002B06DB013082
:10A9000070479B0005D45B0005D4202070470020D1
:10A91000E6E7023070470330704700BF0368014626
:10A9200013F0070207D0DA071FD4980721D55B0878
:10A9300001200B60704798B2A0B11046DAB20AB994
:10A9400008301B0A1A0701D104301B099A0701D1EC
:10A9500002309B08DA0703D45B0800F1010006D03F
:10A960000B6070471B0C1020E8E700207047202088
:10A9700070479B0802200B60704700BF38B5436CDE
:10A9800004460D464BB15868B0B102685A600022C7
:10A9900001234561C0E9032338BD21220421FAF7D0
:10A9A0004DFF034660640028EDD1094B002240F2C0
:10A9B00045110848FAF7F0FA1C2201212046FAF75F
:10A9C0003DFF0028F1D001220223C0E90123DEE788
:10A9D0005CB80010D4B800102DE9F04FD1F8108009
:10A9E00085B015690E469246A84505DB2A465346B2
:10A9F00045468A4690461E4605EB0804DAE90113EF
:10AA0000A342B8BF0131FFF78BFE002800F08B8016
:10AA100000F1140707EB840E774505D23B46002270
:10AA200043F8042B9E45FBD814360AF1140906EBB3
:10AA3000880809EB8505464568D2A5EB0A030AF1AB
:10AA4000150ACDF808E0AE46153B039423F0030346
:10AA5000043355452CBF9B464FF0040B824605E05E
:10AA6000090C2CD1B04507F104074CD956F8041B4A
:10AA70008DB2002DF4D0CC463C46002301965CF804
:10AA8000040B216886B2E6458AB24FEA104005FB06
:10AA900006224FEA11411A4405FB001101EB124155
:10AAA00092B24FEA114342EA014244F8042BE6D83D
:10AAB000019E47F80B3056F8041C090CD2D03B68B5
:10AAC000002248463D461C46944602889BB201FB44
:10AAD00002C202EB144243EA024345F8043B50F839
:10AAE000043B2C684FEA134C7045A3B201FB0C33B6
:10AAF00003EB12434FEA134CE7D3B04547F80B3052
:10AB000007F10407B2D85046DDE902E4002C02DC6C
:10AB100005E0013C03D05EF8043D002BF9D0046150
:10AB200005B0BDE8F08F0246024B4FF4B171024808
:10AB3000FAF732FA5CB80010D4B8001012F0030330
:10AB40002DE9F041144607462CD10D46A4101CD027
:10AB50003E6C86B3E3074FF0000806D4641014D0AF
:10AB60003068A8B10646E307F8D53246294638468C
:10AB7000FFF732FF35B17B6C696853F821202A60FA
:10AB800043F8215064100546EAD12846BDE8F0811B
:10AB9000324631463846FFF71FFF30600646C0F8A0
:10ABA0000080E0E7013B0F4A52F823200023FFF723
:10ABB000E7FD0546CAE701213846FFF7B1FD064625
:10ABC00040B1012340F27122C0E90432002338640D
:10ABD0000360BFE70246044B40F245110348FAF711
:10ABE000DBF900BF50F100105CB80010D4B80010C1
:10ABF0002DE9F0470C46904606464FEA6219276950
:10AC0000A36807EB621749687D1C9D4203DD5B006A
:10AC100001319D42FBDC3046FFF782FD002850D019
:10AC2000B9F1000F00F1140C0EDD09F105026346C5
:10AC300000214FEA820E00EB820243F8041B93428C
:10AC4000FBD1AEF114039C4404F11403216918F004
:10AC50001F0803EB81012BD0C8F12009E6464FF015
:10AC6000000A1A6802FA08F242EA0A024EF8042BB5
:10AC700053F8042B994222FA09FAF2D80B1B04F17B
:10AC80001502153B23F003030433914238BF04231C
:10AC90004CF803A0BAF1000F00D13D46736C626816
:10ACA000056153F82210216043F82240BDE8F08787
:10ACB000ACF1040C53F8042B99424CF8042FF9D84A
:10ACC000EBE70246024B4FF4EF710248FAF764F9E2
:10ACD0005CB80010D4B8001084460B690069C01A33
:10ACE00016D10CF1140C14310CEB830201EB83032D
:10ACF00010B401E0944508D252F8044D53F8041DF5
:10AD00008C42F7D005D24FF0FF305DF8044B70470E
:10AD1000704701205DF8044B704700BF2DE9F04FEC
:10AD200015460A6983B088462B69D21A002A40F07A
:10AD30008B8001F1140605F1140101EB830106EB90
:10AD4000830302E09E4280F0828053F8044D51F864
:10AD5000042D9442F6D078D32B46002445469846DD
:10AD60006968FFF7DDFC002800F08C802E6905F192
:10AD7000140B08F1140ED8F8103000F1140A05F184
:10AD800010020EEB83094FF0000C0BEB86015746C7
:10AD9000C460CDF804B05EF8044B52F8045F1FFAAB
:10ADA00084FBF145ABB24FEA1444A3EB0B03C4EBB5
:10ADB0001544634404EB23449BB24FEA244C43EA1A
:10ADC000044347F8043BE6D8A9EB080408F115084A
:10ADD000DDF804B0C145A4F1150434BF4FF00008FC
:10ADE0004FF00108A408B8F1000F04F101024FEA86
:10ADF000820208BF04220BEB02055244A94231D95A
:10AE000017462C4654F8043B1FFA83F8A1424FEA38
:10AE1000134E6344C4449BB20EEB2C4C43EA0C43E8
:10AE20004FEA2C4C47F8043BECD80139491B21F080
:10AE300003010A4423B952F8043D013E002BFAD025
:10AE4000066103B0BDE8F08F86DA012488E70021AF
:10AE5000FFF766FC78B101220023C0E9042303B0A8
:10AE6000BDE8F08FB8F1000F4FEA840408BF00245A
:10AE70000AEB0402DEE70246064B40F237210648A1
:10AE8000FAF78AF80246034B40F245210248FAF7E6
:10AE900083F800BF5CB80010D4B80010114B0B4011
:10AEA000A3F15073002B03DD0022194610467047B2
:10AEB0005B42B3F1A07F4FEA235106DA4FF400233F
:10AEC00000220B4110461946704714391E2904DD33
:10AED000012200231046194670474FF00042CA4035
:10AEE000F7E700BF0000F07F2DE9F041026900F1B3
:10AEF000140707EB820252F8046CA2F104083046F2
:10AF0000FFF7E8FCC0F120030A280B6035DD474558
:10AF1000A0F10B011BD252F8083C31B3C1F1200C57
:10AF20008E40A2F1080023FA0CF48B40874246EAD7
:10AF3000040646F07F5545F440151AD252F80C2C01
:10AF4000294622FA0CF213431846BDE8F0810B287B
:10AF50000AD006FA01F1002341F07F55184645F466
:10AF600040152946BDE8F081002346F07F5545F4A1
:10AF7000401518462946BDE8F081C0F10B0347454E
:10AF800026FA03F141F07F5545F4401509D300221C
:10AF900000F11503294606FA03F313431846BDE8EA
:10AFA000F08152F8082CDA40F2E700BFF0B5012139
:10AFB00083B016461F46FFF7B3FB0546002849D06D
:10AFC000C7F30A54C7F313030CB143F48013002EE4
:10AFD000019315D101A8FFF7A1FC0199012200F10D
:10AFE000200369612A611CB3A4F23344C3F1350024
:10AFF0001C44089B1C60099B1860284603B0F0BDE8
:10B0000068460096FFF78AFC019A034600B3C0F138
:10B01000200102FA01F1C240009801920143002A86
:10B02000C5E905120CBF012202222A61002CDBD1E6
:10B03000A3F23243089805EB820103600869FFF729
:10B0400049FC099BC0EB42101860284603B0F0BDD4
:10B050000099E4E70246034B40F20F310248F9F74A
:10B060009BFF00BF5CB80010D4B800102DE9F0437E
:10B0700083B0884681466946FFF736FF04460D4691
:10B08000404601A9FFF730FFD9F81030D8F810205A
:10B09000A3EB020CDDE900329B1A03EB4C13002BEF
:10B0A0000BDD05EB03573D4602460B46204629467D
:10B0B000F7F7C6FB03B0BDE8F083C3EB033301EB46
:10B0C00003594946F0E700BF013902F114034FEA82
:10B0D000611C116903EB81010CF1010C8B4200EB47
:10B0E0008C0C16D210B5A0F1040E53F8044B994203
:10B0F0004EF8044FF9D88B1A153B23F003030433A1
:10B100001844844504D9002340F8043B8445FBD807
:10B1100010BD844505D9002340F8043B8445FBD885
:10B120007047704703694A111430934209DA00EB03
:10B13000830302E053F8042DAAB98342FAD8002011
:10B14000704700EB8203F8DD11F01F01F5D010B459
:10B1500050F8224024FA01F28A40944209D001209A
:10B160005DF8044B70470120704753F8042D002A06
:10B17000F5D18342F9D800205DF8044B704700BF39
:10B18000154B984226D840F6F90C70B54FF0000EDA
:10B19000124D03E004F1010EF44519DB1CEB0E0225
:10B1A00048BF013222F00103541003EB620305EBA8
:10B1B00043015B004A784E88898842EA062211449E
:10B1C0008842E7D8904204F1FF3CE5D3E85C70BDCB
:10B1D000FF2070BDFF207047EF010E0050F20010FD
:10B1E000F8B500BF000000005FF800F07105002016
:10B1F0005FF800F0210600205FF800F06D020020EB
:10B200005FF800F0110100205FF800F0010200205B
:10B2100039260010AD250010E1250010852600100C
:10B2200019260010152500106126001001250010B8
:10B23000051B001065260010711E00105D25001012
:10B240004D260010FD2500102D1700105517001079
:08B2500019020010C95500109D
:10B258001B5B25643B256448000000001B5B316DC7
:10B26800000000001B5B33383B353B25646D000054
:10B278001B5B34383B353B25646D00004B617270B5
:10B288006C75732D5374726F6E6720537472696E88
:10B29800672053796E746820666F7220727032333B
:10B2A80035302C206563653437363020436F726E35
:10B2B800656C6C20556E69766572736974792C209B
:10B2C80032303235000000001B5B306D000000009A
:10B2D800706C75636B2028312F30293D2564202040
:10B2E80020000000706C75636B74797065202830DD
:10B2F8002D33293D2564202020000000706C7563E3
:10B308006B77696474682028312D3135293D2564AF
:10B318002020200064616D70696E673D25352E33ED
:10B3280066202020000000006C6F77706173733D09
:10B3380025352E3366202020000000006E6F7465CE
:10B34800206475726174696F6E3D25352E326620F2
:10B3580020200000626F772061747461636B3D2563
:10B36800352E336620202000626F77206465636184
:10B37800793D25352E33662020200000626F772026
:10B38800616D703D25352E306620202000000000BC
:10B39800626F77206672657175656E63793D2535D4
:10B3A8002E33662020200000626F77207479706544
:10B3B8003D256420202000001B5B33326D00000017
:10B3C8000A0D2A2A2A636F6D6D616E64732A2A2A10
:10B3D8000A0D706C6179202D2D20706C61792073B5
:10B3E80063616C650A0D000073746F70202D2D2049
:10B3F800706C61796E670A0D00000000706C7563EF
:10B408006B20312F30202D2D20656E61626C6520F8
:10B41800696E697469616C20706C75636B0A0D00E4
:10B42800706C75636B7479706520302D33202D2D09
:10B43800206E6F6973652C206C70206E6F69736560
:10B448002C20676175737369616E2C207361777442
:10B458006F6F74680A0D0000706C75636B776964B0
:10B468007468202D2D203120746F20323020666FB3
:10B478007220747970652032206761757373696111
:10B488006E200A0D00000000626F776174746163BA
:10B498006B2074696D65202D2D2072697365207489
:10B4A800696D6520696E207365636F6E64730A0D3C
:10B4B80000000000626F7764656361792074696DCC
:10B4C80065202D2D2066616C6C2074696D6520697E
:10B4D8006E207365636F6E64730A0D00626F776127
:10B4E8006D7020616D706C6974756465202D2D20F8
:10B4F800696E7465676572203020746F2031303052
:10B5080030200A0D00000000626F777479706520A2
:10B51800302D31202D2D2073696E652F6E6F697364
:10B5280065200A0D00000000626F77667265712061
:10B5380072656C61746976655F66726571202D2D20
:10B548002072656C617469766520746F20737472FB
:10B55800696E672066756E64616D656E74616C0AEC
:10B568000D00000064616D70696E6720636F656629
:10B5780066202D2D20302E3820746F20312E300A71
:10B588000D0000006C6F777061737320636F6566E0
:10B5980066202D2D20302E3520746F20312E30203E
:10B5A800200A0D0074656D706F2074696D65202D1B
:10B5B8002D207365636F6E647320200A0D000000F0
:10B5C8002020202020202020202020202020202073
:10B5D80020202020000000004B5320636D643E2093
:10B5E80000000000706C61790000000073746F70D7
:10B5F80000000000706C75636B000000256400009B
:10B60800706C75636B74797065000000706C75639D
:10B618006B77696474680000626F77617474616342
:10B628006B00000025660000626F776465636179CE
:10B6380000000000626F77616D700000626F7766CE
:10B6480072657100626F77747970650064616D70FE
:10B65800696E67006C6F77706173730074656D70E5
:10B668006F0000002A2A2A6875683F2062616420FA
:10B67800636F6D6D616E642A2A2A20000A0D50726C
:10B688006F746F746872656164732052503230341D
:10B69800302076312E332074776F2D636F72652CCE
:10B6A800207072696F726974790A0D000A2A2A2A51
:10B6B8002050414E4943202A2A2A0A000A00000045
:10B6C800486172647761726520616C61726D2025D2
:10B6D8006420616C726561647920636C61696D6571
:10B6E80064000000486172642061737365727400BD
:10B6F8004F7574206F66206D656D6F72790000005C
:10B7080052656C6561736500626F6F74325F773282
:10B718003571303830000000322E312E30000000F4
:10B728007069636F320000006772617068696373E3
:10B738005F746573740000004A616E2031332032F3
:10B7480030323500666E692B00000000666E6900B5
:10B758006E616E00666E692D000000002C20667513
:10B768006E6374696F6E3A20000000006173736540
:10B778007274696F6E2022257322206661696C6578
:10B78800643A2066696C6520222573222C206C6936
:10B798006E65202564257325730A000055415254AF
:10B7A80020737464696E00005541525420737464A8
:10B7B8006F7574005541525420737464696E202F5C
:10B7C800207374646F757400646F75626C652072A1
:10B7D80065736574202D3E20424F4F5453454C00ED
:10B7E80065256C64000000002E0000004C435F4398
:10B7F8004F4C4C41544500004C435F43545950450D
:10B80800000000004C435F4D4F4E455441525900D3
:10B818004C435F4E554D4552494300004C435F54DD
:10B82800494D45004C435F4D4553534147455300EF
:10B838006E660000696E697479000000616E000030
:10B848004A495300534A4953000000004555434AAA
:10B858005000000042616C6C6F6320737563636510
:10B8680065646564000000002F646174612F6A6577
:10B878006E6B696E732F776F726B73706163652F70
:10B88800474E552D746F6F6C636861696E2F6172D6
:10B898006D2D31332F7372632F6E65776C69622D4E
:10B8A80063796777696E2F6E65776C69622F6C694B
:10B8B80062632F7374646C69622F6764746F612D9F
:10B8C8006765746865782E63000000002F646174F2
:10B8D800612F6A656E6B696E732F776F726B737009
:10B8E8006163652F474E552D746F6F6C636861698E
:10B8F8006E2F61726D2D31332F7372632F6E6577E2
:10B908006C69622D63796777696E2F6E65776C69EC
:10B91800622F6C6962632F7374646C69622F6D7037
:10B928007265632E6300000006005250D3F0754222
:10B9380008B7001006005250E182887F10B7001047
:10B9480006005250ABB3605320B7001006005250A7
:10B95800BBFF3CB628B7001006005250861C0302F5
:10B9680030B70010060052505422A29D40B7001074
:10B9780005005250DE65F468E03801100000000050
:10B98800000000000000F03F00000000000024401C
:10B9980000000000000059400000000000408F40F7
:10B9A800000000000088C34000000000006AF84062
:10B9B8000000000080842E4100000000D012634186
:10B9C8000000000084D797410000000065CDCD41FC
:10B9D8000D0A00000600525053B4F4A1BCB7001081
:10B9E8000800525012000000080052509210000047
:10B9F8000600525053B4F4A1D0B700100020202004
:10BA08002020202020202828282828202020202006
:10BA180020202020202020202020202020881010D6
:10BA28001010101010101010101010101004040432
:10BA380004040404040404101010101010104141F0
:10BA480041414141010101010101010101010101DE
:10BA580001010101010101011010101010104242F2
:10BA680042424242020202020202020202020202AE
:10BA7800020202020202020210101010200000004E
:10BA880000000000000000000000000000000000AE
:10BA9800000000000000000000000000000000009E
:10BAA800000000000000000000000000000000008E
:10BAB800000000000000000000000000000000007E
:10BAC800000000000000000000000000000000006E
:10BAD800000000000000000000000000000000005E
:10BAE800000000000000000000000000000000004E
:10BAF800000000000000000000000000000000003E
:10BB08000A00010002000300040005000600070007
:10BB1800080009000A000B000C000D000E000F00C1
:10BB28001000000034000000CEFBFFFFCB03000034
:10BB3800010000000000000035000000CEFBFFFF00
:10BB4800CB0300000100000000000000000000001E
:10BB5800BC89D897B2D29C3C33A7A8D523F64939DB
:10BB68003DA7F444FD0FA5329D978CCF08BA5B25FD
:10BB7800436FAC64280668110C5F104E154E2A4EB0
:10BB8800314E364E3C4E3F4E424E564E584E824EE9
:10BB9800854E6B8C8A4E12820D5F8E4E9E4E9F4E46
:10BBA800A04EA24EB04EB34EB64ECE4ECD4EC44E63
:10BBB800C64EC24ED74EDE4EED4EDF4EF74E094F03
:10BBC8005A4F304F5B4F5D4F574F474F764F884F17
:10BBD8008F4F984F7B4F694F704F914F6F4F864FE4
:10BBE800964F1851D44FDF4FCE4FD84FDB4FD14F20
:10BBF800DA4FD04FE44FE54F1A50285014502A50CE
:10BC0800255005501C4FF64F215029502C50FE4FFF
:10BC1800EF4F11500650435047500367555050504E
:10BC280048505A5056506C50785080509A50855011
:10BC3800B450B250C950CA50B350C250D650DE505A
:10BC4800E550ED50E350EE50F950F55009510151CF
:10BC580002511651155114511A5121513A51375167
:10BC68003C513B513F51405152514C5154516251FA
:10BC7800F87A69516A516E5180518251D8568C5167
:10BC880089518F519151935195519651A451A65173
:10BC9800A251A951AA51AB51B351B151B251B051AE
:10BCA800B551BD51C551C951DB51E0515586E951D6
:10BCB800ED51F051F551FE5104520B5214520E52EF
:10BCC80027522A522E52335239524F5244524B5213
:10BCD8004C525E5254526A527452695273527F5295
:10BCE8007D528D5294529252715288529152A88F1D
:10BCF800A78FAC52AD52BC52B552C152CD52D75299
:10BD0800DE52E352E652ED98E052F352F552F85201
:10BD1800F9520653085338750D5310530F531553E2
:10BD28001A5323532F5331533353385340534653E5
:10BD38004553174E49534D53D6515E5369536E536D
:10BD480018597B53775382539653A053A653A55340
:10BD5800AE53B053B653C353127CD996DF53FC6627
:10BD6800EE71EE53E853ED53FA5301543D544054E9
:10BD78002C542D543C542E54365429541D544E548E
:10BD88008F5475548E545F54715477547054925430
:10BD98007B5480547654845490548654C754A25487
:10BDA800B854A554AC54C454C854A854AB54C25441
:10BDB800A454BE54BC54D854E554E6540F551455F5
:10BDC800FD54EE54ED54FA54E25439554055635538
:10BDD8004C552E555C554555565557553855335580
:10BDE8005D5599558055AF548A559F557B557E555D
:10BDF80098559E55AE557C558355A9558755A855D8
:10BE0800DA55C555DF55C455DC55E455D455145697
:10BE1800F7551656FE55FD551B56F9554E565056B4
:10BE2800DF7134563656325638566B5664562F568E
:10BE38006C566A56865680568A56A05694568F5621
:10BE4800A556AE56B656B456C256BC56C156C3567B
:10BE5800C056C856CE56D156D356D756EE56F95672
:10BE68000057FF560457095708570B570D571357D4
:10BE780018571657C7551C572657375738574E5710
:10BE88003B5740574F576957C057885761577F5797
:10BE980089579357A057B357A457AA57B057C357B2
:10BEA800C657D457D257D3570A58D657E3570B58C3
:10BEB80019581D587258215862584B587058C06B01
:10BEC80052583D5879588558B9589F58AB58BA5860
:10BED800DE58BB58B858AE58C558D358D158D7585B
:10BEE800D958D858E558DC58E458DF58EF58FA586C
:10BEF800F958FB58FC58FD5802590A5910591B5952
:10BF0800A66825592C592D59325938593E59D27A93
:10BF1800555950594E595A59585962596059675983
:10BF28006C596959785981599D595E4FAB4FA3593E
:10BF3800B259C659E859DC598D59D959DA59255A8F
:10BF48001F5A115A1C5A095A1A5A405A6C5A495AB5
:10BF5800355A365A625A6A5A9A5ABC5ABE5ACB5AF3
:10BF6800C25ABD5AE35AD75AE65AE95AD65AFA5A21
:10BF7800FB5A0C5B0B5B165B325BD05A2A5B365B59
:10BF88003E5B435B455B405B515B555B5A5B5B5B70
:10BF9800655B695B705B735B755B785B88657A5B17
:10BFA800805B835BA65BB85BC35BC75BC95BD45B29
:10BFB800D05BE45BE65BE25BDE5BE55BEB5BF05B87
:10BFC800F65BF35B055C075C085C0D5C135C205C4E
:10BFD800225C285C385C395C415C465C4E5C535C96
:10BFE800505C4F5C715B6C5C6E5C624E765C795C3D
:10BFF8008C5C915C945C9B59AB5CBB5CB65CBC5C38
:10C00800B75CC55CBE5CC75CD95CE95CFD5CFA5C8E
:10C01800ED5C8C5DEA5C0B5D155D175D5C5D1F5D1D
:10C028001B5D115D145D225D1A5D195D185D4C5D27
:10C03800525D4E5D4B5D6C5D735D765D875D845DC5
:10C04800825DA25D9D5DAC5DAE5DBD5D905DB75DE1
:10C05800BC5DC95DCD5DD35DD25DD65DDB5DEB5D5D
:10C06800F25DF55D0B5E1A5E195E115E1B5E365E53
:10C07800375E445E435E405E4E5E575E545E5F5E72
:10C08800625E645E475E755E765E7A5EBC9E7F5ECB
:10C09800A05EC15EC25EC85ED05ECF5ED65EE35E65
:10C0A800DD5EDA5EDB5EE25EE15EE85EE95EEC5E86
:10C0B800F15EF35EF05EF45EF85EFE5E035F095FBC
:10C0C8005D5F5C5F0B5F115F165F295F2D5F385FF7
:10C0D800415F485F4C5F4E5F2F5F515F565F575F10
:10C0E800595F615F6D5F735F775F835F825F7F5FBB
:10C0F8008A5F885F915F875F9E5F995F985FA05FA7
:10C10800A85FAD5FBC5FD65FFB5FE45FF85FF15F80
:10C11800DD5FB360FF5F21606060196010602960B7
:10C128000E6031601B6015602B6026600F603A60FE
:10C138005A6041606A6077605F604A6046604D603F
:10C1480063604360646042606C606B6059608160EA
:10C158008D60E76083609A6084609B6096609760FA
:10C168009260A7608B60E160B860E060D360B46003
:10C17800F05FBD60C660B560D8604D61156106614D
:10C18800F660F7600061F460FA6003612161FB60AA
:10C19800F1600D610E6147613E61286127614A6166
:10C1A8003F613C612C6134613D614261446173616E
:10C1B8007761586159615A616B6174616F6165613A
:10C1C80071615F615D6153617561996196618761B4
:10C1D800AC6194619A618A619161AB61AE61CC6135
:10C1E800CA61C961F761C861C361C661BA61CB61DF
:10C1F800797FCD61E661E361F661FA61F461FF611F
:10C20800FD61FC61FE610062086209620D620C62F8
:10C2180014621B621E6221622A622E6230623262DE
:10C22800336241624E625E6263625B626062686250
:10C238007C62826289627E62926293629662D46252
:10C2480083629462D762D162BB62CF62FF62C662C8
:10C25800D464C862DC62CC62CA62C262C7629B6292
:10C26800C9620C63EE62F162276302630863EF62DE
:10C27800F56250633E634D631C644F6396638E633F
:10C288008063AB637663A3638F6389639F63B563DE
:10C298006B636963BE63E963C063C663E363C963D1
:10C2A800D263F663C4631664346406641364266454
:10C2B80036641D65176428640F6467646F64766468
:10C2C8004E642A6595649364A564A9648864BC6413
:10C2D800DA64D264C564C764BB64D864C264F164B8
:10C2E800E7640982E064E164AC62E364EF642C65AE
:10C2F800F664F464F264FA640065FD6418651C650C
:10C308000565246523652B653465356537653665B0
:10C3180038654B754865566555654D6558655E6564
:10C328005D6572657865826583658A8B9B659F65A7
:10C33800AB65B765C365C665C165C465CC65D265BF
:10C34800DB65D965E065E165F16572670A660366D4
:10C35800FB6573673566366634661C664F664466E9
:10C36800496641665E665D666466676668665F66BE
:10C3780062667066836688668E6689668466986675
:10C388009D66C166B966C966BE66BC66C466B8669F
:10C39800D666DA66E0663F66E666E966F066F566E2
:10C3A800F7660F6716671E672667276738972E6731
:10C3B8003F67366741673867376746675E67606714
:10C3C80059676367646789677067A9677C676A6785
:10C3D8008C678B67A667A1678567B767EF67B467E0
:10C3E800EC67B367E967B867E467DE67DD67E2674C
:10C3F800EE67B967CE67C667E7679C6A1E684668D6
:10C40800296840684D6832684E68B3682B68596877
:10C41800636877687F689F688F68AD6894689D686F
:10C428009B688368AE6AB9687468B568A068BA68BA
:10C438000F698D687E680169CA680869D8682269C9
:10C448002669E1680C69CD68D468E768D5683669FB
:10C4580012690469D768E3682569F968E068EF68D4
:10C4680028692A691A6923692169C6687969776917
:10C478005C6978696B6954697E696E693969746940
:10C488003D695969306961695E695D6981696A698F
:10C49800B269AE69D069BF69C169D369BE69CE693D
:10C4A800E85BCA69DD69BB69C369A7692E6A9169D6
:10C4B800A0699C699569B469DE69E869026A1B6AC2
:10C4C800FF690A6BF969F269E769056AB1691E6A69
:10C4D800ED69146AEB690A6A126AC16A236A136A07
:10C4E800446A0C6A726A366A786A476A626A596A82
:10C4F800666A486A386A226A906A8D6AA06A846A9B
:10C50800A26AA36A976A1786BB6AC36AC26AB86ACC
:10C51800B36AAC6ADE6AD16ADF6AAA6ADA6AEA6A68
:10C52800FB6A056B1686FA6A126B166B319B1F6BDA
:10C53800386B376BDC76396BEE98476B436B496B1E
:10C54800506B596B546B5B6B5F6B616B786B796B82
:10C558007F6B806B846B836B8D6B986B956B9E6B1D
:10C56800A46BAA6BAB6BAF6BB26BB16BB36BB76BF6
:10C57800BC6BC66BCB6BD36BDF6BEC6BEB6BF36B92
:10C58800EF6BBE9E086C136C146C1B6C246C236CD4
:10C598005E6C556C626C6A6C826C8D6C9A6C816C8A
:10C5A8009B6C7E6C686C736C926C906CC46CF16C58
:10C5B800D36CBD6CD76CC56CDD6CAE6CB16CBE6CED
:10C5C800BA6CDB6CEF6CD96CEA6C1F6D4D88366DFC
:10C5D8002B6D3D6D386D196D356D336D126D0C6DAC
:10C5E800636D936D646D5A6D796D596D8E6D956D32
:10C5F800E46F856DF96D156E0A6EB56DC76DE66DE4
:10C60800B86DC66DEC6DDE6DCC6DE86DD26DC56D27
:10C61800FA6DD96DE46DD56DEA6DEE6D2D6E6E6EA9
:10C628002E6E196E726E5F6E3E6E236E6B6E2B6E83
:10C63800766E4D6E1F6E436E3A6E4E6E246EFF6EB2
:10C648001D6E386E826EAA6E986EC96EB76ED36E06
:10C65800BD6EAF6EC46EB26ED46ED56E8F6EA56EA3
:10C66800C26E9F6E416F116F4C70EC6EF86EFE6E6D
:10C678003F6FF26E316FEF6E326FCC6E3E6F136F9D
:10C68800F76E866F7A6F786F816F806F6F6F5B6FF1
:10C69800F36F6D6F826F7C6F586F8E6F916FC26F83
:10C6A800666FB36FA36FA16FA46FB96FC66FAA6FE0
:10C6B800DF6FD56FEC6FD46FD86FF16FEE6FDB6FF4
:10C6C80009700B70FA6F117001700F70FE6F1B709C
:10C6D8001A70746F1D7018701F7030703E70327051
:10C6E8005170637099709270AF70F170AC70B870DF
:10C6F800B370AE70DF70CB70DD70D9700971FD70EA
:10C708001C711971657155718871667162714C710E
:10C7180056716C718F71FB7184719571A871AC71D0
:10C72800D771B971BE71D271C971D471CE71E0710E
:10C73800EC71E771F571FC71F971FF710D7210728E
:10C748001B7228722D722C72307232723B723C72DC
:10C758003F72407246724B72587274727E72827265
:10C768008172877292729672A272A772B972B2724D
:10C77800C372C672C472CE72D272E272E072E17291
:10C78800F972F7720F5017730A731C7316731D73BF
:10C7980034732F73297325733E734E734F73D89E6A
:10C7A80057736A7368737073787375737B737A736E
:10C7B800C873B373CE73BB73C073E573EE73DE7364
:10C7C800A27405746F742574F87332743A745574CE
:10C7D8003F745F74597441745C74697470746374E1
:10C7E8006A7476747E748B749E74A774CA74CF74DA
:10C7F800D474F173E074E374E774E974EE74F2745A
:10C80800F074F174F874F7740475037505750C7594
:10C818000E750D75157513751E7526752C753C7579
:10C8280044754D754A7549755B7546755A756975D0
:10C83800647567756B756D757875767586758775AA
:10C8480074758A758975827594759A759D75A575BF
:10C85800A375C275B375C375B575BD75B875BC7567
:10C86800B175CD75CA75D275D975E375DE75FE7566
:10C87800FF75FC750176F075FA75F275F3750B7630
:10C888000D7609761F76277620762176227624760D
:10C89800347630763B764776487646765C765876B8
:10C8A80061766276687669766A7667766C7670768F
:10C8B8007276767678767C768076837688768B76CE
:10C8C8008E769676937699769A76B076B476B876AA
:10C8D800B976BA76C276CD76D676D276DE76E17637
:10C8E800E576E776EA762F86FB760877077704778A
:10C8F800297724771E77257726771B773777387738
:10C9080047775A7768776B775B7765777F777E7736
:10C9180079778E778B779177A0779E77B077B67790
:10C92800B977BF77BC77BD77BB77C777CD77D77730
:10C93800DA77DC77E377EE77FC770C78127826796C
:10C9480020782A7945788E78747886787C789A78F1
:10C958008C78A378B578AA78AF78D178C678CB7870
:10C96800D478BE78BC78C578CA78EC78E778DA7875
:10C97800FD78F47807791279117919792C792B795E
:10C988004079607957795F795A79557953797A7905
:10C998007F798A799D79A7794B9FAA79AE79B379FE
:10C9A800B979BA79C979D579E779EC79E179E3790F
:10C9B800087A0D7A187A197A207A1F7A8079317A6A
:10C9C8003B7A3E7A377A437A577A497A617A627A39
:10C9D800697A9D9F707A797A7D7A887A977A957A3A
:10C9E800987A967AA97AC87AB07AB67AC57AC47AE1
:10C9F800BF7A8390C77ACA7ACD7ACF7AD57AD37A32
:10CA0800D97ADA7ADD7AE17AE27AE67AED7AF07A38
:10CA1800027B0F7B0A7B067B337B187B197B1E7B93
:10CA2800357B287B367B507B7A7B047B4D7B0B7B6D
:10CA38004C7B457B757B657B747B677B707B717BEF
:10CA48006C7B6E7B9D7B987B9F7B8D7B9C7B9A7B95
:10CA58008B7B927B8F7B5D7B997BCB7BC17BCC7BFC
:10CA6800CF7BB47BC67BDD7BE97B117C147CE67BCA
:10CA7800E57B607C007C077C137CF37BF77B177C71
:10CA88000D7CF67B237C277C2A7C1F7C377C2B7CC7
:10CA98003D7C4C7C437C547C4F7C407C507C587C57
:10CAA8005F7C647C567C657C6C7C757C837C907C2C
:10CAB800A47CAD7CA27CAB7CA17CA87CB37CB27C42
:10CAC800B17CAE7CB97CBD7CC07CC57CC27CD87C8A
:10CAD800D27CDC7CE27C3B9BEF7CF27CF47CF67CB9
:10CAE800FA7C067D027D1C7D157D0A7D457D4B7D8A
:10CAF8002E7D327D3F7D357D467D737D567D4E7D15
:10CB0800727D687D6E7D4F7D637D937D897D5B7DC4
:10CB18008F7D7D7D9B7DBA7DAE7DA37DB57DC77DF7
:10CB2800BD7DAB7D3D7EA27DAF7DDC7DB87D9F7DEB
:10CB3800B07DD87DDD7DE47DDE7DFB7DF27DE17D10
:10CB4800057E0A7E237E217E127E317E1F7E097E2F
:10CB58000B7E227E467E667E3B7E357E397E437E18
:10CB6800377E327E3A7E677E5D7E567E5E7E597E59
:10CB78005A7E797E6A7E697E7C7E7B7E837ED57DC9
:10CB88007D7EAE8F7F7E887E897E8C7E927E907E33
:10CB9800937E947E967E8E7E9B7E9C7E387F3A7FA7
:10CBA800457F4C7F4D7F4E7F507F517F557F547F0F
:10CBB800587F5F7F607F687F697F677F787F827F2C
:10CBC800867F837F887F877F8C7F947F9E7F9D7FF2
:10CBD8009A7FA37FAF7FB27FB97FAE7FB67FB87FE2
:10CBE800718BC57FC67FCA7FD57FD47FE17FE67F03
:10CBF800E97FF37FF97FDC98068004800B80128040
:10CC0800188019801C80218028803F803B804A80C2
:10CC18004680528058805A805F8062806880738026
:10CC280072807080768079807D807F808480868025
:10CC380085809B8093809A80AD809051AC80DB800A
:10CC4800E580D980DD80C480DA80D6800981EF80D4
:10CC5800F1801B81298123812F814B818B9646810D
:10CC68003E8153815181FC8071816E81658166812D
:10CC78007481838188818A8180818281A081958164
:10CC8800A481A3815F819381A981B081B581BE818F
:10CC9800B881BD81C081C281BA81C981CD81D1816C
:10CCA800D981D881C881DA81DF81E081E781FA8181
:10CCB800FB81FE8101820282058207820A820D823F
:10CCC8001082168229822B823882338240825982CE
:10CCD80058825D825A825F826482628268826A8236
:10CCE8006B822E827182778278827E828D82928296
:10CCF800AB829F82BB82AC82E182E382DF82D282F6
:10CD0800F482F382FA8293830383FB82F982DE82C0
:10CD18000683DC820983D982358334831683328380
:10CD2800318340833983508345832F832B83178333
:10CD3800188385839A83AA839F83A28396832383F8
:10CD48008E8387838A837C83B58373837583A0836B
:10CD58008983A883F4831384EB83CE83FD830384C0
:10CD6800D8830B84C183F7830784E083F2830D841F
:10CD780022842084BD8338840685FB836D842A84BD
:10CD88003C845A85848477846B84AD846E848284E1
:10CD9800698446842C846F8479843584CA84628447
:10CDA800B984BF849F84D984CD84BB84DA84D08439
:10CDB800C184C684D684A1842185FF84F484178520
:10CDC80018852C851F8515851485FC844085638509
:10CDD80058854885418502864B8555858085A4857B
:10CDE800888591858A85A8856D8594859B85EA8542
:10CDF80087859C8577857E859085C985BA85CF8509
:10CE0800B985D085D585DD85E585DC85F9850A86F2
:10CE180013860B86FE85FA85068622861A86308654
:10CE28003F864D86554E54865F8667867186938603
:10CE3800A386A986AA868B868C86B686AF86C48684
:10CE4800C686B086C9862388AB86D486DE86E98600
:10CE5800EC86DF86DB86EF861287068708870087E1
:10CE68000387FB86118709870D87F9860A87348728
:10CE78003F8737873B87258729871A8760875F879A
:10CE880078874C874E877487578768876E87598756
:10CE9800538763876A870588A2879F878287AF87BA
:10CEA800CB87BD87C087D087D696AB87C487B38723
:10CEB800C787C687BB87EF87F287E0870F880D880B
:10CEC800FE87F687F7870E88D28711881688158817
:10CED8002288218831883688398827883B88448881
:10CEE8004288528859885E8862886B8881887E88E3
:10CEF8009E8875887D88B588728882889788928888
:10CF0800AE889988A2888D88A488B088BF88B1889F
:10CF1800C388C488D488D888D988DD88F9880289E4
:10CF2800FC88F488E888F28804890C890A891389BE
:10CF380043891E8925892A892B89418944893B8906
:10CF4800368938894C891D8960895E896689648932
:10CF58006D896A896F89748977897E8983898889C7
:10CF68008A8993899889A189A989A689AC89AF8971
:10CF7800B289BA89BD89BF89C089DA89DC89DD8926
:10CF8800E789F489F889038A168A108A0C8A1B8A29
:10CF98001D8A258A368A418A5B8A528A468A488A45
:10CFA8007C8A6D8A6C8A628A858A828A848AA88A3F
:10CFB800A18A918AA58AA68A9A8AA38AC48ACD8ACE
:10CFC800C28ADA8AEB8AF38AE78AE48AF18A148BBE
:10CFD800E08AE28AF78ADE8ADB8A0C8B078B1A8B57
:10CFE800E18A168B108B178B208B338BAB97268B94
:10CFF8002B8B3E8B288B418B4C8B4F8B4E8B498BCD
:10D00800568B5B8B5A8B6B8B5F8B6C8B6F8B748B9C
:10D018007D8B808B8C8B8E8B928B938B968B998B45
:10D028009A8B3A8C418C3F8C488C4C8C4E8C508C13
:10D03800558C628C6C8C788C7A8C828C898C858CE3
:10D048008A8C8D8C8E8C948C7C8C988C1D62AD8C8B
:10D05800AA8CBD8CB28CB38CAE8CB68CC88CC18CAF
:10D06800E48CE38CDA8CFD8CFA8CFB8C048D058DBA
:10D078000A8D078D0F8D0D8D108D4E9F138DCD8CC4
:10D08800148D168D678D6D8D718D738D818D998D34
:10D09800C28DBE8DBA8DCF8DDA8DD68DCC8DDB8DC0
:10D0A800CB8DEA8DEB8DDF8DE38DFC8D088E098E9F
:10D0B800FF8D1D8E1E8E108E1F8E428E358E308EE9
:10D0C800348E4A8E478E498E4C8E508E488E598E9D
:10D0D800648E608E2A8E638E558E768E728E7C8ECE
:10D0E800818E878E858E848E8B8E8A8E938E918E7E
:10D0F800948E998EAA8EA18EAC8EB08EC68EB18E6D
:10D10800BE8EC58EC88ECB8EDB8EE38EFC8EFB8EDC
:10D11800EB8EFE8E0A8F058F158F128F198F138F46
:10D128001C8F1F8F1B8F0C8F268F338F3B8F398F50
:10D13800458F428F3E8F4C8F498F468F4E8F578F2A
:10D148005C8F628F638F648F9C8F9F8FA38FAD8F4F
:10D15800AF8FB78FDA8FE58FE28FEA8FEF8F8790E7
:10D16800F48F0590F98FFA8F1190159021900D90FA
:10D178001E9016900B902790369035903990F88F26
:10D188004F905090519052900E9049903E905690EA
:10D1980058905E9068906F907690A8967290829062
:10D1A8007D90819080908A9089908F90A890AF9080
:10D1B800B190B590E290E4904862DB9002911291B0
:10D1C8001991329130914A91569158916391659194
:10D1D8006991739172918B9189918291A291AB918E
:10D1E800AF91AA91B591B491BA91C091C191C991E9
:10D1F800CB91D091D691DF91E191DB91FC91F591A2
:10D20800F6911E92FF9114922C92159211925E92B1
:10D218005792459249926492489295923F924B92C6
:10D2280050929C92969293929B925A92CF92B992D4
:10D23800B792E9920F93FA9244932E9319932293FB
:10D248001A9323933A9335933B935C9360937C931F
:10D258006E935693B093AC93AD939493B993D6933E
:10D26800D793E893E593D893C393DD93D093C8936A
:10D27800E4931A9414941394039407941094369492
:10D288002B94359421943A944194529444945B9409
:10D29800609462945E946A942992709475947794D9
:10D2A8007D945A947C947E9481947F9482958795FA
:10D2B8008A959495969598959995A095A895A795EA
:10D2C800AD95BC95BB95B995BE95CA95F66FC395B6
:10D2D800CD95CC95D595D495D695DC95E195E595E4
:10D2E800E295219628962E962F9642964C964F9622
:10D2F8004B9677965C965E965D965F966696729666
:10D308006C968D96989695969796AA96A796B196A6
:10D31800B296B096B496B696B896B996CE96CB967F
:10D32800C996CD964D89DC960D97D596F9960497B2
:10D338000697089713970E9711970F9716971997AF
:10D3480024972A97309739973D973E974497469761
:10D358004897429749975C9760976497669768974C
:10D36800D2526B977197799785977C9781977A971F
:10D3780086978B978F9790979C97A897A697A39730
:10D38800B397B497C397C697C897CB97DC97ED9791
:10D398004F9FF297DF7AF697F5970F980C98389881
:10D3A8002498219837983D9846984F984B986B98B1
:10D3B8006F987098719874987398AA98AF98B19864
:10D3C800B698C498C398C698E998EB9803990999B0
:10D3D80012991499189921991D991E99249920999F
:10D3E8002C992E993D993E99429949994599509978
:10D3F8004B99519952994C99559997999899A599FA
:10D40800AD99AE99BC99DF99DB99DD99D899D199F5
:10D41800ED99EE99F199F299FB99F899019A0F9A79
:10D42800059AE299199A2B9A379A459A429A409AFC
:10D43800439A3E9A559A4D9A5B9A579A5F9A629A7E
:10D44800659A649A699A6B9A6A9AAD9AB09ABC9AE4
:10D45800C09ACF9AD19AD39AD49ADE9ADF9AE29A4E
:10D46800E39AE69AEF9AEB9AEE9AF49AF19AF79A77
:10D47800FB9A069B189B1A9B1F9B229B239B259B11
:10D48800279B289B299B2A9B2E9B2F9B329B449B47
:10D49800439B4F9B4D9B4E9B519B589B749B939BCF
:10D4A800839B919B969B979B9F9BA09BA89BB49BC0
:10D4B800C09BCA9BB99BC69BCF9BD19BD29BE39B2E
:10D4C800E29BE49BD49BE19B3A9CF29BF19BF09BF3
:10D4D800159C149C099C139C0C9C069C089C129CF3
:10D4E8000A9C049C2E9C1B9C259C249C219C309C63
:10D4F800479C329C469C3E9C5A9C609C679C769CB0
:10D50800789CE79CEC9CF09C099D089DEB9C039DF6
:10D51800069D2A9D269DAF9D239D1F9D449D159D7B
:10D52800129D419D3F9D3E9D469D489D5D9D5E9DF2
:10D53800649D519D509D599D729D899D879DAB9D70
:10D548006F9D7A9D9A9DA49DA99DB29DC49DC19DE4
:10D55800BB9DB89DBA9DC69DCF9DC29DD99DD39DAB
:10D56800F89DE69DED9DEF9DFD9D1A9E1B9E1E9EBE
:10D57800759E799E7D9E819E889E8B9E8C9E929E96
:10D58800959E919E9D9EA59EA99EB89EAA9EAD9E83
:10D598006197CC9ECE9ECF9ED09ED49EDC9EDE9E72
:10D5A800DD9EE09EE59EE89EEF9EF49EF69EF79E29
:10D5B800F99EFB9EFC9EFD9E079F089FB776159FD0
:10D5C800219F2C9F3E9F4A9F529F549F639F5F9F1E
:10D5D800609F619F669F679F6C9F6A9F779F729FFE
:10D5E800769F959F9C9FA09F2F58C76959906474F8
:10D5F800DC5199719C4E1655035A3F96C0541B61D5
:10D608002863F659229075841C83507AAA60E163D6
:10D61800256EED656684A682F59B93682757A165FC
:10D6280071629B5BD0597B86F498627DBE7D8E9B30
:10D6380016629F7CB788895BB55E09639766486800
:10D64800C7958D974F67E54E0A4F4D4F9D4F4950EF
:10D65800F2563759D459015A095CDF600F6170617D
:10D6680013660569BA704F757075FB79AD7DEF7DEE
:10D67800C3800E846388028B55907A903B53954EF5
:10D68800A54EDF57B280C190EF78004EF158A26ED8
:10D698003890327A28838B822F9C41517053BD5425
:10D6A800E154E056FB59155FF298EB6DE4802D8547
:10D6B80062967096A096FB970B54F353875BCF70D6
:10D6C800BD7FC28FE8966F535C9DBA7A114E9378EE
:10D6D800FC81266E185604551D6B1A853B9CE5592E
:10D6E800A953666DDC748F954256914E4B90F29615
:10D6F8004F830C99E153B655305B715F2066F36632
:10D708000468386CF36C296D5B74C8764E7A34986B
:10D71800F1825B88608AED92B26DAB75CA76C59965
:10D72800A660018B8A8DB2958E69AD5386511257CA
:10D7380030584459B45BF65E2860A963F463BF6C43
:10D74800146F8E7014715971D5713F73017E768292
:10D75800D182978560905B921B9D6958BC655A6C15
:10D768002575F9512E596559805FDC5FBC62FA65F1
:10D778002A6A276BB46B8B73C17F56892C9D0E9DCB
:10D78800C49EA15C966C7B8304514B5CB661C681D8
:10D7980076686172594EFA4F78536960296E4F7AEC
:10D7A800F3970B4E1653EE4E554F3D4FA14F734F07
:10D7B800A052EF5309560F59C15AB65BE15BD179B4
:10D7C80087669C67B6674C6BB36C6B70C2738D7958
:10D7D800BE793C7A877BB182DB8204837783EF83CF
:10D7E800D3836687B28A2956A88CE68F4E901E97F7
:10D7F8008A86C44FE85C116259723B75E581BD8227
:10D80800FE86C08CC5961399D599CB4E1A4FE389DD
:10D81800DE564A58CA58FB5EEB5F2A609460626025
:10D82800D0611262D0623965419B6666B068776DD7
:10D8380070704C758676757DA582F9878B958E9666
:10D848009D8CF151BE521659B354B35B165D686195
:10D858008269AF6D8D78CB845788728AA793B89AFE
:10D868006C6DA899D986A357FF67CE860E9283520E
:10D8780087560454D35EE162B9643C683868BB6B70
:10D888007273BA786B7A9A89D2896B8D038FED900F
:10D89800A39594966997665BB35C7D694D984E989D
:10D8A8009B63207B2B6A7F6AB6680D9C5F6F725200
:10D8B8009D557060EC623B6D076ED16E5B8410897C
:10D8C800448F144E399CF6531B693A6A84972A6828
:10D8D8005C51C37AB284DC918C935B56289D226894
:10D8E80005833184A57C0852C582E6747E4E834F39
:10D8F800A051D25B0A52D852E752FB5D9A552A587A
:10D90800E6598C5B985BDB5B725E795EA3601F6196
:10D918006361BE61DB636265D1675368FA683E6B19
:10D92800536B576C226F976F456FB0741875E37619
:10D938000B77FF7AA17B217CE97D367FF07F9D8084
:10D9480066829E83B389CC8AAB8C849051949395DC
:10D958009195A2956596D39728991882384E2B549D
:10D96800B85CCC5DA9734C763C77A95CEB7F0B8DDA
:10D97800C196119854985898014F0E4F71539C5561
:10D988006856FA574759095BC45B905C0C5E7E5E2B
:10D99800CC5FEE633A67D765E2651F67CB68C468FA
:10D9A8005F6A305EC56B176C7D6C7F754879635B09
:10D9B800007A007DBD5F8F89188AB48C778DCC8EF4
:10D9C8001D8FE2980E9A3C9B804E7D5000519359D2
:10D9D8009C5B2F628062EC643A6BA0729175477908
:10D9E800A97FFB87BC8A708BAC63CA83A097095454
:10D9F8000354AB555468586A708A27787567CD9E6A
:10DA08007453A25B1A8150860690184E454EC74E35
:10DA1800114FCA533854AE5B135F256051653D679B
:10DA2800426C726CE36C78700374767AAE7A087B19
:10DA38001A7DFE7C667DE7655B72BB53455CE85DDD
:10DA4800D262E0621963206E5A86318ADD8DF892BF
:10DA5800016FA6795A9BA84EAB4EAC4E9B4FA04F78
:10DA6800D1504751F67A7151F651545321537F538F
:10DA7800EB53AC558358E15C375F4A5F2F605060C9
:10DA88006D601F6359654B6AC16CC272ED72EF77A6
:10DA9800F880058108824E85F790E193FF975799A2
:10DAA8005A9AF04EDD512D5C81666D69405CF266D4
:10DAB800756989735068817CC550E4524757FE5D8B
:10DAC8002693A465236B3D6B34748179BD794B7BB8
:10DAD800CA7DB982CC837F885F89398BD18FD191F8
:10DAE8001F5480925D4E3650E5533A53D772967361
:10DAF800E977E682AF8EC699C899D29977511A61AB
:10DB08005E86B0557A7A7650D35B47908596324ECA
:10DB1800DB6AE791515C485C98639F7A936C7497D1
:10DB2800618FAA7A8A718896827C1768707E51689C
:10DB38006C93F2521B54AB85138AA47FCD8EE1906F
:10DB4800665388884179C24FBE501152445153558B
:10DB58002D57EA738B575159625F845F7560766100
:10DB68006761A961B2633A646C656F664268136E57
:10DB780066753D7AFB7C4C7D997D4B7E6B7F0E8371
:10DB88004A83CD86088A638A668BFD8E1A988F9D94
:10DB9800B882CE8FE89B87521F628364C06F9996C4
:10DBA80041689150206B7A6C546F747A507D40882C
:10DBB800238A0867F64E3950265065507C513852F2
:10DBC8006352A7550F570558CC5AFA5EB261F861EF
:10DBD800F36272631C69296A7D72AC722E731478C1
:10DBE8006F78797D0C77A9808B89198BE28CD28E1E
:10DBF800639075937A965598139A789E43519F53DC
:10DC0800B3537B5E265F1B6E906E8473FE73437DF9
:10DC18003782008AFA8A50964E4E0B50E4537C5451
:10DC2800FA56D159645BF15DAB5E275F3862456592
:10DC3800AF67566ED072CA7CB488A180E180F08349
:10DC48004E86878AE88D3792C7966798139F944EB9
:10DC5800924E0D4F485349543E542F5A8C5FA15F42
:10DC68009F60A7688E6A5A7481789E8AA48A778B87
:10DC780090915E4EC99BA44E7C4FAF4F19501650E1
:10DC880049516C519F52B952FE529A53E353115461
:10DC98000E5489555157A2577D59545B5D5B8F5B74
:10DCA800E55DE75DF75D785E835E9A5EB75E185F57
:10DCB80052604C619762D862A7633B65026643660F
:10DCC800F4666D6721689768CB695F6C2A6D696D2A
:10DCD8002F6E9D6E327587766C783F7AE07C057D75
:10DCE800187D5E7DB17D15800380AF80B180548141
:10DCF8008F812A8252834C8861881B8BA28CFC8C72
:10DD0800CA90759171923F78FC92A4954D960598AA
:10DD18009999D89A3B9D5B52AB52F7530854D55802
:10DD2800F762E06F6A8C5F8FB99E4B513B524A5441
:10DD3800FD56407A7791609DD29E4473096F708139
:10DD48001175FD5FDA60A89ADB72BC8F646B03986B
:10DD5800CA4EF0566457BE585A5A6860C7610F6673
:10DD680006663968B168F76DD5753A7D6E82429B53
:10DD78009B4E504FC95306556F5DE65DEE5DFB67E0
:10DD8800996C73740278508A9693DF885057A75E0F
:10DD98002B63B550AC508D510067C9545E58BB59C0
:10DDA800B05B695F4D62A1633D68736B086E7D70FF
:10DDB800C7918072157826786D798E65307DDC8301
:10DDC800C188098F9B966452285750676A7FA18C37
:10DDD800B45142572A963A588A69B480B2540E5DB3
:10DDE800FC579578FA9D5C4F4A528B543E642866DE
:10DDF8001467F567847A567B227D2F935C68AD9B08
:10DE0800397B19538A513752DF5BF662AE64E66498
:10DE18002D67BA6BA985D1969076D69B4C630693ED
:10DE2800AB9BBF765266094E9850C253715CE8604E
:10DE3800926463655F68E671CA732375977B827E17
:10DE48009586838BDB8C78911099AC65AB668B6B70
:10DE5800D54ED44E3A4F7F4F3A52F853F253E355CA
:10DE6800DB56EB58CB59C959FF59505B4D5C025EE4
:10DE78002B5ED75F1D6007632F655C5BAF65BD6573
:10DE8800E8659D67626B7B6B0F6C45734979C17957
:10DE9800F87C197D2B7DA2800281F38196895E8AA8
:10DEA800698A668A8C8AEE8AC78CDC8CCC96FC9848
:10DEB8006F6B8B4E3C4F8D4F5051575BFA5B4861EF
:10DEC80001634266216BCB6EBB6C3E72BD74D47528
:10DED800C1783A790C803380EA8194849E8F506CA3
:10DEE8007F9E0F5F588B2B9DFA7AF88E8D5BEB9691
:10DEF800034EF153F7573159C95AA45B89607F6EB5
:10DF0800066FBE75EA8C9F5B0085E07B7250F467F4
:10DF18009D82615C4A851E7E0E829951045C68630D
:10DF2800668D9C656E713E79177D05801D8BCA8E46
:10DF38006E90C786AA901F50FA523A5C53677C705D
:10DF480035724C91C8912B93E582C25B315FF960C1
:10DF58003B4ED653885B4B6231678A6BE972E0733C
:10DF68002E7A6B81A38D529196991251D7536A5488
:10DF7800FF5B8863396AAC7D0097DA56CE536854E4
:10DF8800975B315CDE5DEE4F0161FE62326DC079F8
:10DF9800CB79427D4D7ED27FED811F829084468869
:10DFA8007289908B748E2F8F31904B916C91C6969D
:10DFB8009C91C04E4F4F45514153935F0E62D467B9
:10DFC800416C0B6E6373267ECD918392D45319599D
:10DFD800BF5BD16D5D792E7E9B7C7E589F71FA5117
:10DFE8005388F08FCA4FFB5C2566AC77E37A1C82B6
:10DFF800FF99C651AA5FEC656F69896BF36D966EE0
:10E00800646FFE76147DE15D759087910698E65100
:10E018001D5240629166D9661A6EB65ED27D727FD5
:10E02800F866AF85F785F88AA952D95373598F5E78
:10E03800905F5560E4926496B7501F51DD522053AB
:10E048004753EC53E8544655315517566859BE594D
:10E058003C5AB55B065C0F5C115C1A5C845E8A5E98
:10E06800E05E705F7F628462DB628C637763076661
:10E078000C662D6676667E67A2681F6A356ABC6C78
:10E08800886D096E586E3C7126716771C775017786
:10E098005D7801796579F079E07A117BA77C397D23
:10E0A8009680D6838B8449855D88F3881F8A3C8A4D
:10E0B800548A738A618CDE8CA49166927E9318943C
:10E0C8009C9698970A4E084E1E4E574E975170527E
:10E0D800CE573458CC58225B385EC560FE64616701
:10E0E8005667446DB6727375637AB884728BB8914B
:10E0F80020933156F457FE98ED620D69966BED71D9
:10E10800547E77807282E689DF985587B18F3B5CB1
:10E11800384FE14FB54F0755205ADD5BE95BC35FC8
:10E128004E612F63B0654B66EE689B69786DF16D43
:10E138003375B9751F775E79E679337DE381AF82F0
:10E14800AA85AA893A8AAB8E9B8F3290DD91079770
:10E15800BA4EC14E03527558EC580B5C1A753D5CAB
:10E168004E810A8AC58F63966D97257BCF8A08985A
:10E178006291F356A853179039548257255EA863C5
:10E18800346C8A7061778B7CE07F70884290549100
:10E19800109318938F965E74C49A075D695D7065D5
:10E1A800A267A88DDB966E6349671969C5831798BE
:10E1B800C096FE88846F7A64F85B164E2C705D7585
:10E1C8002F66C4513652E252D359815F27601062DC
:10E1D8003F6574651F667466F2681668636B056E42
:10E1E80072721F75DB76BE7C5680F058FD887F8979
:10E1F800A08A938ACB8A1D909291529759978965E4
:10E208000E7A0681BB962D5EDC601A62A5651466DF
:10E218009067F3774D7A4D7C3E7E0A81AC8C648D95
:10E22800E18D5F8EA9780752D962A563426498622E
:10E238002D8A837AC07BAC8AEA96767D0C824987E0
:10E24800D94E485143536053A35B025C165CDD5DB5
:10E2580026624762B06413683468C96C456D176DEF
:10E26800D3675C6F4E717D71CB657F7AAD7BDA7D4C
:10E278004A7EA87F7A811B823982A6856E8ACE8CD7
:10E28800F58D78907790AD9291928395AE9B4D5293
:10E298008455386F367168518579557EB381CE7C47
:10E2A8004C565158A85CAA63FE66FD665A69D97235
:10E2B8008F758E750E795679DF79977C207D447D30
:10E2C8000786348A3B966190209FE7507552CC535D
:10E2D800E2530950AA55EE584F593D728B5B645C66
:10E2E8001D53E360F3605C6383633F63BB63CD648A
:10E2F800E965F966E35DCD69FD69156FE571894EDC
:10E30800E975F876937ADF7CCF7D9C7D61804983BF
:10E3180058836C84BC84FB85C588708D01906D9092
:10E3280097931C97129ACF5097588E61D381358551
:10E33800088D2090C34F7450475273536F604963E0
:10E348005F672C6EB38D1F90D74F5E5CCA8CCF650C
:10E358009A7D525396887651C363585B6B5B0A5C0F
:10E368000D6451675C90D64E1A592A59706C518ABF
:10E378003E551558A559F0605362C16735825569F5
:10E388004096C499289A534F0658FE5B1080B15C9A
:10E398002F5E855F20604B613462FF66F06CDE6E35
:10E3A800CE807F81D4828B88B88C00902E908A96FC
:10E3B800DB9EDB9BE34EF05327592C7B8D914C98C9
:10E3C800F99DDD6E277053534455855B58629E62F4
:10E3D800D362A26CEF6F2274178A3894C16FFE8AD9
:10E3E8003883E751F886EA53E953464F5490B08F83
:10E3F8006A593181FD5DEA7ABF8FDA68378CF87225
:10E40800489C3D6AB08A394E585306566657C562CD
:10E41800A263E6654E6BE16D5B6EAD70ED77EF7AEA
:10E42800AA7BBB7D3D80C680CB86958A5B93E356ED
:10E43800C7583E5FAD659666806AB56B3775C78A03
:10E448002450E57730571B5F65607A66606CF47519
:10E458001A7A6E7FF48118874590B399C97B5C75E9
:10E46800F97A517BC4841090E979927A3683E15A1B
:10E4780040772D4EF24E995BE05FBD623C66F167D6
:10E48800E86C6B8677883B8A4E91F392D099176A2D
:10E4980026702A73E7825784AF8C014E4651CB51C0
:10E4A8008B55F55B165E335E815E145F355F6B5F7F
:10E4B800B45FF2611163A2661D676E6F52723A759E
:10E4C8003A777480398178817687BF8ADC8A858D2E
:10E4D800F38D9A9277950298E59CC5525763F47626
:10E4E8001567886CCD73C38CAE937396256D9C5855
:10E4F8000E69CC69FD8F9A93DB751A905A58026899
:10E50800B463FB69434F2C6FD867BB8F2685B47DF6
:10E5180054933F69706F6A57F7582C5B2C7D2A72A9
:10E528000A54E391B49DAD4E4E4F5C507550435222
:10E538009E8C485424589A5B1D5E955EAD5EF75ECE
:10E548001F5F8C60B5623A63D063AF68406C8778B0
:10E558008E790B7AE07D4782028AE68A448E139090
:10E56800B8902D91D8910E9FE56C5864E26475655A
:10E57800F46E84761B7B6990D193BA6EF254B95FBE
:10E58800A4644D8FED8F449278516B582959555C8E
:10E59800975EFB6D8F7E1C75BC8CE28E5B98B970A4
:10E5A8001D4FBF6BB16F3075FB964E5110543558E7
:10E5B8005758AC59605C925F97655C67216E7B76B3
:10E5C800DF83ED8C1490FD904D9325783A78AA520C
:10E5D800A65E1F577459126012505A51AC51CD5152
:10E5E80000521055545858585759955BF65C8B5D36
:10E5F800BC6095622D6471674368BC68DF68D77634
:10E60800D86D6F6E9B6D6F70C871535FD8757779D1
:10E61800497B547B527BD67C717D305263846985FB
:10E62800E4850E8A048B468C0F8E03900F90199404
:10E6380076962D98309AD895CD50D5520C540258CC
:10E648000E5CA7619E641E6DB377E57AF48004843E
:10E6580053908592E05C079D3F53975FB35F9C6D35
:10E6680079726377BF79E47BD26BEC72AD8A036809
:10E67800616AF851817A34694A5CF69CEB82C55B21
:10E6880049911E7078566F5CC76066658C6C5A8CB1
:10E69800419013985154C7660D924859A3908551DB
:10E6A8004D4EEA5199850E8B58707A634B93626987
:10E6B800B499047E777557536069DF8EE3965D6C75
:10E6C8008C4E3C5C105FE98F0253D18C898079862F
:10E6D800FF5EE565734E655182593F5CEE97FB4ED0
:10E6E8008A59CD5F8D8AE16FB0796279E75B718471
:10E6F8002B73B171745EF55F7B639A64C371987C08
:10E70800434EFC5E4B4EDC57A256A960C36F0D7D8D
:10E71800FD803381BF81B28F9789A486F45D8A62B8
:10E72800AD6487897767E26C3E6D36743478465AF3
:10E73800757FAD82AC99F34FC35EDD629263576516
:10E748006F67C3764C72CC80BA80298F4D910D507B
:10E75800F957925A856873696471FD72B78CF258DB
:10E76800E08C6A9619907F87E479E77729842F4FA0
:10E7780065525A53CD62CF67CA6C7D76947B957C7F
:10E7880036828485EB8FDD66206F06721B7EAB8335
:10E79800C199A69EFD51B17B7278B87B8780487B72
:10E7A800E86A615E8C80517560756B5162928C6EFF
:10E7B8007A769791EA9A104F707F9C624F7BA59565
:10E7C800E99C7A565958E486BC96344F24524A53E9
:10E7D800CD53DB53065E2C6491657F673E6C4E6CAF
:10E7E8004872AF72ED735475417E2C82E985A98C0D
:10E7F800C47BC69169711298EF983D6369666A7522
:10E80800E476D0784385EE862A53515326548359AB
:10E81800875E7C5FB26049627962AB629065D46B57
:10E82800CC6CB275AE769178D879CB7D777FA580A0
:10E83800AB88B98ABB8C7F905E97DB980B6A387C73
:10E8480099503E5CAE5F8767D86B357409778E7FC9
:10E858003B9FCA67177A39538B75ED9A665F9D811E
:10E86800F18398803C5FC55F6275467B3C90676822
:10E87800EB599B5A107D7E762C8BF54F6A5F196A8F
:10E88800376C026FE27468796888558A798CDF5E24
:10E89800CF63C575D279D7822893F2929C84ED868E
:10E8A8002D9CC1546C5F8C655C6D1570A78CD38CE6
:10E8B8003B984F65F6740D4ED84EE0572B59665A63
:10E8C800CC5BA851035E9C5E166076627765A7658F
:10E8D8006E666E6D3672267B50819A8199825C8B4A
:10E8E800A08CE68C748D1C964496AE4FAB64666B18
:10E8F8001E8261846A85E890015C5369A8987A84CD
:10E9080057850F4F6F52A95F455E0D678F797981E3
:10E9180007898689F56D175F5562B86CCF4E6972A5
:10E92800929B06523B547456B358A4616E621A7196
:10E938006E59897CDE7C1B7DF09687655E80194E5A
:10E94800754F75514058635E735E0A5FC467264E03
:10E958003D8589955B96737C0198FB50C158567626
:10E96800A7782552A5771185867B4F50095947729C
:10E97800C77BE87DBA8FD48F4D90BF4FC952295AB3
:10E98800015FAD97DD4F1782EA9203575563696BB4
:10E998002B75DC88148F427ADF52935855610A62CE
:10E9A800AE66CD6B3F7CE9832350F84F0553465440
:10E9B800315849599D5BF05CEF5C295D965EB16208
:10E9C80067633E65B9650B67D56CE16CF9703278A1
:10E9D8002B7EDE80B3820C84EC84028712892A8A1B
:10E9E8004A8CA690D292FD98F39C6C9D4F4EA14EF6
:10E9F8008D5056524A57A8593D5ED85FD95F3F623D
:10EA0800B4661B67D067D2689251217DAA80A8811D
:10EA1800008B8C8CBF8C7E92329620542C98175386
:10EA2800D5505C53A858B264346767726677467AE3
:10EA3800E691C352A16C866B00584C5E54592C6702
:10EA4800FB7FE151C6766964E878549BBB9ECB573F
:10EA5800B95927669A67CE6BE954D969555E9C8186
:10EA68009567AA9BFE67529C5D68A64EE34FC85304
:10EA7800B9622B67AB6CC48FAD4F6D7EBF9E074EDE
:10EA88006261806E2B6F138573542A67459BF35D13
:10EA9800957BAC5CC65B1C874A6ED184147A08816E
:10EAA80099598D7C116C2077D952225921715F7246
:10EAB800DB772797619D0B697F5A185AA5510D542A
:10EAC8007D540E66DF76F78F9892F49CEA595D7252
:10EAD800C56E4D51C968BF7DEC7D6297BA9E78645A
:10EAE800216A028384595F5BDB6B1B73F276B27D0C
:10EAF8001780998432512867D99EEE766267FF5253
:10EB08000599245C3B627E7CB08C4F55B6600B7DCA
:10EB1800809501535F4EB6511C593A723680CE919A
:10EB2800255FE2778453795F047DAC85338A8D8EC7
:10EB38005697F367AE85539409610861B96C5276AC
:10EB4800ED8A388F2F55514F2A51C752CB53A55BA9
:10EB58007D5EA0608261D6630967DA67676E8C6D37
:10EB68003673377331755079D588988A4A90919061
:10EB7800F590C4968D871559884E594F0E4E898A3F
:10EB88003F8F1098AD507C5E9659B95BB85EDA63DA
:10EB9800FA63C164DC664A69D8690B6DB66E947114
:10EBA8002875AF7A8A7F00804984C9848189218B3E
:10EBB8000A8E65907D960A997E619162326B836CAC
:10EBC800746DCC7FFC7FC06D857FBA87F8886567D8
:10EBD800B1833C98F7961B6D617D3D846A91714EB7
:10EBE8007553505D046BEB6FCD852D86A78929522F
:10EBF8000F54655C4E67A86806748374E275CF8805
:10EC0800E188CC91E29678968B5F8773CB7A4E84B5
:10EC1800A06365758952416D9C6E097459756B784E
:10EC2800927C8696DC7A8D9FB64F6E61C5655C8650
:10EC3800864EAE4EDA50214ECC51EE5B9965816816
:10EC4800BC6D1F734276AD771C7AE77C6F82D28ADF
:10EC58007C90CF91759618989B52D17D2B509853E4
:10EC68009767CB6DD0713374E8812A8FA396579C30
:10EC78009F9E60744158996D2F7D5E98E44E364F83
:10EC88008B4FB751B152BA5D1C60B2733C79D382D5
:10EC98003492B796F6960A97979E629FA666746B0B
:10ECA8001752A352C870C288C95E4B609061236F27
:10ECB80049713E7CF47D6F80EE8423902C934254FE
:10ECC8006F9BD36A8970C28CEF8D3297B452415AC8
:10ECD800CA5E045F17677C6994696A6D0F6F627218
:10ECE800FC72ED7B01807E804B87CE906D51939EA8
:10ECF80084798B803293D68A2D508C54718A6A6BB2
:10ED0800C48C0781D160A067F29D994E984E109CE3
:10ED18006B8AC185688500697E6E97785581000089
:10ED2800002502250C251025182514251C252C2521
:10ED3800242534253C25012503250F2513251B25CE
:10ED48001725232533252B253B254B2520252F2526
:10ED5800282537253F251D253025252538254225F9
:10ED680010041104120413041404150401041604F5
:10ED78001704180419041A041B041C041D041E0497
:10ED88001F04200421042204230424042504260447
:10ED98002704280429042A042B042C042D042E04F7
:10EDA8002F04000000000000000000000000000028
:10EDB800000000000000000000000000000000004B
:10EDC8003004310432043304340435045104360465
:10EDD8003704380439043A043B043C043D043E0437
:10EDE8003F044004410442044304440445044604E7
:10EDF8004704480449044A044B044C044D044E0497
:10EE08004F04000091039203930394039503960320
:10EE18009703980399039A039B039C039D039E03FE
:10EE28009F03A003A103A303A403A503A603A703A9
:10EE3800A803A90300000000000000000000000073
:10EE480000000000B103B203B303B403B503B60373
:10EE5800B703B803B903BA03BB03BC03BD03BE03BE
:10EE6800BF03C003C103C303C403C503C603C70369
:10EE7800C803C903000000000000000000000000F3
:10EE88000000000101010101010101010100000070
:10EE9800000000000101010101010101010101015E
:10EEA800010101010101010101010101010100004C
:10EEB800000000000001010101010101010101013F
:10EEC800010101010101010101010101010101002B
:10EED800C625A125A025B325B225BD25BC253B20E7
:10EEE80012309221902191219321133000000000CB
:10EEF800000000000000000000000000000000000A
:10EF0800000008220B2286228722822283222A22BC
:10EF1800292200000000000000000000000000009E
:10EF2800000027222822AC00D221D421002203226B
:10EF3800292200000000000000000000000000007E
:10EF48000000000000002022A5221223022207222E
:10EF5800612252226A226B221A223D221D22352268
:10EF68002B222C22000000000000000000000000FE
:10EF780000002B2130206F266D266A2620202120B4
:10EF8800B6002C22000000000000EF250030013000
:10EF980002300CFF0EFFFB301AFF1BFF1FFF01FFA3
:10EFA8009B309C30B40040FFA8003EFF3E203FFF4E
:10EFB800FD30FE309D309E300330DD4E053006308A
:10EFC8000730FC30142010200FFF3CFF1C301620A7
:10EFD8005CFF26202520182019201C201D2008FF52
:10EFE80009FF143015303BFF3DFF5BFF5DFF083024
:10EFF80009300A300B300C300D300E300F30103025
:10F0080011300BFF1222B100D700F7001DFF60225C
:10F018001CFF1EFF662267221E223422422640263B
:10F02800B000322033200321A50004FFA200A30072
:10F0380005FF03FF06FF0AFF20FFA7000626052697
:10F04800CB25CF25CE25C7250000000000000000F5
:10F0580000000000000000000000000000000000A8
:10F068000000000000000000000000000000000098
:10F0780000000000000000001011121314151617EC
:10F088001819000000000000001A1B1C1D1E1F009C
:10F098000000000000000000000000000000000068
:10F0A8000000000000000000001A1B1C1D1E1F00AD
:10F0B8000000000000000000000000000000000048
:10F0C8000000000000000000000000000000000038
:10F0D8000000000000000000000000000000000028
:10F0E8000000000000000000000000000000000018
:10F0F8000000000000000000000000000000000008
:10F1080000000000000000000000000000000000F7
:10F1180000000000000000000000000000000000E7
:10F1280000000000000000000000000000000000D7
:10F1380000000000000000000000000000000000C7
:10F148000000000000000000050000001900000099
:10F158007D000000000000000080E03779C34143D3
:10F16800176E05B5B5B89346F5F93FE9034F384D25
:10F17800321D30F94877825A3CBF737FDD4F1575D1
:10F18800000000000000F03F0000000000002440E4
:10F1980000000000000059400000000000408F40BF
:10F1A800000000000088C34000000000006AF8402A
:10F1B8000000000080842E4100000000D01263414E
:10F1C8000000000084D797410000000065CDCD41C4
:10F1D800000000205FA00242000000E876483742A5
:10F1E800000000A2941A6D42000040E59C30A24243
:10F1F8000000901EC4BCD64200003426F56B0C43B8
:10F208000080E03779C3414300A0D885573476435E
:10F2180000C84E676DC1AB43003D9160E458E143BF
:10F22800408CB5781DAF154450EFE2D6E41A4B4434
:10F2380092D54D06CFF08044F64AE1C7022DB54479
:10F24800B49DD9794378EA44000000001F001C20CF
:10F258000000000014210000020016240000000035
:10F2680014250000020015280000000011290000E4
:10F278000000142A00000000182B00000000142CC5
:10F2880000000000102D00000000142E00000100F6
:10F298000C3000000900143A00000100183C00007E
:10F2A8000200143F00000100034100001900155B33
:10F2B80000000000145C00000000115D0000000068
:10F2C800175E000000000F5F0000000017600000DC
:10F2D8000000036100001900157B00000000187C85
:10F2E80000000000117D00000000187E00000000F2
:10F2F800007F000020001CA00000000014A10000F6
:10F30800000016A20000030019A60000000014A7C0
:10F318000000000017A80000000019A90000000064
:10F3280006AA0000000013AB0000000018AC0000A3
:10F33800000001AD0000000019AE0000000017AF8A
:10F348000000000019B00000000018B10000000023
:10F358000EB20000010017B40000000003B5000061
:10F36800000014B60000010017B8000000000EB934
:10F378000000000006BA0000000012BB00000000F8
:10F388000EBC0000020014BF0000000003C0000013
:10F39800160018D70000000003D80000060004DF9C
:10F3A8000000000003E00000160018F7000000004D
:10F3B80003F800003F000438010000000339010091
:10F3C8000F00044901000000034A01004200048DB7
:10F3D80001000000038E01000C00049B01000000E6
:10F3E800039C01000D0004AA0100010003AC010008
:10F3F8000D0004BA0100000006BB0100000003BCB8
:10F408000100010004BE0100000003BF010000006C
:10F4180006C00100030003C40100000007C5010085
:10F42800000003C60100010007C80100000003C96D
:10F438000100010007CB0100000003CC01002300FC
:10F4480004F00100000003F10100000007F20100D0
:10F45800000003F301002D00042102000000032234
:10F4680002001100043402000500033A02001A00E9
:10F47800045502000000035602000100045802006F
:10F488000000035902000000045A02000000035B58
:10F4980002000100045D0200020003600200010096
:10F4A800046202000000036302000000046402001A
:10F4B8000000036502000100046702000000036801
:10F4C80002000400046D02000100036F0200000046
:10F4D80004700200000003710200010004730200BE
:10F4E8000100037502000000047602000600037D97
:10F4F80002000000047E02000100038002000000F8
:10F50800048102000000038202000100048402005A
:10F518000200038702000500048D02000400039224
:10F52800020000000493020000000694020000009C
:10F53800049502000700039D02000100049F0200D9
:10F54800100005B00200110017C20200030005C632
:10F5580002000B0017D202000D0005E002000400B3
:10F5680017E50200060005EC0200000017ED020096
:10F57800000005EE0200000017EF020010000B006B
:10F5880003006F000370030003000574030000000C
:10F59800177503000000037603000100057A0300D5
:10F5A8000000037B03000200147E03000000037FB9
:10F5B8000300000017840300010003860300000015
:10F5C800148703000000038803000200038C030073
:10F5D8000000038E03000100049003000000039163
:10F5E8000300100003A303000C0004B00300000094
:10F5F80003B10300200008D20300020003D5030072
:10F60800200018F60300000003F70300040004FCC0
:10F618000300000003FD03008400198204000000B9
:10F628000B83040004000A8804000100038A040014
:10F63800A500033105002500055905000000145AEE
:10F6480005000500046005000000036105002500B1
:10F65800048705000100148905000000108A0500D0
:10F668000000198D05000100168F050000000B91A0
:10F6780005002C0010BE050000000BBF05000000AF
:10F6880014C0050000000BC10500010014C30500EB
:10F6980000000BC40500010014C6050000000BC7DC
:10F6A8000500000006D005001A0006EF050003005B
:10F6B80014F3050001000100060005001806060005
:10F6C8000200140906000100160B06000000140CC5
:10F6D80006000100190E060001000B1006000A00C2
:10F6E800141B06000000011C06000000141D060083
:10F6F8000200062006001F00054006000000064123
:10F70800060009000B4B060014000C6006000900F7
:10F71800146A06000300066E060001000B7006005E
:10F72800000006710600620014D40600000006D529
:10F73800060000000BD60600060001DD06000000EA
:10F7480019DE060000000BDF0600050005E50600CF
:10F7580001000BE70600010019E9060000000BEAAA
:10F768000600030006EE060001000CF00600090082
:10F7780006FA0600020019FD0600010006FF060051
:10F788000000140007000D00010F0700000006101C
:10F79800070000000B1107000000061207001D00FB
:10F7A8000B3007001A00064D070058000BA607008B
:10F7B8000A0006B1070000000CC00700090006CACD
:10F7C800070020000BEB0700080005F40700010004
:10F7D80019F60700000014F70700020005FA0700F1
:10F7E80000000BFD0700000016FE070001000600E0
:10F7F800080015000B1608000300051A0800000091
:10F808000B1B080008000524080000000B25080051
:10F8180002000528080000000B2908000400143025
:10F8280008000E000640080018000B5908000200E6
:10F83800145E08000000066008000A000670080050
:10F8480017001788080000000689080005000190C5
:10F85800080001000B980800070006A0080028000F
:10F8680005C9080000000BCA0800170001E20800DB
:10F8780000000BE308001F0009030900000006044C
:10F88800090035000B3A09000000093B0900000097
:10F898000B3C09000000063D09000000093E090074
:10F8A80002000B41090007000949090003000B4D3C
:10F8B80009000000094E0900010006500900000077
:10F8C8000B51090006000658090009000B620900DF
:10F8D80001001464090001000C6609000900147095
:10F8E80009000000057109000000067209000E00F9
:10F8F8000B81090000000982090001000685090042
:10F908000700068F0900010006930900150006AAE2
:10F918000900060006B20900000006B60900030047
:10F928000BBC0900000006BD0900000009BE090063
:10F9380002000BC10900030009C70900010009CB37
:10F94800090001000BCD0900000006CE09000000E7
:10F9580009D70900000006DC0900010006DF0900DC
:10F9680002000BE2090001000CE60900090006F09C
:10F978000900010016F2090001000EF40900050053
:10F9880019FA0900000016FB0900000006FC09002E
:10F99800000014FD090000000BFE090000000B0127
:10F9A8000A00010009030A00000006050A00050014
:10F9B800060F0A00010006130A001500062A0A00AD
:10F9C800060006320A00010006350A000100063862
:10F9D8000A0001000B3C0A000000093E0A00020070
:10F9E8000B410A0001000B470A0001000B4B0A00FB
:10F9F80002000B510A00000006590A000300065EC7
:10FA08000A0000000C660A0009000B700A000100D9
:10FA180006720A0002000B750A00000014760A003C
:10FA280000000B810A00010009830A000000068516
:10FA38000A000800068F0A00020006930A00150053
:10FA480006AA0A00060006B20A00010006B50A0066
:10FA580004000BBC0A00000006BD0A00000009BE35
:10FA68000A0002000BC10A0004000BC70A000100CB
:10FA780009C90A00000009CB0A0001000BCD0A00E1
:10FA8800000006D00A00000006E00A0001000BE2B0
:10FA98000A0001000CE60A00090014F00A00000040
:10FAA80016F10A00000006F90A0000000BFA0A0025
:10FAB80005000B010B00000009020B000100060500
:10FAC8000B000700060F0B00010006130B001500C2
:10FAD800062A0B00060006320B00010006350B0053
:10FAE80004000B3C0B000000063D0B000000093E23
:10FAF8000B0000000B3F0B00000009400B0000004A
:10FB08000B410B00030009470B000100094B0B00D8
:10FB180001000B4D0B0000000B550B0001000957AD
:10FB28000B000000065C0B000100065F0B000200E2
:10FB38000B620B0001000C660B00090019700B002A
:10FB4800000006710B0000000E720B0005000B820E
:10FB58000B00000006830B00000006850B00050063
:10FB6800068E0B00020006920B00030006990B009C
:10FB78000100069C0B000000069E0B00010006A376
:10FB88000B00010006A80B00020006AE0B000B00DC
:10FB980009BE0B0001000BC00B00000009C10B00DF
:10FBA800010009C60B00020009CA0B0002000BCDB8
:10FBB8000B00000006D00B00000009D70B00000066
:10FBC8000CE60B0009000EF00B00020019F30B0005
:10FBD800050016F90B00000019FA0B0000000B00D5
:10FBE8000C00000009010C0002000B040C000000CE
:10FBF80006050C000700060E0C00020006120C0099
:10FC08001600062A0C000F000B3C0C000000063DF5
:10FC18000C0000000B3E0C00020009410C00030020
:10FC28000B460C0002000B4A0C0003000B550C009D
:10FC3800010006580C000200065D0C00000006607A
:10FC48000C0001000B620C0001000C660C0009009E
:10FC580014770C0000000E780C000600197F0C00C9
:10FC6800000006800C0000000B810C0000000982D7
:10FC78000C00010014840C00000006850C0007002D
:10FC8800068E0C00020006920C00160006AA0C0054
:10FC9800090006B50C0004000BBC0C00000006BDF2
:10FCA8000C00000009BE0C0000000BBF0C00000097
:10FCB80009C00C0004000BC60C00000009C70C00AA
:10FCC800010009CA0C0001000BCC0C00010009D589
:10FCD8000C00010006DD0C00010006E00C0001002C
:10FCE8000BE20C0001000CE60C00090006F10C0008
:10FCF800010009F30C0000000B000D0001000902CF
:10FD08000D00010006040D000800060E0D0002009B
:10FD180006120D0028000B3B0D000100063D0D00EA
:10FD28000000093E0D0002000B410D0003000946CA
:10FD38000D000200094A0D0002000B4D0D000000E5
:10FD4800064E0D000000194F0D00000006540D006E
:10FD5800020009570D0000000E580D000600065F4E
:10FD68000D0002000B620D0001000C660D00090079
:10FD78000E700D00080019790D000000067A0D00BC
:10FD880005000B810D00000009820D0001000685A9
:10FD98000D001100069A0D00170006B30D000800AB
:10FDA80006BD0D00000006C00D0006000BCA0D00C0
:10FDB800000009CF0D0002000BD20D0002000BD687
:10FDC8000D00000009D80D0007000CE60D00090021
:10FDD80009F20D00010014F40D00000006010E00E8
:10FDE8002F000B310E00000006320E0001000B340C
:10FDF8000E000600163F0E00000006400E0005002B
:10FE080005460E0000000B470E000700144F0E00B9
:10FE180000000C500E000900145A0E000100068163
:10FE28000E00010006840E00000006860E00040085
:10FE3800068C0E00170006A50E00000006A70E008F
:10FE480009000BB10E00000006B20E0001000BB451
:10FE58000E00080006BD0E00000006C00E000400DB
:10FE680005C60E0000000BC80E0006000CD00E00E0
:10FE7800090006DC0E00030006000F00000019014F
:10FE88000F00020014040F000E0019130F000000E9
:10FE980014140F00000019150F0002000B180F00B2
:10FEA8000100191A0F0005000C200F0009000E2A86
:10FEB8000F00090019340F0000000B350F00000077
:10FEC80019360F0000000B370F00000019380F001B
:10FED80000000B390F000000153A0F000000113B1D
:10FEE8000F000000153C0F000000113D0F0000003E
:10FEF800093E0F00010006400F00070006490F00E9
:10FF080023000B710F000D00097F0F0000000B800C
:10FF18000F00040014850F0000000B860F0001007D
:10FF280006880F0004000B8D0F000A000B990F00C4
:10FF3800230019BE0F0007000BC60F00000019C7E9
:10FF48000F00050019CE0F00010014D00F000400A7
:10FF580019D50F00030014D90F0001000600100086
:10FF68002A00092B100001000B2D10000300093195
:10FF7800100000000B3210000500093810000000C6
:10FF88000B3910000100093B100001000B3D100067
:10FF98000100063F100000000C4010000900144A40
:10FFA8001000050006501000050009561000010059
:10FFB8000B5810000100065A100003000B5E1000D9
:10FFC80002000661100000000962100002000665C8
:10FFD80010000100096710000600066E10000200FC
:10FFE8000B7110000300067510000C000B82100046
:08FFF800000009831000010064
:020000041001E9
:100000000B85100001000987100005000B8D100002
:100010000000068E10000000098F100000000C90F8
:1000200010000900099A100002000B9D100000004A
:10003000199E1000010003A01000250003C7100046
:10004000000003CD1000000003D010002A0014FBB4
:100050001000000005FC1000000003FD100002006D
:10006000060011004801064A120003000650120063
:100070000600065812000000065A1200030006602F
:1000800012002800068A12000300069012002000C9
:1000900006B21200030006B81200060006C01200E5
:1000A000000006C21200030006C812000E0006D8A7
:1000B0001200380006121300030006181300420055
:1000C0000B5D130002001460130008000E6913009A
:1000D0001300068013000F0019901300090003A0FD
:1000E0001300550003F81300050010001400000071
:1000F000060114006B02196D16000000146E160044
:100100000000066F160010001C801600000006811B
:1001100016001900159B16000000119C1600000027
:1001200006A016004A0014EB160002000DEE1600A1
:10013000020006F1160007000600170011000B125E
:1001400017000200091517000000061F1700120013
:100150000B32170001000934170000001435170096
:1001600001000640170011000B5217000100066045
:1001700017000C00066E170002000B72170001003A
:100180000680170033000BB41700010009B61700F2
:1001900000000BB71700060009BE170007000BC6CA
:1001A0001700000009C7170001000BC917000A005B
:1001B00014D41700020005D71700000014D8170048
:1001C000020016DB1700000006DC170000000BDD44
:1001D000170000000CE0170009000EF017000900DE
:1001E000140018000500100618000000140718007D
:1001F00003000B0B18000200010E180000000B0F8B
:10020000180000000C101800090006201800220039
:10021000054318000000064418003400068018004A
:1002200004000B85180001000687180021000BA9A7
:100230001800000006AA1800000006B018004500CB
:10024000060019001E000B201900020009231900E6
:1002500003000B27190001000929190002000930C9
:10026000190001000B3219000000093319000500C4
:100270000B3919000200194019000000144419003C
:1002800001000C4619000900065019001D000670F7
:1002900019000400068019002B0006B0190019008F
:1002A0000CD0190009000EDA1900000019DE19003F
:1002B000210006001A0016000B171A000100091988
:1002C0001A0001000B1B1A000000141E1A00010086
:1002D00006201A00340009551A0000000B561A00B7
:1002E000000009571A0000000B581A0006000B60A6
:1002F0001A00000009611A0000000B621A000000D9
:1003000009631A0001000B651A000700096D1A0045
:1003100005000B731A0009000B7F1A0000000C8007
:100320001A0009000C901A00090014A01A00060017
:1003300005A71A00000014A81A0005000BB01A0047
:100340000D000ABE1A0000000BBF1A000F000B00C0
:100350001B00030009041B00000006051B002E0003
:100360000B341B00000009351B0000000B361B007E
:100370000400093B1B0000000B3C1B000000093D72
:100380001B0004000B421B00000009431B0001007E
:1003900006451B0007000C501B000900145A1B00E7
:1003A000060019611B0009000B6B1B000800197483
:1003B0001B000800147D1B0001000B801B000100C6
:1003C00009821B00000006831B001D0009A11B0001
:1003D00000000BA21B00030009A61B0001000BA8D4
:1003E0001B00010009AA1B0000000BAB1B00020050
:1003F00006AE1B0001000CB01B00090006BA1B0072
:100400002B000BE61B00000009E71B0000000BE8B7
:100410001B00010009EA1B0002000BED1B0000009D
:1004200009EE1B0000000BEF1B00020009F21B008D
:10043000010014FC1B00030006001C00230009241B
:100440001C0007000B2C1C00070009341C000100D5
:100450000B361C000100143B1C0004000C401C0067
:100460000900064D1C0002000C501C000900065A31
:100470001C001D0005781C000500147E1C000100F6
:1004800003801C00080003901C002A0003BD1C0010
:10049000020014C01C0007000BD01C00020014D383
:1004A0001C0000000BD41C000C0009E11C00000023
:1004B0000BE21C00060006E91C0003000BED1C000B
:1004C000000006EE1C0005000BF41C00000006F501
:1004D0001C00010009F71C0000000BF81C000100C3
:1004E00006FA1C00000004001D002B00052C1D0056
:1004F0003E00046B1D000C0005781D000000037910
:100500001D000000047A1D000200037D1D00000094
:10051000047E1D000F00038E1D000000048F1D00CF
:100520000B00059B1D0024000BC01D003F000300B5
:100530001E00950004961E000400039B1E00000090
:10054000049C1E000100039E1E000000049F1E006C
:10055000000003A01E00750003181F000500032003
:100560001F00250003481F00050004501F00000065
:1005700003511F00000004521F00000003531F001E
:10058000000004541F00000003551F000000045623
:100590001F00000003571F00000003591F00000048
:1005A000035B1F000000035D1F000000035F1F00CE
:1005B0001E0003801F00070007881F00070003902C
:1005C0001F00070007981F00070003A01F00070077
:1005D00007A81F00070003B01F00010004B21F009E
:1005E000000003B31F00000004B41F00000004B6A5
:1005F0001F00010003B81F00030007BC1F0000001C
:1006000017BD1F00000003BE1F00000017BF1F0022
:10061000020004C21F00000003C31F00000004C446
:100620001F00000004C61F00010003C81F000300D4
:1006300007CC1F00000017CD1F00020003D01F00D1
:10064000010004D21F00010004D61F00010003D8DE
:100650001F00030017DD1F00020003E01F00010060
:1006600004E21F00020003E51F00000004E61F0073
:10067000010003E81F00040017ED1F00020004F250
:100680001F00000003F31F00000004F41F0000001F
:1006900004F61F00010003F81F00030007FC1F0001
:1006A000000017FD1F0001001C0020000A00010BC4
:1006B0002000040010102000050014162000010086
:1006C000131820000000121920000000151A200045
:1006D0000000131B20000100121D20000000151E49
:1006E00020000000131F200000001420200007003D
:1006F0001A28200000001B2920000000012A2000E9
:1007000004001C2F200000001430200008001339C2
:1007100020000000123A20000000143B20000300DB
:100720000F3F200001001441200002001844200067
:10073000000015452000000011462000000014476D
:1007400020000A001852200000001453200000006E
:100750000F54200000001455200009001C5F2000E9
:1007600000000160200004000166200009000E70F6
:10077000200000000571200000000E74200005001C
:10078000187A20000200157D20000000117E200054
:100790000000057F200000000E8020000900188A5C
:1007A00020000200158D20000000118E20000000A6
:1007B000059020000C0016A0200020000BD0200087
:1007C0000C000ADD200003000BE1200000000AE21B
:1007D000200002000BE520000B00190021000100A1
:1007E000080221000000190321000300080721006E
:1007F0000000190821000100040A21000000080B74
:1008000021000200040E2100010008102100020056
:100810000413210000001914210000000815210014
:100820000000191621000100181821000000081905
:1008300021000400191E21000500082421000000E9
:10084000192521000000032621000000192721009E
:100850000000082821000000192921000000032AB7
:1008600021000100082C21000100192E21000000A8
:10087000042F210000000830210001000332210074
:100880000000083321000000043421000000063578
:1008900021000300043921000000193A2100010061
:1008A000043C21000100083E210001001840210005
:1008B0000400084521000000044621000300194AF5
:1008C00021000000184B21000000194C21000100FC
:1008D000034E21000000194F210000000E5021009E
:1008E0000F000D60210022000383210001000D850F
:1008F000210003000E8921000000198A2100010057
:10090000189021000400199521000400189A210074
:100910000100199C2100030018A02100000019A16A
:100920002100010018A32100000019A421000100EA
:1009300018A62100000019A72100060018AE21000A
:10094000000019AF21001E0018CE2100010019D0AF
:100950002100010018D22100000019D3210000005D
:1009600018D42100000019D521001E0018F4210020
:100970000B011900230007001508230000001109CE
:1009800023000000150A23000000110B23000000C3
:10099000190C230013001820230001001922230042
:1009A0000600152923000000112A23000000192B3E
:1009B00023005000187C23000000197D23001D0037
:1009C000189B2300180019B42300270018DC23000B
:1009D000050019E223004400194024000A000E60BB
:1009E00024003B00199C24004D000EEA2400150051
:1009F00019002500B60018B72500000019B8250019
:100A0000080018C12500000019C22500350018F89B
:100A100025000700190026006E00186F2600000050
:100A200019702600F70015682700000011692700DB
:100A30000000156A27000000116B27000000156CEC
:100A400027000000116D27000000156E2700000030
:100A5000116F27000000157027000000117127009A
:100A600000001572270000001173270000001574A4
:100A7000270000001175270000000E7627001D00DA
:100A8000199427002B0018C02700040015C5270063
:100A9000000011C62700000018C727001E0015E639
:100AA0002700000011E72700000015E827000000DC
:100AB00011E92700000015EA2700000011EB2700CC
:100AC000000015EC2700000011ED2700000015EED6
:100AD0002700000011EF2700000018F027000F008A
:100AE00019002800FF001800290082001583290042
:100AF00000001184290000001585290000001186DE
:100B00002900000015872900000011882900000035
:100B1000158929000000118A29000000158B290081
:100B20000000118C29000000158D29000000118E95
:100B300029000000158F29000000119029000000F5
:100B40001591290000001192290000001593290039
:100B5000000011942900000015952900000011964D
:100B600029000000159729000000119829000000B5
:100B7000189929003E0015D82900000011D9290034
:100B8000000015DA2900000011DB2900000018DC44
:100B900029001F0015FC2900000011FD290000009C
:100BA00018FE2900010119002B002F0018302B001E
:100BB000140019452B00010018472B000500194DA2
:100BC0002B00260019762B001F0019972B006800B8
:100BD00003002C00700004712C00000003722C0034
:100BE000010004742C00000003752C000100047740
:100BF0002C000400057C2C000100037E2C00650005
:100C000004E42C00000019E52C00050003EB2C0087
:100C100003000BEF2C00020003F22C00010014F97A
:100C20002C0003000EFD2C00000014FE2C0001001F
:100C300003002D00250003272D000000032D2D00AB
:100C4000000006302D003700056F2D0000001470E5
:100C50002D0000000B7F2D00000006802D001600E7
:100C600006A02D00060006A82D00060006B02D00E7
:100C7000060006B82D00060006C02D00060006C8B6
:100C80002D00060006D02D00060006D82D00060017
:100C90000BE02D001F0014002E00010013022E0097
:100CA000000012032E00000013042E0000001205A5
:100CB0002E00000014062E00020013092E00000072
:100CC000120A2E000000140B2E000000130C2E0040
:100CD0000000120D2E000000140E2E000800101748
:100CE0002E00000014182E000100101A2E00000023
:100CF000141B2E000000131C2E000000121D2E00DD
:100D00000000141E2E00010013202E0000001221EE
:100D10002E00000015222E00000011232E000000DE
:100D200015242E00000011252E00000015262E008F
:100D3000000011272E00000015282E0000001129A8
:100D40002E000000142A2E000400052F2E000000A3
:100D500014302E000900103A2E000100143C2E0021
:100D6000030010402E00000014412E000000154228
:100D70002E00000014432E000C0019502E0001001C
:100D800014522E00020015552E00000011562E00A0
:100D9000000015572E00000011582E0000001559B4
:100DA0002E000000115A2E000000155B2E000000DE
:100DB000115C2E000000105D2E00000019802E0036
:100DC0001900199B2E00580019002F00D50019F0AA
:100DD0002F000B001C003000000014013000020046
:100DE0001904300000000505300000000606300040
:100DF00000000D0730000000150830000000110948
:100E000030000000150A30000000110B3000000017
:100E1000150C30000000110D30000000150E3000E0
:100E20000000110F300000001510300000001111FB
:100E300030000000191230000100151430000000CD
:100E40001115300000001516300000001117300099
:100E50000000151830000000111930000000151AAC
:100E600030000000111B30000000101C300000009A
:100E7000151D30000000111E300001001920300047
:100E800000000D21300008000B2A30000300092E5D
:100E90003000010010303000000005313000040047
:100EA0001936300001000D3830000200053B3000DB
:100EB0000000063C30000000143D30000000193EE8
:100EC000300001000641300055000B993000010050
:100ED000179B30000100059D30000100069F300087
:100EE000000010A03000000006A13000590014FBE3
:100EF0003000000005FC3000020006FF300000005A
:100F0000060531002A00063131005D0019903100DC
:100F100001000E923100030019963100090006A06D
:100F200031001F0019C03100230006F031000F000E
:100F3000190032001E000E2032000900192A32006A
:100F40001D000E48320007001950320000000E51FB
:100F500032000E00196032001F000E8032000900BE
:100F6000198A320026000EB132000E0019C032007C
:100F70003F0106003400BF1919C04D003F000600B4
:100F80004E0014520515A00000000616A0007604BD
:100F90001990A400360006D0A400270005F8A4008C
:100FA000050014FEA40001000600A5000B01050CBD
:100FB000A6000000140DA60002000610A6000F00F7
:100FC0000C20A6000900062AA60001000340A60086
:100FD0002D00066EA60000000B6FA60000000A7030
:100FE000A60002001473A60000000B74A6000900FE
:100FF000147EA6000000057FA60000000380A60066
:101000001B00059CA60001000B9EA600010006A087
:10101000A60045000DE6A60009000BF0A6000100A1
:1010200014F2A60005001700A70016000517A70078
:1010300008001720A70001000322A7000D000430BC
:10104000A70001000332A7003D000570A7000000C3
:101050000471A70007000379A7000E000588A70008
:1010600000001789A7000100038BA7000200048E6F
:10107000A7000000068FA70000000390A70004004F
:101080000495A70000000396A700180004AFA7006E
:10109000000003B0A7001A0003D0A700010004D38A
:1010A000A700000004D5A700000003D6A700030096
:1010B00005F2A700020003F5A700010006F7A7004C
:1010C000000005F8A700010004FAA700000006FBD5
:1010D000A70006000B02A80000000603A8000200FB
:1010E0000B06A80000000607A80003000B0BA800D1
:1010F0000000060CA80016000923A80001000B251B
:10110000A80001000927A80000001928A800030072
:101110000B2CA80000000E30A80005001936A8000E
:1011200001001638A80000001939A8000000064088
:10113000A80033001474A80003000980A80001006F
:101140000682A800310009B4A8000F000BC4A80053
:10115000010014CEA80001000CD0A80009000BE08B
:10116000A800110006F2A800050014F8A80002006B
:1011700006FBA800000014FCA800000006FDA80063
:1011800001000BFFA80000000C00A9000900060ADE
:10119000A9001B000B26A9000700142EA9000100BE
:1011A0000630A90016000B47A9000A000952A90041
:1011B0000100145FA90000000660A9001C000B805C
:1011C000A90002000983A90000000684A9002E00DE
:1011D0000BB3A900000009B4A90001000BB6A900D7
:1011E000030009BAA90001000BBCA900010009BE57
:1011F000A900020014C1A9000C0005CFA90000003D
:101200000CD0A900090014DEA900010006E0A90025
:1012100004000BE5A900000005E6A900000006E7B0
:10122000A90008000CF0A900090006FAA9000400B2
:101230000600AA0028000B29AA000500092FAA0011
:1012400001000B31AA0001000933AA0001000B358F
:10125000AA0001000640AA0002000B43AA000000F9
:101260000644AA0007000B4CAA000000094DAA0082
:1012700000000C50AA000900145CAA0003000660DC
:10128000AA000F000570AA0000000671AA00050060
:101290001977AA000200067AAA000000097BAA00BA
:1012A00000000B7CAA000000097DAA000000067E59
:1012B000AA0031000BB0AA00000006B1AA0000008D
:1012C0000BB2AA00020006B5AA0001000BB7AA00E3
:1012D000010006B9AA0004000BBEAA00010006C066
:1012E000AA0000000BC1AA00000006C2AA0000006C
:1012F00006DBAA00010005DDAA00000014DEAA003A
:10130000010006E0AA000A0009EBAA0000000BECAD
:10131000AA00010009EEAA00010014F0AA000100D1
:1013200006F2AA00000005F3AA00010009F5AA00D0
:1013300000000BF6AA0000000601AB00050006093C
:10134000AB0005000611AB0005000620AB0006004F
:101350000628AB0006000430AB0022000353AB00AC
:1013600000000454AB000600175BAB000000055CF6
:10137000AB0003000460AB0008000569AB0000008F
:10138000176AAB0001000370AB004F0006C0AB0052
:10139000220009E3AB0001000BE5AB00000009E609
:1013A000AB0001000BE8AB00000009E9AB00010055
:1013B00014EBAB00000009ECAB0000000BEDAB0040
:1013C00000000CF0AB0009000600AC00A32B06B037
:1013D000D700160006CBD70030000200D800FF0768
:1013E0000600F9006D010670FA0069000400FB00B8
:1013F00006000413FB000400061DFB0000000B1E8A
:10140000FB000000061FFB0009001829FB0000007C
:10141000062AFB000C000638FB000400063EFB0019
:1014200000000640FB0001000643FB0001000646E9
:10143000FB006B0017B2FB00100006D3FB006A0133
:10144000113EFD000000153FFD0000001940FD00A9
:101450000F000650FD003F000692FD00350019CF39
:10146000FD00000006F0FD000B0016FCFD00000072
:1014700019FDFD0002000B00FE000F001410FE001D
:1014800006001517FE0000001118FE0000001419D8
:10149000FE0000000B20FE000F001430FE000000D4
:1014A0001031FE0001000F33FE0001001535FE0073
:1014B00000001136FE0000001537FE000000113854
:1014C000FE0000001539FE000000113AFE00000089
:1014D000153BFE000000113CFE000000153DFE0023
:1014E0000000113EFE000000153FFE00000011400C
:1014F000FE0000001541FE0000001142FE00000049
:101500001543FE0000001144FE0000001445FE00DB
:1015100001001547FE0000001148FE0000001449BC
:10152000FE0003000F4DFE0002001450FE000200FA
:101530001454FE0003001058FE0000001559FE0070
:101540000000115AFE000000155BFE000000115C57
:10155000FE000000155DFE000000115EFE000000B0
:10156000145FFE0002001862FE0000001063FE001F
:1015700000001864FE0002001468FE0000001669F6
:10158000FE000000146AFE0001000670FE00040068
:101590000676FE00860001FFFE0000001401FF0039
:1015A00002001604FF0000001405FF0002001508E9
:1015B000FF0000001109FF000000140AFF000000F6
:1015C000180BFF000000140CFF000000100DFF00BE
:1015D0000000140EFF0001000C10FF000900141A97
:1015E000FF000100181CFF000200141FFF00010093
:1015F0000321FF001900153BFF000000143CFF0011
:101600000000113DFF000000173EFF0000000F3FEB
:10161000FF0000001740FF0000000341FF00190019
:10162000155BFF000000185CFF000000115DFF006B
:101630000000185EFF000000155FFF000000116051
:10164000FF0000001461FF0000001562FF000000B1
:101650001163FF0000001464FF0001000666FF0034
:1016600009000570FF0000000671FF002C00059EB8
:10167000FF00010006A0FF001E0006C2FF000500DB
:1016800006CAFF00050006D2FF00050006DAFF00CB
:10169000020016E0FF00010018E2FF00000017E35F
:1016A000FF00000019E4FF00000016E5FF00010044
:1016B00019E8FF00000018E9FF00030019EDFF0022
:1016C000010001F9FF00020019FCFF000100060003
:1016D00000010B00060D0001190006280001120090
:1016E000063C00010100063F00010E00065000010B
:1016F0000D00068000017A001400010102000E07AF
:1017000001012C001937010108000D4001013400CE
:101710000E75010103001979010110000E8A010103
:101720000100198C01010200199001010C0019A09F
:101730000101000019D001012C000BFD0101000086
:10174000068002011C0006A0020130000BE002012D
:1017500000000EE102011A00060003011F000E2026
:1017600003010300062D030113000D4103010000D6
:101770000642030107000D4A030100000650030161
:1017800025000B7603010400068003011D00149F51
:101790000301000006A00301230006C8030107009F
:1017A00014D0030100000DD1030104000300040163
:1017B0004F00065004014D000CA00401090003B0C5
:1017C0000401230003D804012300060005012700BB
:1017D000063005013300146F050100000370050198
:1017E0000A00037C05010E00038C0501060003942A
:1017F00005010100039705010A0003A305010E007E
:1018000003B30501060003BB050101000600060144
:101810003601064007011500066007010700058034
:101820000701050005870701290005B20701080027
:10183000060008010500060808010000060A080164
:101840002B00063708010100063C08010000063F96
:10185000080116001457080100000E58080107007F
:101860000660080116001977080101000E790801C9
:101870000600068008011E000EA70801080006E009
:101880000801120006F4080101000EFB0801040023
:101890000600090115000E1609010500141F0901B3
:1018A0000000062009011900143F0901000006800C
:1018B000090137000EBC0901010006BE0901010043
:1018C0000EC009010F000ED209012D0006000A0109
:1018D00000000B010A0102000B050A0101000B0CBC
:1018E0000A01030006100A01030006150A0102009E
:1018F00006190A011C000B380A0102000B3F0A01FD
:1019000000000E400A01080014500A010800066099
:101910000A011C000E7D0A010100147F0A0100006B
:1019200006800A011C000E9D0A01020006C00A0181
:10193000070019C80A01000006C90A011B000BE5CF
:101940000A0101000EEB0A01040014F00A0106006E
:1019500006000B01350014390B01060006400B018F
:1019600015000E580B01070006600B0112000E78DF
:101970000B01070006800B01110014990B010300F5
:101980000EA90B01060006000C01480003800C01A3
:10199000320003C00C0132000EFA0C0105000600F3
:1019A0000D0123000B240D0103000C300D01090073
:1019B0000E600E011E0006800E0129000BAB0E0109
:1019C000010010AD0E01000006B00E0101000BFD7C
:1019D0000E01020006000F011C000E1D0F01090080
:1019E00006270F01000006300F0115000B460F01FE
:1019F0000A000E510F01030014550F010400067078
:101A00000F0111000B820F01030014860F01030068
:101A100006B00F0114000EC50F01060006E00F010D
:101A200016000900100100000B011001000009025E
:101A3000100100000603100134000B3810010E00E5
:101A40001447100106000E52100113000C6610011D
:101A500009000B70100100000671100101000B73EA
:101A6000100101000675100100000B7F100102003B
:101A7000098210010000068310012C0009B010013A
:101A800002000BB31001030009B7100101000BB9EC
:101A90001001010014BB1001010001BD1001000084
:101AA00014BE100103000BC21001000001CD100193
:101AB000000006D0100118000CF0100109000B0006
:101AC000110102000603110123000B27110104007C
:101AD000092C110100000B2D110107000C3611011A
:101AE00009001440110103000644110100000945DA
:101AF00011010100064711010000065011012200EA
:101B00000B7311010000147411010100067611011C
:101B100000000B8011010100098211010000068301
:101B200011012F0009B3110102000BB611010800C9
:101B300009BF1101010006C11101030014C5110103
:101B400003000BC91101030014CD1101000009CEDF
:101B5000110100000BCF110100000CD01101090090
:101B600006DA1101000014DB1101000006DC11018E
:101B7000000014DD110102000EE111011300060046
:101B800012011100061312011800092C12010200A3
:101B90000B2F120102000932120101000B34120155
:101BA00000000935120100000B3612010100143843
:101BB000120105000B3E12010000063F1201010058
:101BC0000B41120100000680120106000688120176
:101BD0000000068A12010300068F12010E00069F04
:101BE0001201090014A91201000006B012012E0012
:101BF0000BDF1201000009E0120102000BE31201E9
